 ProcList

 Timestamp is 5dd493dd (Wed Nov 20 04:16:13 2019)

 Preferred load address is 10000000

 Start         Length     Name                   Class
 0001:00000000 00000004H .CRT$XCA                CODE
 0001:00000004 00000004H .CRT$XCZ                CODE
 0001:00000008 00000004H .CRT$XIA                CODE
 0001:0000000c 0000000cH .CRT$XIC                CODE
 0001:00000018 00000004H .CRT$XIZ                CODE
 0001:0000001c 00000004H .CRT$XPA                CODE
 0001:00000020 00000008H .CRT$XPX                CODE
 0001:00000028 00000004H .CRT$XPXA               CODE
 0001:0000002c 00000004H .CRT$XPZ                CODE
 0001:00000030 00000004H .CRT$XTA                CODE
 0001:00000034 0000000cH .CRT$XTZ                CODE
 0001:00000038 00000000H .gfids$y                CODE
 0001:00000040 00006950H .rdata                  CODE
 0001:00006990 00000130H .rdata$r                CODE
 0001:00006ac0 0000000cH .rdata$sxdata           CODE
 0001:00006acc 0000029cH .rdata$zzzdbg           CODE
 0001:00006d68 00000004H .rtc$IAA                CODE
 0001:00006d6c 00000004H .rtc$IZZ                CODE
 0001:00006d70 00000004H .rtc$TAA                CODE
 0001:00006d74 0000000cH .rtc$TZZ                CODE
 0001:00006d80 000167e0H .text$mn                CODE
 0001:0001d557 00000000H .text$x                 CODE
 0001:0001d560 00000040H .text$yd                CODE
 0001:0001d5a0 00000470H .xdata$x                CODE
 0001:0001da10 00000192H .edata                  CODE
 0002:00000000 00000a40H .data                   DATA
 0002:00000a40 00000078H .data$r                 DATA
 0002:00000ab8 00025ab0H .bss                    DATA
 0003:00000000 0000022cH .idata$5                DATA
 0003:0000022c 00000004H .00cfg                  DATA
 0003:00000230 0000008cH .idata$2                DATA
 0003:000002bc 00000014H .idata$3                DATA
 0003:000002d0 0000022cH .idata$4                DATA
 0003:000004fc 00000986H .idata$6                DATA
 0004:00000000 00000060H .rsrc$01                DATA
 0004:00000060 00000378H .rsrc$02                DATA

  Address         Publics by Value              Rva+Base       Lib:Object

 0000:00000000       ___guard_iat_count         00000000     <absolute>
 0000:00000000       ___guard_longjmp_count     00000000     <absolute>
 0000:00000000       ___guard_fids_count        00000000     <absolute>
 0000:00000000       ___guard_longjmp_table     00000000     <absolute>
 0000:00000000       ___hybrid_code_map_count   00000000     <absolute>
 0000:00000000       __except_list              00000000     <absolute>
 0000:00000000       ___hybrid_auxiliary_iat    00000000     <absolute>
 0000:00000000       ___guard_fids_table        00000000     <absolute>
 0000:00000000       ___dynamic_value_reloc_table 00000000     <absolute>
 0000:00000000       ___guard_iat_table         00000000     <absolute>
 0000:00000000       ___volatile_metadata       00000000     <absolute>
 0000:00000000       ___enclave_config          00000000     <absolute>
 0000:00000000       ___hybrid_code_map         00000000     <absolute>
 0000:00000003       ___safe_se_handler_count   00000003     <absolute>
 0000:00000100       ___guard_flags             00000100     <absolute>
 0000:00000000       ___ImageBase               10000000     <linker-defined>
 0001:00000000       ___xc_a                    10001000     LIBCMT:initializers.obj
 0001:00000004       ___xc_z                    10001004     LIBCMT:initializers.obj
 0001:00000008       ___xi_a                    10001008     LIBCMT:initializers.obj
 0001:0000000c       ___acrt_multibyte_initializer 1000100c     libucrt:multibyte_initializer.obj
 0001:00000010       ___acrt_stdio_initializer  10001010     libucrt:stdio_initializer.obj
 0001:00000014       ___acrt_tran_sse2_initializer 10001014     libucrt:sse2_initializer.obj
 0001:00000018       ___xi_z                    10001018     LIBCMT:initializers.obj
 0001:0000001c       ___xp_a                    1000101c     LIBCMT:initializers.obj
 0001:00000020       ___acrt_locale_terminator  10001020     libucrt:locale_initializer.obj
 0001:00000024       ___dcrt_console_output_terminator 10001024     libucrt:console_output_initializer.obj
 0001:00000028       ___acrt_stdio_terminator   10001028     libucrt:stdio_initializer.obj
 0001:0000002c       ___xp_z                    1000102c     LIBCMT:initializers.obj
 0001:00000030       ___xt_a                    10001030     LIBCMT:initializers.obj
 0001:00000034       ___xt_z                    10001034     LIBCMT:initializers.obj
 0001:0000009c       ??_C@_11LOCGONAA@@         1000109c     handles.obj
 0001:000000a0       ??_C@_1BE@DNDHOCGP@?$AAD?$AAi?$AAr?$AAe?$AAc?$AAt?$AAo?$AAr?$AAy@ 100010a0     handles.obj
 0001:000000b4       ??_C@_1BK@KDPOKCA@?$AAS?$AAy?$AAm?$AAb?$AAo?$AAl?$AAi?$AAc?$AAL?$AAi?$AAn?$AAk@ 100010b4     handles.obj
 0001:000000d0       ??_C@_1M@JFPKKFCK@?$AAT?$AAo?$AAk?$AAe?$AAn@ 100010d0     handles.obj
 0001:000000dc       ??_C@_1BA@NMDNJJOO@?$AAP?$AAr?$AAo?$AAc?$AAe?$AAs?$AAs@ 100010dc     handles.obj
 0001:000000ec       ??_C@_1O@CDOGJPJJ@?$AAT?$AAh?$AAr?$AAe?$AAa?$AAd@ 100010ec     handles.obj
 0001:000000fc       ??_C@_1M@JJBFPLJB@?$AAE?$AAv?$AAe?$AAn?$AAt@ 100010fc     handles.obj
 0001:00000108       ??_C@_1BE@EBMGBMON@?$AAE?$AAv?$AAe?$AAn?$AAt?$AAP?$AAa?$AAi?$AAr@ 10001108     handles.obj
 0001:0000011c       ??_C@_1O@FBKOCLFA@?$AAM?$AAu?$AAt?$AAa?$AAn?$AAt@ 1000111c     handles.obj
 0001:0000012c       ??_C@_1BE@NPGPGCB@?$AAS?$AAe?$AAm?$AAa?$AAp?$AAh?$AAo?$AAr?$AAe@ 1000112c     handles.obj
 0001:00000140       ??_C@_1M@EEEEDEMN@?$AAT?$AAi?$AAm?$AAe?$AAr@ 10001140     handles.obj
 0001:0000014c       ??_C@_1BA@OKEJPPOI@?$AAP?$AAr?$AAo?$AAf?$AAi?$AAl?$AAe@ 1000114c     handles.obj
 0001:0000015c       ??_C@_1BM@JIPCCEDL@?$AAW?$AAi?$AAn?$AAd?$AAo?$AAw?$AAS?$AAt?$AAa?$AAt?$AAi?$AAo?$AAn@ 1000115c     handles.obj
 0001:00000178       ??_C@_1BA@CBCBMBGJ@?$AAD?$AAe?$AAs?$AAk?$AAt?$AAo?$AAp@ 10001178     handles.obj
 0001:00000188       ??_C@_1BA@LHDKDEEN@?$AAS?$AAe?$AAc?$AAt?$AAi?$AAo?$AAn@ 10001188     handles.obj
 0001:00000198       ??_C@_17KACEIPNC@?$AAK?$AAe?$AAy@ 10001198     handles.obj
 0001:000001a0       ??_C@_19OBNDINH@?$AAP?$AAo?$AAr?$AAt@ 100011a0     handles.obj
 0001:000001ac       ??_C@_1BK@GACLFIOK@?$AAW?$AAa?$AAi?$AAt?$AAa?$AAb?$AAl?$AAe?$AAP?$AAo?$AAr?$AAt@ 100011ac     handles.obj
 0001:000001c8       ??_C@_17EKANHMLE@?$AAJ?$AAo?$AAb@ 100011c8     handles.obj
 0001:000001d0       ??_C@_1BK@HCMNLOAL@?$AAI?$AAo?$AAC?$AAo?$AAm?$AAp?$AAl?$AAe?$AAt?$AAi?$AAo?$AAn@ 100011d0     handles.obj
 0001:000001ec       ??_C@_19DDLLJDOO@?$AAF?$AAi?$AAl?$AAe@ 100011ec     handles.obj
 0001:000001f8       ??_C@_1BA@KLFBJALL@?$AAW?$AAm?$AAi?$AAG?$AAu?$AAi?$AAd@ 100011f8     handles.obj
 0001:00000208       ??_C@_17CNPHIMPH@?$AA?$CF?$AAl?$AAs@ 10001208     handles.obj
 0001:00000210       ??_C@_1BE@ELICABCK@?$AA?$DM?$AAu?$AAn?$AAk?$AAn?$AAo?$AAw?$AAn?$AA?$DO@ 10001210     handles.obj
 0001:00000224       ??_C@_1BA@FDFONNEJ@?$AA?$CF?$AAs?$AA?5?$AA?$CI?$AA?$CF?$AAd?$AA?$CJ@ 10001224     handles.obj
 0001:00000234       ??_C@_1BA@LGCEDAAB@?$AAT?$AAI?$AAD?$AA?3?$AA?5?$AA?$CF?$AAd@ 10001234     handles.obj
 0001:00000244       ??_C@_1BG@OKCBELMP@?$AA?2?$AAR?$AAE?$AAG?$AAI?$AAS?$AAT?$AAR?$AAY?$AA?2@ 10001244     handles.obj
 0001:0000025c       ??_C@_19KGHAHCFG@?$AAU?$AAS?$AAE?$AAR@ 1000125c     handles.obj
 0001:00000268       ??_C@_19JAPAIJDE@?$AAH?$AAK?$AAC?$AAU@ 10001268     handles.obj
 0001:00000274       ??_C@_1BC@PGMOPNLK@?$AA_?$AAC?$AAl?$AAa?$AAs?$AAs?$AAe?$AAs@ 10001274     handles.obj
 0001:00000288       ??_C@_1BK@OEABCBLA@?$AAH?$AAK?$AAC?$AAU?$AA?2?$AAC?$AAl?$AAa?$AAs?$AAs?$AAe?$AAs@ 10001288     handles.obj
 0001:000002a4       ??_C@_17PJOJPMPB@?$AAH?$AAK?$AAU@ 100012a4     handles.obj
 0001:000002ac       ??_C@_1DC@OIDKFHBF@?$AAM?$AAA?$AAC?$AAH?$AAI?$AAN?$AAE?$AA?2?$AAS?$AAO?$AAF?$AAT?$AAW?$AAA?$AAR@ 100012ac     handles.obj
 0001:000002e0       ??_C@_19NCHLBIN@?$AAH?$AAK?$AAC?$AAR@ 100012e0     handles.obj
 0001:000002ec       ??_C@_1BA@INBMCOAP@?$AAM?$AAA?$AAC?$AAH?$AAI?$AAN?$AAE@ 100012ec     handles.obj
 0001:000002fc       ??_C@_19PEALEEJB@?$AAH?$AAK?$AAL?$AAM@ 100012fc     handles.obj
 0001:00000308       ??_C@_15GANGMFKL@?$AA?$CF?$AAs@ 10001308     handles.obj
 0001:00000310       ??_C@_1O@EAOKCHFC@?$AA?$CF?$AA?9?$AA1?$AA3?$AAs?$AA?5@ 10001310     handles.obj
 0001:00000320       ??_C@_1O@HAOIKAHJ@?$AA?$CF?$AAs?$AA?6?$AA?$CF?$AAs?$AA?6@ 10001320     handles.obj
 0001:00000330       ??_C@_1BG@OCPCMCEA@?$AA?$CF?$AA5?$AAX?$AA?5?$AA?5?$AA?$CF?$AA0?$AA8?$AAX?$AA?5@ 10001330     handles.obj
 0001:00000348       ??_C@_1BA@IGEMANKH@?$AA?2?$AAS?$AA?9?$AA?$CF?$AAl?$AAu?$AA?9@ 10001348     handles.obj
 0001:00000358       ??_C@_1EC@MPDKEHCN@?$AA0?$AAx?$AA?$CF?$AA0?$AA2?$AAh?$AAx?$AA?$CF?$AA0?$AA2?$AAh?$AAx?$AA?$CF?$AA0?$AA2@ 10001358     handles.obj
 0001:0000039c       ??_C@_17IJMNDCL@?$AA?$CF?$AAl?$AAu@ 1000139c     handles.obj
 0001:000003a4       ??_C@_19DEJHOMFE@?$AA?9?$AA?$CF?$AAl?$AAu@ 100013a4     handles.obj
 0001:000003b0       ??_7?$DialogItemBinding@UFarDialogItem@@@@6B@ 100013b0     PCFG.OBJ
 0001:000003b8       ??_7PluginCheckBoxBinding@@6B@ 100013b8     PCFG.OBJ
 0001:000003c0       ??_7PluginRadioButtonBinding@@6B@ 100013c0     PCFG.OBJ
 0001:000003c8       ??_7PluginIntEditFieldBinding@@6B@ 100013c8     PCFG.OBJ
 0001:000003d0       ??_C@_15EFLNJKHH@?$AA?$CF?$AAu@ 100013d0     PCFG.OBJ
 0001:000003d8       ??_7PluginUIntEditFieldBinding@@6B@ 100013d8     PCFG.OBJ
 0001:000003e0       ??_7?$DialogBuilderBase@UFarDialogItem@@@@6B@ 100013e0     PCFG.OBJ
 0001:00000404       ??_7PluginDialogBuilder@@6B@ 10001404     PCFG.OBJ
 0001:00000428       ??_C@_1O@BJPKKLLM@?$AAC?$AAo?$AAn?$AAf?$AAi?$AAg@ 10001428     PCFG.OBJ
 0001:00000438       ??_C@_1BO@NGDOFANC@?$AAA?$AAd?$AAd?$AAT?$AAo?$AAD?$AAi?$AAs?$AAk?$AAs?$AAM?$AAe?$AAn?$AAu@ 10001438     PCFG.OBJ
 0001:00000458       ??_C@_1CC@PNNAOHJC@?$AAA?$AAd?$AAd?$AAT?$AAo?$AAP?$AAl?$AAu?$AAg?$AAi?$AAn?$AAs?$AAM?$AAe?$AAn@ 10001458     PCFG.OBJ
 0001:0000047c       ??_C@_1CE@JIPJNDMD@?$AAE?$AAx?$AAp?$AAo?$AAr?$AAt?$AAE?$AAn?$AAv?$AAi?$AAr?$AAo?$AAn?$AAm?$AAe@ 1000147c     PCFG.OBJ
 0001:000004a0       ??_C@_1CC@OABICAMP@?$AAE?$AAx?$AAp?$AAo?$AAr?$AAt?$AAM?$AAo?$AAd?$AAu?$AAl?$AAe?$AAI?$AAn?$AAf@ 100014a0     PCFG.OBJ
 0001:000004c4       ??_C@_1CI@OFLGHPDG@?$AAE?$AAx?$AAp?$AAo?$AAr?$AAt?$AAM?$AAo?$AAd?$AAu?$AAl?$AAe?$AAV?$AAe?$AAr@ 100014c4     PCFG.OBJ
 0001:000004ec       ??_C@_1CE@GNMOKOAL@?$AAE?$AAx?$AAp?$AAo?$AAr?$AAt?$AAP?$AAe?$AAr?$AAf?$AAo?$AAr?$AAm?$AAa?$AAn@ 100014ec     PCFG.OBJ
 0001:00000510       ??_C@_1BM@KMCHODLM@?$AAE?$AAx?$AAp?$AAo?$AAr?$AAt?$AAH?$AAa?$AAn?$AAd?$AAl?$AAe?$AAs@ 10001510     PCFG.OBJ
 0001:0000052c       ??_C@_1CK@CLFOOHFA@?$AAE?$AAx?$AAp?$AAo?$AAr?$AAt?$AAH?$AAa?$AAn?$AAd?$AAl?$AAe?$AAs?$AAU?$AAn@ 1000152c     PCFG.OBJ
 0001:00000558       ??_C@_1BE@PKILIDFH@?$AAE?$AAn?$AAa?$AAb?$AAl?$AAe?$AAW?$AAM?$AAI@ 10001558     PCFG.OBJ
 0001:0000056c       ??_7PluginEditFieldBinding@@6B@ 1000156c     Pclass.obj
 0001:00000574       ??_C@_13JCKOPPNP@?$AAK@    10001574     Pclass.obj
 0001:00000578       ??_C@_13LHMFKAAD@?$AAM@    10001578     Pclass.obj
 0001:0000057c       ??_C@_1BC@IALIJCAM@?$AAS?$AAo?$AAr?$AAt?$AAM?$AAo?$AAd?$AAe@ 1000157c     Pclass.obj
 0001:00000590       ??_C@_1BO@OMKAPLPJ@?$AAS?$AAt?$AAa?$AAr?$AAt?$AAP?$AAa?$AAn?$AAe?$AAl?$AAM?$AAo?$AAd?$AAe@ 10001590     Pclass.obj
 0001:00000620       ??_C@_1CM@OLKFIHMK@?$AAN?$AA?0?$AAX?$AA1?$AA5?$AAT?$AA?0?$AAX?$AA1?$AA6?$AAT?$AA?0?$AAX?$AA1?$AA7@ 10001620     Pclass.obj
 0001:0000064c       ??_C@_1BG@MNPGDOEP@?$AA1?$AA2?$AA?0?$AA0?$AA?0?$AA0?$AA?0?$AA0?$AA?0?$AA4@ 1000164c     Pclass.obj
 0001:00000664       ??_C@_1CE@JPABPOMI@?$AAN?$AA?0?$AAX?$AAI?$AA?0?$AAX?$AAB?$AA?0?$AAX?$AAP?$AA?0?$AAX?$AA0?$AAS?$AA?0@ 10001664     Pclass.obj
 0001:00000688       ??_C@_1BI@EFANNANC@?$AA0?$AA?0?$AA6?$AA?0?$AA2?$AA?0?$AA2?$AA?0?$AA3?$AA?0?$AA9@ 10001688     Pclass.obj
 0001:000006a0       ??_C@_17KNGPBKAK@?$AAN?$AA?0?$AAN@ 100016a0     Pclass.obj
 0001:000006a8       ??_C@_17JPFFEOAH@?$AA0?$AA?0?$AA0@ 100016a8     Pclass.obj
 0001:000006b0       ??_C@_1BO@JAFIOFIL@?$AAN?$AA?0?$AAX?$AAI?$AA?0?$AAX?$AAB?$AA?0?$AAX?$AAC?$AA?0?$AAD?$AA?0?$AAT@ 100016b0     Pclass.obj
 0001:000006d0       ??_C@_1BI@LFIMKDME@?$AA0?$AA?0?$AA6?$AA?0?$AA2?$AA?0?$AA6?$AA?0?$AA0?$AA?0?$AA0@ 100016d0     Pclass.obj
 0001:000006e8       ??_C@_1BG@MICALLFD@?$AAN?$AA?0?$AAX?$AAI?$AA?0?$AAX?$AA4?$AA?0?$AAX?$AA6@ 100016e8     Pclass.obj
 0001:00000700       ??_C@_1BA@MMHHFCDG@?$AA0?$AA?0?$AA6?$AA?0?$AA9?$AA?0?$AA9@ 10001700     Pclass.obj
 0001:00000710       ??_C@_1DI@NKOPFHII@?$AAN?$AA?0?$AAX?$AAI?$AA?0?$AAX?$AA4?$AA?0?$AAX?$AA6?$AA?0?$AAX?$AA1?$AA0?$AA?0@ 10001710     Pclass.obj
 0001:00000748       ??_C@_1CG@EOFMIEJC@?$AA1?$AA2?$AA?0?$AA6?$AA?0?$AA0?$AA?0?$AA0?$AA?0?$AA0?$AA?0?$AA0?$AA?0?$AA8?$AA?0@ 10001748     Pclass.obj
 0001:00000770       ??_C@_19ILLMDDHI@?$AAN?$AA?0?$AAZ?$AAD@ 10001770     Pclass.obj
 0001:0000077c       ??_C@_19NMOJBHGD@?$AA1?$AA2?$AA?0?$AA0@ 1000177c     Pclass.obj
 0001:00000788       ??_C@_1EA@HPDEOPPH@?$AAN?$AA?0?$AAX?$AAP?$AA?0?$AAX?$AA0?$AAS?$AA?0?$AAX?$AA1?$AAS?$AA?0?$AAX?$AA2@ 10001788     Pclass.obj
 0001:000007c8       ??_C@_1CA@MGMNHCLL@?$AA0?$AA?0?$AA2?$AA?0?$AA3?$AA?0?$AA2?$AA?0?$AA2?$AA?0?$AA3?$AA?0?$AA4?$AA?0?$AA3@ 100017c8     Pclass.obj
 0001:000007e8       ??_C@_1O@JGFFCAGM@?$AAN?$AA?0?$AAX?$AAI?$AA?0?$AAO@ 100017e8     Pclass.obj
 0001:000007f8       ??_C@_1O@FLEOANAI@?$AA0?$AA?0?$AA6?$AA?0?$AA1?$AA5@ 100017f8     Pclass.obj
 0001:00000808       ??_C@_1CC@FANCGEGE@?$AAN?$AA?0?$AAX?$AAI?$AA?0?$AAX?$AAT?$AA?0?$AAX?$AA3?$AA?0?$AAX?$AAG?$AA?0?$AAX@ 10001808     Pclass.obj
 0001:0000082c       ??_C@_1BI@PMPHDFGH@?$AA0?$AA?0?$AA6?$AA?0?$AA3?$AA?0?$AA4?$AA?0?$AA4?$AA?0?$AA4@ 1000182c     Pclass.obj
 0001:00000898       ??_C@_1BG@COBJEPBB@?$AAN?$AA?0?$AAX?$AAI?$AA?0?$AAX?$AAT?$AA?0?$AAX?$AA3@ 10001898     Pclass.obj
 0001:000008b0       ??_C@_1BA@KPNNJGCD@?$AA0?$AA?0?$AA6?$AA?0?$AA3?$AA?0?$AA4@ 100018b0     Pclass.obj
 0001:000008c0       ??_C@_1O@CBODAMOP@?$AAM?$AAo?$AAd?$AAe?$AA?$CF?$AAd@ 100018c0     Pclass.obj
 0001:000008d0       ??_C@_1CA@HLBJOHGN@?$AAF?$AAu?$AAl?$AAl?$AAS?$AAc?$AAr?$AAe?$AAe?$AAn?$AAL?$AAo?$AAc?$AAa?$AAl@ 100018d0     Pclass.obj
 0001:000008f0       ??_C@_1CC@EBBNDNOD@?$AAF?$AAu?$AAl?$AAl?$AAS?$AAc?$AAr?$AAe?$AAe?$AAn?$AAR?$AAe?$AAm?$AAo?$AAt@ 100018f0     Pclass.obj
 0001:00000914       ??_C@_1BK@HMOODHKK@?$AAC?$AAo?$AAl?$AAu?$AAm?$AAn?$AAs?$AAL?$AAo?$AAc?$AAa?$AAl@ 10001914     Pclass.obj
 0001:00000930       ??_C@_1BM@EDHFKJEJ@?$AAC?$AAo?$AAl?$AAu?$AAm?$AAn?$AAs?$AAR?$AAe?$AAm?$AAo?$AAt?$AAe@ 10001930     Pclass.obj
 0001:0000094c       ??_C@_1BI@FOOHDOCI@?$AAW?$AAi?$AAd?$AAt?$AAh?$AAs?$AAL?$AAo?$AAc?$AAa?$AAl@ 1000194c     Pclass.obj
 0001:00000964       ??_C@_1BK@DDBMMJCN@?$AAW?$AAi?$AAd?$AAt?$AAh?$AAs?$AAR?$AAe?$AAm?$AAo?$AAt?$AAe@ 10001964     Pclass.obj
 0001:00000980       ??_C@_13DEFPDAGF@?$AA?0@   10001980     Pclass.obj
 0001:00000984       ??_C@_15LNKNCLHH@?$AAS?$AAs@ 10001984     Pclass.obj
 0001:0000098c       ??_C@_1BA@MFHNOFIJ@?$AA?$CF?$AAs?$AA?3?$AA?5?$AA?$CF?$AAs?$AA?5@ 1000198c     Pclass.obj
 0001:0000099c       ??_C@_19MPDKCIDK@?$AA?5?$AA?$CF?$AAs?$AA?5@ 1000199c     Pclass.obj
 0001:000009a8       ??_C@_15JOGBDECP@?$AA?0?$AA?5@ 100019a8     Pclass.obj
 0001:000009b0       ??_C@_15DNHPCDHG@?$AAT?$AAt@ 100019b0     Pclass.obj
 0001:00000a50       ??_C@_1BC@OMEIHGFC@?$AAW?$AAS?$AA_?$AAP?$AAO?$AAP?$AAU?$AAP@ 10001a50     Pclass.obj
 0001:00000a64       ??_C@_1BC@ONEEOLLM@?$AAW?$AAS?$AA_?$AAC?$AAH?$AAI?$AAL?$AAD@ 10001a64     Pclass.obj
 0001:00000a78       ??_C@_1BI@GHDIGAD@?$AAW?$AAS?$AA_?$AAM?$AAI?$AAN?$AAI?$AAM?$AAI?$AAZ?$AAE@ 10001a78     Pclass.obj
 0001:00000a90       ??_C@_1BG@KLPFHNBP@?$AAW?$AAS?$AA_?$AAV?$AAI?$AAS?$AAI?$AAB?$AAL?$AAE@ 10001a90     Pclass.obj
 0001:00000aa8       ??_C@_1BI@NKODCGOF@?$AAW?$AAS?$AA_?$AAD?$AAI?$AAS?$AAA?$AAB?$AAL?$AAE?$AAD@ 10001aa8     Pclass.obj
 0001:00000ac0       ??_C@_1CA@PCFJBBHH@?$AAW?$AAS?$AA_?$AAC?$AAL?$AAI?$AAP?$AAS?$AAI?$AAB?$AAL?$AAI?$AAN?$AAG?$AAS@ 10001ac0     Pclass.obj
 0001:00000ae0       ??_C@_1CA@MPLGGIO@?$AAW?$AAS?$AA_?$AAC?$AAL?$AAI?$AAP?$AAC?$AAH?$AAI?$AAL?$AAD?$AAR?$AAE?$AAN@ 10001ae0     Pclass.obj
 0001:00000b00       ??_C@_1BI@OLBAGOJG@?$AAW?$AAS?$AA_?$AAM?$AAA?$AAX?$AAI?$AAM?$AAI?$AAZ?$AAE@ 10001b00     Pclass.obj
 0001:00000b18       ??_C@_1BE@DAMMEKNP@?$AAW?$AAS?$AA_?$AAB?$AAO?$AAR?$AAD?$AAE?$AAR@ 10001b18     Pclass.obj
 0001:00000b2c       ??_C@_1BI@EDHINADK@?$AAW?$AAS?$AA_?$AAD?$AAL?$AAG?$AAF?$AAR?$AAA?$AAM?$AAE@ 10001b2c     Pclass.obj
 0001:00000b44       ??_C@_1BG@CKCLFGFA@?$AAW?$AAS?$AA_?$AAV?$AAS?$AAC?$AAR?$AAO?$AAL?$AAL@ 10001b44     Pclass.obj
 0001:00000b5c       ??_C@_1BG@OMIOJOGF@?$AAW?$AAS?$AA_?$AAH?$AAS?$AAC?$AAR?$AAO?$AAL?$AAL@ 10001b5c     Pclass.obj
 0001:00000b74       ??_C@_1BG@KJOBMDJC@?$AAW?$AAS?$AA_?$AAS?$AAY?$AAS?$AAM?$AAE?$AAN?$AAU@ 10001b74     Pclass.obj
 0001:00000b8c       ??_C@_1BM@GPNNOPCH@?$AAW?$AAS?$AA_?$AAT?$AAH?$AAI?$AAC?$AAK?$AAF?$AAR?$AAA?$AAM?$AAE@ 10001b8c     Pclass.obj
 0001:00000ba8       ??_C@_1BO@FODKBODI@?$AAW?$AAS?$AA_?$AAM?$AAI?$AAN?$AAI?$AAM?$AAI?$AAZ?$AAE?$AAB?$AAO?$AAX@ 10001ba8     Pclass.obj
 0001:00000bc8       ??_C@_1BO@IDJMAOMI@?$AAW?$AAS?$AA_?$AAM?$AAA?$AAX?$AAI?$AAM?$AAI?$AAZ?$AAE?$AAB?$AAO?$AAX@ 10001bc8     Pclass.obj
 0001:00000c88       ??_C@_1CI@PKBCIOPN@?$AAW?$AAS?$AA_?$AAE?$AAX?$AA_?$AAD?$AAL?$AAG?$AAM?$AAO?$AAD?$AAA?$AAL?$AAF@ 10001c88     Pclass.obj
 0001:00000cb0       ??_C@_1CK@KJECLHMG@?$AAW?$AAS?$AA_?$AAE?$AAX?$AA_?$AAN?$AAO?$AAP?$AAA?$AAR?$AAE?$AAN?$AAT?$AAN@ 10001cb0     Pclass.obj
 0001:00000cdc       ??_C@_1BM@OCBKBALE@?$AAW?$AAS?$AA_?$AAE?$AAX?$AA_?$AAT?$AAO?$AAP?$AAM?$AAO?$AAS?$AAT@ 10001cdc     Pclass.obj
 0001:00000cf8       ??_C@_1CE@JIDMMICL@?$AAW?$AAS?$AA_?$AAE?$AAX?$AA_?$AAA?$AAC?$AAC?$AAE?$AAP?$AAT?$AAF?$AAI?$AAL@ 10001cf8     Pclass.obj
 0001:00000d1c       ??_C@_1CE@PFFPBMCF@?$AAW?$AAS?$AA_?$AAE?$AAX?$AA_?$AAT?$AAR?$AAA?$AAN?$AAS?$AAP?$AAA?$AAR?$AAE@ 10001d1c     Pclass.obj
 0001:00000d40       ??_C@_1BO@MEOEJPLO@?$AAW?$AAS?$AA_?$AAE?$AAX?$AA_?$AAM?$AAD?$AAI?$AAC?$AAH?$AAI?$AAL?$AAD@ 10001d40     Pclass.obj
 0001:00000d60       ??_C@_1CC@IEIGGJGG@?$AAW?$AAS?$AA_?$AAE?$AAX?$AA_?$AAT?$AAO?$AAO?$AAL?$AAW?$AAI?$AAN?$AAD?$AAO@ 10001d60     Pclass.obj
 0001:00000d84       ??_C@_1CC@PLPNIKGL@?$AAW?$AAS?$AA_?$AAE?$AAX?$AA_?$AAW?$AAI?$AAN?$AAD?$AAO?$AAW?$AAE?$AAD?$AAG@ 10001d84     Pclass.obj
 0001:00000da8       ??_C@_1CC@IAPGCLEG@?$AAW?$AAS?$AA_?$AAE?$AAX?$AA_?$AAC?$AAL?$AAI?$AAE?$AAN?$AAT?$AAE?$AAD?$AAG@ 10001da8     Pclass.obj
 0001:00000dcc       ??_C@_1CE@EANKNCIF@?$AAW?$AAS?$AA_?$AAE?$AAX?$AA_?$AAC?$AAO?$AAN?$AAT?$AAE?$AAX?$AAT?$AAH?$AAE@ 10001dcc     Pclass.obj
 0001:00000df0       ??_C@_1BI@GFIADCMK@?$AAW?$AAS?$AA_?$AAE?$AAX?$AA_?$AAR?$AAI?$AAG?$AAH?$AAT@ 10001df0     Pclass.obj
 0001:00000e08       ??_C@_1CC@JOFCJJPB@?$AAW?$AAS?$AA_?$AAE?$AAX?$AA_?$AAR?$AAT?$AAL?$AAR?$AAE?$AAA?$AAD?$AAI?$AAN@ 10001e08     Pclass.obj
 0001:00000e2c       ??_C@_1CI@EFLDECAB@?$AAW?$AAS?$AA_?$AAE?$AAX?$AA_?$AAL?$AAE?$AAF?$AAT?$AAS?$AAC?$AAR?$AAO?$AAL@ 10001e2c     Pclass.obj
 0001:00000e54       ??_C@_1CI@CIFGFFJB@?$AAW?$AAS?$AA_?$AAE?$AAX?$AA_?$AAC?$AAO?$AAN?$AAT?$AAR?$AAO?$AAL?$AAP?$AAA@ 10001e54     Pclass.obj
 0001:00000e7c       ??_C@_1CC@BGEPLDCA@?$AAW?$AAS?$AA_?$AAE?$AAX?$AA_?$AAS?$AAT?$AAA?$AAT?$AAI?$AAC?$AAE?$AAD?$AAG@ 10001e7c     Pclass.obj
 0001:00000ea0       ??_C@_1CA@DOAIHHLO@?$AAW?$AAS?$AA_?$AAE?$AAX?$AA_?$AAA?$AAP?$AAP?$AAW?$AAI?$AAN?$AAD?$AAO?$AAW@ 10001ea0     Pclass.obj
 0001:00000ec0       ??_C@_1BM@FAODAMGD@?$AAW?$AAS?$AA_?$AAE?$AAX?$AA_?$AAL?$AAA?$AAY?$AAE?$AAR?$AAE?$AAD@ 10001ec0     Pclass.obj
 0001:00000edc       ??_C@_1CM@DJKNBOGD@?$AAW?$AAS?$AA_?$AAE?$AAX?$AA_?$AAN?$AAO?$AAI?$AAN?$AAH?$AAE?$AAR?$AAI?$AAT@ 10001edc     Pclass.obj
 0001:00000f08       ??_C@_1CA@KMHLBMFI@?$AAW?$AAS?$AA_?$AAE?$AAX?$AA_?$AAL?$AAA?$AAY?$AAO?$AAU?$AAT?$AAR?$AAT?$AAL@ 10001f08     Pclass.obj
 0001:00000f28       ??_C@_1CC@LOFMDOPL@?$AAW?$AAS?$AA_?$AAE?$AAX?$AA_?$AAN?$AAO?$AAA?$AAC?$AAT?$AAI?$AAV?$AAA?$AAT@ 10001f28     Pclass.obj
 0001:00000f4c       ??_C@_19GGNHIDOH@?$AA?4?$AAt?$AAx?$AAt@ 10001f4c     Pclass.obj
 0001:00000f58       ??_C@_1O@CNKEJBH@?$AA?0?$AA?5?$AA?$CF?$AAd?$AA?$CF?$AAs@ 10001f58     Pclass.obj
 0001:00000f68       ??_C@_1BC@NEODPHBM@?$AA?$CF?$AAs?$AA?5?$AA?$CF?$AAs?$AA?$CF?$AAs?$AA?6@ 10001f68     Pclass.obj
 0001:00000f7c       ??_C@_1O@CIJHDDGA@?$AA?$CF?$AAs?$AA?5?$AA?$CF?$AAs?$AA?6@ 10001f7c     Pclass.obj
 0001:00000f8c       ??_C@_1O@DGEEABED@?$AA?$CF?$AAs?$AA?5?$AA?$CF?$AAd?$AA?6@ 10001f8c     Pclass.obj
 0001:00000f9c       ??_C@_17GMPJMPF@?$AA?$CF?$AAs?$AA?5@ 10001f9c     Pclass.obj
 0001:00000fa4       ??_C@_1BE@OMBNFFBH@?$AA?$CF?$AAu?$AA?5?$AA?5?$AA?$CI?$AA?$CF?$AAs?$AA?$CJ?$AA?6@ 10001fa4     Pclass.obj
 0001:00000fb8       ??_C@_17BPBJDALC@?$AA?$CF?$AAu?$AA?6@ 10001fb8     Pclass.obj
 0001:00000fc0       ??_C@_1O@POMONAHN@?$AA?$CF?$AAs?$AA?5?$AA?$CF?$AAu?$AA?6@ 10001fc0     Pclass.obj
 0001:00000fd0       ??_C@_1BG@MDLBKGIE@?$AA?6?$AA?$CF?$AAs?$AA?5?$AA?$CF?$AAs?$AA?5?$AA?$CF?$AAs?$AA?6@ 10001fd0     Pclass.obj
 0001:00000fe8       ??_C@_1BA@OBCELLNO@?$AA?6?$AA?$CF?$AAs?$AA?5?$AA?$CF?$AAs?$AA?6@ 10001fe8     Pclass.obj
 0001:00000ff8       ??_C@_1BC@MLKIHIFN@?$AA?6?$AA?$CF?$AAs?$AA?3?$AA?6?$AA?$CF?$AAs?$AA?6@ 10001ff8     Pclass.obj
 0001:0000100c       ??_C@_1BA@DHHNFIMD@?$AA?6?$AA?$CF?$AAs?$AA?5?$AA?$CF?$AAu?$AA?6@ 1000200c     Pclass.obj
 0001:0000101c       ??_C@_1BE@JKDBKCGH@?$AA?$CF?$AA?9?$AA2?$AA2?$AAs?$AA?5?$AA?$CF?$AAp?$AA?6@ 1000201c     Pclass.obj
 0001:00001030       ??_C@_1M@NOMFOFMP@?$AAH?$AAW?$AAN?$AAD?$AA?3@ 10002030     Pclass.obj
 0001:0000103c       ??_C@_13HOIJIPNN@?$AA?5@   1000203c     Pclass.obj
 0001:00001040       ??_C@_1BO@LJMHGFAK@?$AA?$CF?$AA?9?$AA2?$AA2?$AAs?$AA?5?$AA?$CF?$AA0?$AA8?$AAX?$AA?5?$AA?$CF?$AAs?$AA?6@ 10002040     Pclass.obj
 0001:00001060       ??_C@_1BE@PEGLKBKB@?$AA?6?$AA?$CF?$AAs?$AA?6?$AA?$CF?$AAs?$AA?$CF?$AAs?$AA?6@ 10002060     Pclass.obj
 0001:00001074       ??_C@_17JJIMNMHK@?$AA?5?$AA?$CG?$AA?$FO@ 10002074     Pclass.obj
 0001:00001090       ??_C@_15DDHGOCBH@?$AA?4?$AA?4@ 10002090     Pclass.obj
 0001:00001098       ??_C@_17FJPEEFCB@?$AAp?$AAr?$AAc@ 10002098     Pclass.obj
 0001:000010a0       ??_C@_1BC@ENICKDH@?$AAC?$AAo?$AAn?$AAt?$AAe?$AAn?$AAt?$AAs@ 100020a0     Pclass.obj
 0001:000010b4       ??_C@_1CK@DGKCELDD@?$AAP?$AAr?$AAo?$AAc?$AAe?$AAs?$AAs?$AAL?$AAi?$AAs?$AAt?$AA?4?$AAC?$AAo?$AAm@ 100020b4     Pclass.obj
 0001:000010e0       ??_C@_1CK@ECJCGOEK@?$AAP?$AAr?$AAo?$AAc?$AAe?$AAs?$AAs?$AAL?$AAi?$AAs?$AAt?$AA?4?$AAU?$AAs?$AAe@ 100020e0     Pclass.obj
 0001:0000110c       ??_C@_15LEKKCGMK@?$AA?2?$AA?2@ 1000210c     Pclass.obj
 0001:00001114       ??_C@_1M@HKFBKEEN@?$AA?$CF?$AA?$CF?$AA?5?$AA?$CF?$AAs@ 10002114     Pclass.obj
 0001:00001120       ??_C@_1M@MOFLFCEC@?$AA?$CF?$AAs?$AA?5?$AA?$CF?$AAs@ 10002120     Pclass.obj
 0001:0000112c       ??_C@_17DJGLCLAO@?$AA?$CF?$AAs?$AA?3@ 1000212c     Pclass.obj
 0001:00001134       ??_C@_1M@EJMLOAMM@?$AA?$CF?$AA?9?$AA2?$AA2?$AAs@ 10002134     Pclass.obj
 0001:00001170       ??_C@_1CE@OMPPCAIJ@?$AA?$CF?$AAd?$AA?5?$AA?$CF?$AA0?$AA2?$AAd?$AA?3?$AA?$CF?$AA0?$AA2?$AAd?$AA?3?$AA?$CF?$AA0@ 10002170     Pclass.obj
 0001:00001194       ??_C@_1BO@EHJBCONC@?$AA?$CF?$AA0?$AA2?$AAd?$AA?3?$AA?$CF?$AA0?$AA2?$AAd?$AA?3?$AA?$CF?$AA0?$AA2?$AAd@ 10002194     Pclass.obj
 0001:000011b4       ??_C@_17JLFEDMMI@?$AA?$DP?$AA?$DP?$AA?$DP@ 100021b4     Pclass.obj
 0001:000011dc       ??_C@_1CG@PJJCHAJ@?$AA?2?$AA?$CF?$AAs?$AA?2?$AA?$CF?$AAs?$AA?2?$AAF?$AAi?$AAl?$AAe?$AAV?$AAe?$AAr?$AAs@ 100021dc     Pclass.obj
 0001:00001204       ??_C@_1CO@PDLCNLLF@?$AA?2?$AA?$CF?$AAs?$AA?2?$AA?$CF?$AAs?$AA?2?$AAF?$AAi?$AAl?$AAe?$AAD?$AAe?$AAs?$AAc@ 10002204     Pclass.obj
 0001:00001234       ??_C@_17CHCGIDNB@?$AA?$CF?$AAs?$AA?2@ 10002234     Pclass.obj
 0001:0000123c       ??_C@_1M@CBILFCKF@?$AA?5?$AA?$CI?$AA?$CF?$AAs?$AA?$CJ@ 1000223c     Pclass.obj
 0001:00001248       ??_C@_1BC@OMEIBLAI@?$AAw?$AAb?$AAe?$AAm?$AAc?$AAo?$AAm?$AAn@ 10002248     Pclass.obj
 0001:0000125c       ??_C@_1CC@DNHMJIKH@?$AA?$CF?$AA?5?$AAP?$AAr?$AAo?$AAc?$AAe?$AAs?$AAs?$AAo?$AAr?$AA?5?$AAT?$AAi?$AAm@ 1000225c     perfthread.obj
 0001:00001280       ??_C@_1CE@FNEMIHOD@?$AA?$CF?$AA?5?$AAP?$AAr?$AAi?$AAv?$AAi?$AAl?$AAe?$AAg?$AAe?$AAd?$AA?5?$AAT?$AAi@ 10002280     perfthread.obj
 0001:000012a4       ??_C@_1BI@IIOPEKIO@?$AA?$CF?$AA?5?$AAU?$AAs?$AAe?$AAr?$AA?5?$AAT?$AAi?$AAm?$AAe@ 100022a4     perfthread.obj
 0001:000012bc       ??_C@_1BK@FAAJNJIB@?$AAH?$AAa?$AAn?$AAd?$AAl?$AAe?$AA?5?$AAC?$AAo?$AAu?$AAn?$AAt@ 100022bc     perfthread.obj
 0001:000012d8       ??_C@_1CA@KJMNGIDJ@?$AAP?$AAa?$AAg?$AAe?$AA?5?$AAF?$AAi?$AAl?$AAe?$AA?5?$AAB?$AAy?$AAt?$AAe?$AAs@ 100022d8     perfthread.obj
 0001:000012f8       ??_C@_1CK@FGGMBBIH@?$AAP?$AAa?$AAg?$AAe?$AA?5?$AAF?$AAi?$AAl?$AAe?$AA?5?$AAB?$AAy?$AAt?$AAe?$AAs@ 100022f8     perfthread.obj
 0001:00001324       ??_C@_1BI@GCOMDKEO@?$AAW?$AAo?$AAr?$AAk?$AAi?$AAn?$AAg?$AA?5?$AAS?$AAe?$AAt@ 10002324     perfthread.obj
 0001:0000133c       ??_C@_1CC@OFJLEPCP@?$AAW?$AAo?$AAr?$AAk?$AAi?$AAn?$AAg?$AA?5?$AAS?$AAe?$AAt?$AA?5?$AAP?$AAe?$AAa@ 1000233c     perfthread.obj
 0001:00001360       ??_C@_1CI@LLKMGPEG@?$AAP?$AAo?$AAo?$AAl?$AA?5?$AAN?$AAo?$AAn?$AAp?$AAa?$AAg?$AAe?$AAd?$AA?5?$AAB@ 10002360     perfthread.obj
 0001:00001388       ??_C@_1CC@IMBAECJF@?$AAP?$AAo?$AAo?$AAl?$AA?5?$AAP?$AAa?$AAg?$AAe?$AAd?$AA?5?$AAB?$AAy?$AAt?$AAe@ 10002388     perfthread.obj
 0001:000013ac       ??_C@_1BM@DGDPAMAA@?$AAP?$AAr?$AAi?$AAv?$AAa?$AAt?$AAe?$AA?5?$AAB?$AAy?$AAt?$AAe?$AAs@ 100023ac     perfthread.obj
 0001:000013c8       ??_C@_1CA@GADAGCME@?$AAP?$AAa?$AAg?$AAe?$AA?5?$AAF?$AAa?$AAu?$AAl?$AAt?$AAs?$AA?1?$AAs?$AAe?$AAc@ 100023c8     perfthread.obj
 0001:000013e8       ??_C@_1BM@FMIOMJAE@?$AAV?$AAi?$AAr?$AAt?$AAu?$AAa?$AAl?$AA?5?$AAB?$AAy?$AAt?$AAe?$AAs@ 100023e8     perfthread.obj
 0001:00001404       ??_C@_1CG@KJOKFONA@?$AAV?$AAi?$AAr?$AAt?$AAu?$AAa?$AAl?$AA?5?$AAB?$AAy?$AAt?$AAe?$AAs?$AA?5?$AAP@ 10002404     perfthread.obj
 0001:0000142c       ??_C@_1CE@DFDFLLAO@?$AAI?$AAO?$AA?5?$AAD?$AAa?$AAt?$AAa?$AA?5?$AAB?$AAy?$AAt?$AAe?$AAs?$AA?1?$AAs@ 1000242c     perfthread.obj
 0001:00001450       ??_C@_1CE@EFLEKJAB@?$AAI?$AAO?$AA?5?$AAR?$AAe?$AAa?$AAd?$AA?5?$AAB?$AAy?$AAt?$AAe?$AAs?$AA?1?$AAs@ 10002450     perfthread.obj
 0001:00001474       ??_C@_1CG@MEJHKKKF@?$AAI?$AAO?$AA?5?$AAW?$AAr?$AAi?$AAt?$AAe?$AA?5?$AAB?$AAy?$AAt?$AAe?$AAs?$AA?1@ 10002474     perfthread.obj
 0001:0000149c       ??_C@_1CG@LBBBPCJA@?$AAI?$AAO?$AA?5?$AAO?$AAt?$AAh?$AAe?$AAr?$AA?5?$AAB?$AAy?$AAt?$AAe?$AAs?$AA?1@ 1000249c     perfthread.obj
 0001:000014c4       ??_C@_1CO@LIEOHDCC@?$AAI?$AAO?$AA?5?$AAD?$AAa?$AAt?$AAa?$AA?5?$AAO?$AAp?$AAe?$AAr?$AAa?$AAt?$AAi@ 100024c4     perfthread.obj
 0001:000014f4       ??_C@_1CO@LIIKBHDH@?$AAI?$AAO?$AA?5?$AAR?$AAe?$AAa?$AAd?$AA?5?$AAO?$AAp?$AAe?$AAr?$AAa?$AAt?$AAi@ 100024f4     perfthread.obj
 0001:00001524       ??_C@_1DA@HICMAFKK@?$AAI?$AAO?$AA?5?$AAW?$AAr?$AAi?$AAt?$AAe?$AA?5?$AAO?$AAp?$AAe?$AAr?$AAa?$AAt@ 10002524     perfthread.obj
 0001:00001554       ??_C@_1DA@BEHINMGJ@?$AAI?$AAO?$AA?5?$AAO?$AAt?$AAh?$AAe?$AAr?$AA?5?$AAO?$AAp?$AAe?$AAr?$AAa?$AAt@ 10002554     perfthread.obj
 0001:00001588       ??_C@_1HE@NBDABLAL@?$AAS?$AAo?$AAf?$AAt?$AAw?$AAa?$AAr?$AAe?$AA?2?$AAM?$AAi?$AAc?$AAr?$AAo?$AAs@ 10002588     perfthread.obj
 0001:000015fc       ??_C@_1BC@IICCDNLG@?$AAC?$AAo?$AAu?$AAn?$AAt?$AAe?$AAr?$AAs@ 100025fc     perfthread.obj
 0001:00001610       ??_C@_1BG@NKNJPBCD@?$AAI?$AAD?$AA?5?$AAP?$AAr?$AAo?$AAc?$AAe?$AAs?$AAs@ 10002610     perfthread.obj
 0001:00001628       ??_C@_1BM@KCAKLHJN@?$AAP?$AAr?$AAi?$AAo?$AAr?$AAi?$AAt?$AAy?$AA?5?$AAB?$AAa?$AAs?$AAe@ 10002628     perfthread.obj
 0001:00001644       ??_C@_1BK@KCHPPKHP@?$AAT?$AAh?$AAr?$AAe?$AAa?$AAd?$AA?5?$AAC?$AAo?$AAu?$AAn?$AAt@ 10002644     perfthread.obj
 0001:00001660       ??_C@_1CI@FNIEMNAI@?$AAC?$AAr?$AAe?$AAa?$AAt?$AAi?$AAn?$AAg?$AA?5?$AAP?$AAr?$AAo?$AAc?$AAe?$AAs@ 10002660     perfthread.obj
 0001:00001688       ??_C@_1BK@IKAFHKBD@?$AAE?$AAl?$AAa?$AAp?$AAs?$AAe?$AAd?$AA?5?$AAT?$AAi?$AAm?$AAe@ 10002688     perfthread.obj
 0001:000016a4       ??_C@_19DOGDICKI@?$AA?4?$AAe?$AAx?$AAe@ 100026a4     perfthread.obj
 0001:000016b0       ??_C@_1CC@DMDJMJLM@?$AAS?$AAe?$AAD?$AAe?$AAb?$AAu?$AAg?$AAP?$AAr?$AAi?$AAv?$AAi?$AAl?$AAe?$AAg@ 100026b0     Plist.obj
 0001:000016d4       ??_C@_1M@GPDJLPMI@?$AA?4?$AA?$CF?$AA0?$AA3?$AAd@ 100026d4     Plist.obj
 0001:000016e0       ??_C@_13EBCNDICG@?$AA?3@   100026e0     Plist.obj
 0001:000016e4       ??_C@_1O@KBBIJFEI@?$AA?$CF?$AA?9?$AA2?$AA4?$AAs?$AA?5@ 100026e4     Plist.obj
 0001:000016f4       ??_C@_1BC@CIAMCHCM@?$AA?$CF?$AA1?$AA0?$AAI?$AA6?$AA4?$AAu?$AA?6@ 100026f4     Plist.obj
 0001:00001708       ??_C@_1BK@OIAGEDCG@?$AA?$CF?$AAs?$AA?5?$AA?$CF?$AA7?$AAI?$AA6?$AA4?$AAu?$AA?$CF?$AA?$CF?$AA?6@ 10002708     Plist.obj
 0001:00001724       ??_C@_1CG@FOOPEKLK@?$AA?$CF?$AA1?$AA0?$AAI?$AA6?$AA4?$AAu?$AA?5?$AA?5?$AA?$CF?$AA5?$AAI?$AA6?$AA4?$AAu@ 10002724     Plist.obj
 0001:0000174c       ??_C@_1BA@LFJAMCEC@?$AA?$CF?$AAs?$AA?5?$AA?$CF?$AAs?$AA?6?$AA?6@ 1000274c     Plist.obj
 0001:0000175c       ??_C@_19FJPIAKGM@?$AA?$CF?$AAs?$AA?6?$AA?6@ 1000275c     Plist.obj
 0001:00001768       ??_C@_17MJEANDKP@?$AA?$CF?$AAs?$AA?6@ 10002768     Plist.obj
 0001:00001770       ??_C@_1BE@KPJOOIA@?$AA?5?$AA?5?$AA?$CF?$AAp?$AA?5?$AA?5?$AA?$CF?$AA6?$AAX@ 10002770     Plist.obj
 0001:00001784       ??_C@_17ENEANJDH@?$AA?5?$AA?$CF?$AAs@ 10002784     Plist.obj
 0001:0000178c       ??_C@_1BG@FFJGBKCB@?$AAE?$AAr?$AAr?$AAo?$AAr?$AA?5?$AA0?$AAx?$AA?$CF?$AAx@ 1000278c     Pmix.obj
 0001:000017a4       ??_C@_15JNBOKNOG@?$AA?$AN?$AA?6@ 100027a4     Pmix.obj
 0001:000017ac       _IID_IWbemLocator          100027ac     WMI.obj
 0001:000017bc       _CLSID_WbemLocator         100027bc     WMI.obj
 0001:000017cc       ??_C@_1DA@BIBEJFMF@?$AAW?$AAi?$AAn?$AA3?$AA2?$AA_?$AAP?$AAr?$AAo?$AAc?$AAe?$AAs?$AAs?$AA?4?$AAH@ 100027cc     WMI.obj
 0001:000017fc       ??_C@_1BO@CLCOBGDE@?$AAE?$AAx?$AAe?$AAc?$AAu?$AAt?$AAa?$AAb?$AAl?$AAe?$AAP?$AAa?$AAt?$AAh@ 100027fc     WMI.obj
 0001:0000181c       ??_C@_1BC@JHNNEHFE@?$AAP?$AAr?$AAi?$AAo?$AAr?$AAi?$AAt?$AAy@ 1000281c     WMI.obj
 0001:00001830       ??_C@_1BC@HJJANEGO@?$AAG?$AAe?$AAt?$AAO?$AAw?$AAn?$AAe?$AAr@ 10002830     WMI.obj
 0001:00001844       ??_C@_19PIJILKAI@?$AAU?$AAs?$AAe?$AAr@ 10002844     WMI.obj
 0001:00001850       ??_C@_1O@OAMNPMOM@?$AAD?$AAo?$AAm?$AAa?$AAi?$AAn@ 10002850     WMI.obj
 0001:00001860       ??_C@_1BI@OIPNMPCL@?$AAG?$AAe?$AAt?$AAO?$AAw?$AAn?$AAe?$AAr?$AAS?$AAi?$AAd@ 10002860     WMI.obj
 0001:00001878       ??_C@_17NKMLOKHF@?$AAS?$AAi?$AAd@ 10002878     WMI.obj
 0001:00001880       ??_C@_1BE@CFEJJKFE@?$AAS?$AAe?$AAs?$AAs?$AAi?$AAo?$AAn?$AAI?$AAd@ 10002880     WMI.obj
 0001:00001894       ??_C@_1BM@MLGLIGHJ@?$AAW?$AAi?$AAn?$AA3?$AA2?$AA_?$AAP?$AAr?$AAo?$AAc?$AAe?$AAs?$AAs@ 10002894     WMI.obj
 0001:000018b0       ??_C@_1BI@FLOHINJE@?$AAR?$AAe?$AAt?$AAu?$AAr?$AAn?$AAV?$AAa?$AAl?$AAu?$AAe@ 100028b0     WMI.obj
 0001:000018c8       ??_C@_1BI@NKNJJIDM@?$AAS?$AAe?$AAt?$AAP?$AAr?$AAi?$AAo?$AAr?$AAi?$AAt?$AAy@ 100028c8     WMI.obj
 0001:000018e0       ??_C@_1O@GGHBFGJC@?$AAR?$AAe?$AAa?$AAs?$AAo?$AAn@ 100028e0     WMI.obj
 0001:000018f0       ??_C@_1BE@PBPGMODO@?$AAT?$AAe?$AAr?$AAm?$AAi?$AAn?$AAa?$AAt?$AAe@ 100028f0     WMI.obj
 0001:00001904       ??_C@_13JOFGPIOO@?$AA?4@   10002904     WMI.obj
 0001:00001908       ??_C@_1CA@ECJNGEII@?$AA?2?$AA?2?$AA?$CF?$AAs?$AA?2?$AAr?$AAo?$AAo?$AAt?$AA?2?$AAc?$AAi?$AAm?$AAv?$AA2@ 10002908     WMI.obj
 0001:00001928       _MainGuid                  10002928     Proclist.obj
 0001:00001938       _MenuGuid                  10002938     Proclist.obj
 0001:00001948       _ConfigDialogGuid          10002948     Proclist.obj
 0001:00001958       ??_C@_1M@OAIMIKLP@?$AAn?$AAt?$AAd?$AAl?$AAl@ 10002958     Proclist.obj
 0001:00001964       ??_C@_0BK@EGDDIFMK@NtQueryInformationProcess@ 10002964     Proclist.obj
 0001:00001980       ??_C@_0BJ@HKKELGGC@NtQueryInformationThread@ 10002980     Proclist.obj
 0001:0000199c       ??_C@_0O@IFMDHOMC@NtQueryObject@ 1000299c     Proclist.obj
 0001:000019ac       ??_C@_0BJ@NDLOPGCH@NtQuerySystemInformation@ 100029ac     Proclist.obj
 0001:000019c8       ??_C@_0BH@DLPGICA@NtQueryInformationFile@ 100029c8     Proclist.obj
 0001:000019e0       ??_C@_1BC@GDMECMAK@?$AAk?$AAe?$AAr?$AAn?$AAe?$AAl?$AA3?$AA2@ 100029e0     Proclist.obj
 0001:000019f4       ??_C@_0P@LKABJJMO@IsWow64Process@ 100029f4     Proclist.obj
 0001:00001a04       ??_C@_1BC@DNHGCMLG@?$AAa?$AAd?$AAv?$AAa?$AAp?$AAi?$AA3?$AA2@ 10002a04     Proclist.obj
 0001:00001a18       ??_C@_0L@KJHKJIPF@IsValidSid@ 10002a18     Proclist.obj
 0001:00001a24       ??_C@_0BK@FIHGNING@GetSidIdentifierAuthority@ 10002a24     Proclist.obj
 0001:00001a40       ??_C@_0BI@LPFJALDI@GetSidSubAuthorityCount@ 10002a40     Proclist.obj
 0001:00001a58       ??_C@_0BD@LMGFHOAE@GetSidSubAuthority@ 10002a58     Proclist.obj
 0001:00001a6c       ??_C@_0BD@MCBOPCDK@LookupAccountNameW@ 10002a6c     Proclist.obj
 0001:00001a80       ??_C@_1O@BCCLBEOE@?$AAu?$AAs?$AAe?$AAr?$AA3?$AA2@ 10002a80     Proclist.obj
 0001:00001a90       ??_C@_0BA@FKGDNIJG@GetGuiResources@ 10002a90     Proclist.obj
 0001:00001aa0       ??_C@_1M@FFPAMFOB@?$AAo?$AAl?$AAe?$AA3?$AA2@ 10002aa0     Proclist.obj
 0001:00001aac       ??_C@_0BC@IOEGILCE@CoSetProxyBlanket@ 10002aac     Proclist.obj
 0001:00001ac0       ??_C@_1BC@PDEABLIN@?$AAP?$AAr?$AAo?$AAc?$AAL?$AAi?$AAs?$AAt@ 10002ac0     Proclist.obj
 0001:00001ad4       ??_C@_1DK@DCAMPEPJ@?$AAP?$AAr?$AAo?$AAc?$AAe?$AAs?$AAs?$AA?5?$AAL?$AAi?$AAs?$AAt?$AA?5?$AAf?$AAo@ 10002ad4     Proclist.obj
 0001:00001b10       ??_C@_1DE@BGKMIKPD@?$AAE?$AAu?$AAg?$AAe?$AAn?$AAe?$AA?5?$AAR?$AAo?$AAs?$AAh?$AAa?$AAl?$AA?5?$AA?$CG@ 10002b10     Proclist.obj
 0001:00001b44       ??_C@_1M@MNPEKPKO@?$AAp?$AAl?$AAi?$AAs?$AAt@ 10002b44     Proclist.obj
 0001:00001b50       __imp__EncodePointer@4     10002b50     vc_crt_fix.obj
 0001:00001b54       __imp__DecodePointer@4     10002b54     vc_crt_fix.obj
 0001:00001b58       __imp__GetModuleHandleExW@12 10002b58     vc_crt_fix.obj
 0001:00001b5c       __imp__InitializeSListHead@4 10002b5c     vc_crt_fix.obj
 0001:00001b60       __imp__InterlockedFlushSList@4 10002b60     vc_crt_fix.obj
 0001:00001b64       __imp__InterlockedPopEntrySList@4 10002b64     vc_crt_fix.obj
 0001:00001b68       __imp__InterlockedPushEntrySList@8 10002b68     vc_crt_fix.obj
 0001:00001b6c       __imp__InterlockedPushListSListEx@16 10002b6c     vc_crt_fix.obj
 0001:00001b70       __imp__RtlFirstEntrySList@4 10002b70     vc_crt_fix.obj
 0001:00001b74       __imp__QueryDepthSList@4   10002b74     vc_crt_fix.obj
 0001:00001b78       __imp__GetNumaHighestNodeNumber@4 10002b78     vc_crt_fix.obj
 0001:00001b7c       __imp__GetLogicalProcessorInformation@8 10002b7c     vc_crt_fix.obj
 0001:00001b80       __imp__SetThreadStackGuarantee@4 10002b80     vc_crt_fix.obj
 0001:00001ba4       ??_C@_0O@NLDKAIKN@EncodePointer@ 10002ba4     vc_crt_fix_impl.obj
 0001:00001bb4       ??_C@_0O@KBPMFGHI@DecodePointer@ 10002bb4     vc_crt_fix_impl.obj
 0001:00001bc4       ??_C@_0BD@GIGEJCNH@GetModuleHandleExW@ 10002bc4     vc_crt_fix_impl.obj
 0001:00001bd8       ??_C@_0BE@NBEJPEJA@InitializeSListHead@ 10002bd8     vc_crt_fix_impl.obj
 0001:00001bec       ??_C@_0BG@PLLPFLHB@InterlockedFlushSList@ 10002bec     vc_crt_fix_impl.obj
 0001:00001c04       ??_C@_0BJ@PNEEKDOK@InterlockedPopEntrySList@ 10002c04     vc_crt_fix_impl.obj
 0001:00001c20       ??_C@_0BK@JFGGAIOA@InterlockedPushEntrySList@ 10002c20     vc_crt_fix_impl.obj
 0001:00001c3c       ??_C@_0BL@FOECAEGO@InterlockedPushListSListEx@ 10002c3c     vc_crt_fix_impl.obj
 0001:00001c58       ??_C@_0BD@FHMMIGCI@RtlFirstEntrySList@ 10002c58     vc_crt_fix_impl.obj
 0001:00001c6c       ??_C@_0BA@FGPHPMJB@QueryDepthSList@ 10002c6c     vc_crt_fix_impl.obj
 0001:00001c7c       ??_C@_0BJ@NLNFLAMA@GetNumaHighestNodeNumber@ 10002c7c     vc_crt_fix_impl.obj
 0001:00001c98       ??_C@_0BP@KHGALBC@GetLogicalProcessorInformation@ 10002c98     vc_crt_fix_impl.obj
 0001:00001cb8       ??_C@_0BI@BKLFFAPO@SetThreadStackGuarantee@ 10002cb8     vc_crt_fix_impl.obj
 0001:00001cd0       __pRawDllMain              10002cd0     LIBCMT:dll_dllmain.obj
 0001:00001cd0       __pDefaultRawDllMain       10002cd0     LIBCMT:dll_dllmain.obj
 0001:00001cd8       ??_7exception@std@@6B@     10002cd8     LIBCMT:throw_bad_alloc.obj
 0001:00001ce0       ??_C@_0BC@EOODALEL@Unknown?5exception@ 10002ce0     LIBCMT:throw_bad_alloc.obj
 0001:00001cf8       ??_7bad_alloc@std@@6B@     10002cf8     LIBCMT:throw_bad_alloc.obj
 0001:00001d00       ??_C@_0P@GHFPNOJB@bad?5allocation@ 10002d00     LIBCMT:throw_bad_alloc.obj
 0001:00001d14       ??_7bad_array_new_length@std@@6B@ 10002d14     LIBCMT:throw_bad_alloc.obj
 0001:00001d1c       ??_C@_0BF@KINCDENJ@bad?5array?5new?5length@ 10002d1c     LIBCMT:throw_bad_alloc.obj
 0001:00001d38       ??_7type_info@@6B@         10002d38     LIBCMT:std_type_info_static.obj
 0001:00001d70       ??_C@_1DM@KHCHBNEB@?$AAa?$AAp?$AAi?$AA?9?$AAm?$AAs?$AA?9?$AAw?$AAi?$AAn?$AA?9?$AAc?$AAo?$AAr?$AAe@ 10002d70     libvcruntime:winapi_downlevel.obj
 0001:00001dac       ??_C@_1DK@LPPGFMPP@?$AAa?$AAp?$AAi?$AA?9?$AAm?$AAs?$AA?9?$AAw?$AAi?$AAn?$AA?9?$AAc?$AAo?$AAr?$AAe@ 10002dac     libvcruntime:winapi_downlevel.obj
 0001:00001de8       ??_C@_1BA@PFFKHIOG@?$AAa?$AAp?$AAi?$AA?9?$AAm?$AAs?$AA?9@ 10002de8     libvcruntime:winapi_downlevel.obj
 0001:00001df8       ??_C@_1BA@IAIFMGEF@?$AAe?$AAx?$AAt?$AA?9?$AAm?$AAs?$AA?9@ 10002df8     libvcruntime:winapi_downlevel.obj
 0001:00001e10       ??_C@_08KNHFBNJ@FlsAlloc@  10002e10     libvcruntime:winapi_downlevel.obj
 0001:00001e24       ??_C@_07PEJMOBNF@FlsFree@  10002e24     libvcruntime:winapi_downlevel.obj
 0001:00001e34       ??_C@_0M@GDNOONDI@FlsGetValue@ 10002e34     libvcruntime:winapi_downlevel.obj
 0001:00001e48       ??_C@_0M@JCPCPOEF@FlsSetValue@ 10002e48     libvcruntime:winapi_downlevel.obj
 0001:00001e5c       ??_C@_0BM@HCFOFFN@InitializeCriticalSectionEx@ 10002e5c     libvcruntime:winapi_downlevel.obj
 0001:00002014       ??_C@_08EHJDFFNH@__based?$CI@ 10003014     libvcruntime:undname.obj
 0001:00002020       ??_C@_07KOLFKCDI@__cdecl@  10003020     libvcruntime:undname.obj
 0001:00002028       ??_C@_08GHMPAG@__pascal@   10003028     libvcruntime:undname.obj
 0001:00002034       ??_C@_09IFJBGAPI@__stdcall@ 10003034     libvcruntime:undname.obj
 0001:00002040       ??_C@_0L@NPHFGOKO@__thiscall@ 10003040     libvcruntime:undname.obj
 0001:0000204c       ??_C@_0L@JMKHOMEK@__fastcall@ 1000304c     libvcruntime:undname.obj
 0001:00002058       ??_C@_0N@BCKKPABJ@__vectorcall@ 10003058     libvcruntime:undname.obj
 0001:00002068       ??_C@_09HIJEGCPM@__clrcall@ 10003068     libvcruntime:undname.obj
 0001:00002074       ??_C@_06GHPCKEAG@__eabi@   10003074     libvcruntime:undname.obj
 0001:0000207c       ??_C@_09IOPIDJLG@__swift_1@ 1000307c     libvcruntime:undname.obj
 0001:00002088       ??_C@_09KFNFGKHF@__swift_2@ 10003088     libvcruntime:undname.obj
 0001:00002094       ??_C@_07JOMMBBKO@__ptr64@  10003094     libvcruntime:undname.obj
 0001:0000209c       ??_C@_0L@PILCLIHE@__restrict@ 1000309c     libvcruntime:undname.obj
 0001:000020a8       ??_C@_0M@GFIIJFMG@__unaligned@ 100030a8     libvcruntime:undname.obj
 0001:000020b4       ??_C@_09DHDLOLLB@restrict?$CI@ 100030b4     libvcruntime:undname.obj
 0001:000020be       ??_C@_00CNPNBAHC@@         100030be     libvcruntime:undname.obj
 0001:000020c0       ??_C@_04NIHEBCM@?5new@     100030c0     libvcruntime:undname.obj
 0001:000020c8       ??_C@_07FPCDHGMM@?5delete@ 100030c8     libvcruntime:undname.obj
 0001:000020d0       ??_C@_01NEMOKFLO@?$DN@     100030d0     libvcruntime:undname.obj
 0001:000020d4       ??_C@_02GPIOPFAK@?$DO?$DO@ 100030d4     libvcruntime:undname.obj
 0001:000020d8       ??_C@_02FODMEDOG@?$DM?$DM@ 100030d8     libvcruntime:undname.obj
 0001:000020dc       ??_C@_01DCLJPIOD@?$CB@     100030dc     libvcruntime:undname.obj
 0001:000020e0       ??_C@_02EGOFBIJA@?$DN?$DN@ 100030e0     libvcruntime:undname.obj
 0001:000020e4       ??_C@_02FDNJECIE@?$CB?$DN@ 100030e4     libvcruntime:undname.obj
 0001:000020e8       ??_C@_02GPECMEKF@?$FL?$FN@ 100030e8     libvcruntime:undname.obj
 0001:000020ec       ??_C@_08LHJFAFGD@operator@ 100030ec     libvcruntime:undname.obj
 0001:000020f8       ??_C@_02HBOOOICD@?9?$DO@   100030f8     libvcruntime:undname.obj
 0001:000020fc       ??_C@_01NBENCBCI@?$CK@     100030fc     libvcruntime:undname.obj
 0001:00002100       ??_C@_02ECNGHCIF@?$CL?$CL@ 10003100     libvcruntime:undname.obj
 0001:00002104       ??_C@_02BAABKJLB@?9?9@     10003104     libvcruntime:undname.obj
 0001:00002108       ??_C@_01JOAMLHOP@?9@       10003108     libvcruntime:undname.obj
 0001:0000210c       ??_C@_01MIFGBAGJ@?$CL@     1000310c     libvcruntime:undname.obj
 0001:00002110       ??_C@_01HNPIGOCE@?$CG@     10003110     libvcruntime:undname.obj
 0001:00002114       ??_C@_03MNHNFDLC@?9?$DO?$CK@ 10003114     libvcruntime:undname.obj
 0001:00002118       ??_C@_01KMDKNFGN@?1@       10003118     libvcruntime:undname.obj
 0001:0000211c       ??_C@_01FGNFDNOH@?$CF@     1000311c     libvcruntime:undname.obj
 0001:00002120       ??_C@_01MNNFJEPP@?$DM@     10003120     libvcruntime:undname.obj
 0001:00002124       ??_C@_02EHCHHCKH@?$DM?$DN@ 10003124     libvcruntime:undname.obj
 0001:00002128       ??_C@_01PPODPGHN@?$DO@     10003128     libvcruntime:undname.obj
 0001:0000212c       ??_C@_02EEKDKGMJ@?$DO?$DN@ 1000312c     libvcruntime:undname.obj
 0001:00002130       ??_C@_01IHBHIGKO@?0@       10003130     libvcruntime:undname.obj
 0001:00002134       ??_C@_02HCKGKOFO@?$CI?$CJ@ 10003134     libvcruntime:undname.obj
 0001:00002138       ??_C@_01PJKLJHI@?$HO@      10003138     libvcruntime:undname.obj
 0001:0000213c       ??_C@_01JKBOJNNK@?$FO@     1000313c     libvcruntime:undname.obj
 0001:00002140       ??_C@_01DNKMNLPK@?$HM@     10003140     libvcruntime:undname.obj
 0001:00002144       ??_C@_02PPKAJPJL@?$CG?$CG@ 10003144     libvcruntime:undname.obj
 0001:00002148       ??_C@_02NONPIBCD@?$HM?$HM@ 10003148     libvcruntime:undname.obj
 0001:0000214c       ??_C@_02FPIMKNGF@?$CK?$DN@ 1000314c     libvcruntime:undname.obj
 0001:00002150       ??_C@_02FOEOMHFC@?$CL?$DN@ 10003150     libvcruntime:undname.obj
 0001:00002154       ??_C@_02FKMDLLOA@?9?$DN@   10003154     libvcruntime:undname.obj
 0001:00002158       ??_C@_02FJEHGPIO@?1?$DN@   10003158     libvcruntime:undname.obj
 0001:0000215c       ??_C@_02FENAOKFI@?$CF?$DN@ 1000315c     libvcruntime:undname.obj
 0001:00002160       ??_C@_03IKFCCPFF@?$DO?$DO?$DN@ 10003160     libvcruntime:undname.obj
 0001:00002164       ??_C@_03CDNPDDLA@?$DM?$DM?$DN@ 10003164     libvcruntime:undname.obj
 0001:00002168       ??_C@_02FGJGFEAB@?$CG?$DN@ 10003168     libvcruntime:undname.obj
 0001:0000216c       ??_C@_02DHLNPPGH@?$HM?$DN@ 1000316c     libvcruntime:undname.obj
 0001:00002170       ??_C@_02MHEGNOJ@?$FO?$DN@  10003170     libvcruntime:undname.obj
 0001:00002174       ??_C@_09IFPLHPGF@?$GAvftable?8@ 10003174     libvcruntime:undname.obj
 0001:00002180       ??_C@_09BLBHBJP@?$GAvbtable?8@ 10003180     libvcruntime:undname.obj
 0001:0000218c       ??_C@_07FEEIOKP@?$GAvcall?8@ 1000318c     libvcruntime:undname.obj
 0001:00002194       ??_C@_08LLFFHHDJ@?$GAtypeof?8@ 10003194     libvcruntime:undname.obj
 0001:000021a0       ??_C@_0BF@KDPPACIK@?$GAlocal?5static?5guard?8@ 100031a0     libvcruntime:undname.obj
 0001:000021b8       ??_C@_08OBABFOLI@?$GAstring?8@ 100031b8     libvcruntime:undname.obj
 0001:000021c4       ??_C@_0BD@JDLKDPAB@?$GAvbase?5destructor?8@ 100031c4     libvcruntime:undname.obj
 0001:000021d8       ??_C@_0BN@DEGPLNFK@?$GAvector?5deleting?5destructor?8@ 100031d8     libvcruntime:undname.obj
 0001:000021f8       ??_C@_0BO@OBMKPJIG@?$GAdefault?5constructor?5closure?8@ 100031f8     libvcruntime:undname.obj
 0001:00002218       ??_C@_0BN@IMDCHIKM@?$GAscalar?5deleting?5destructor?8@ 10003218     libvcruntime:undname.obj
 0001:00002238       ??_C@_0BO@PFGOCPJJ@?$GAvector?5constructor?5iterator?8@ 10003238     libvcruntime:undname.obj
 0001:00002258       ??_C@_0BN@LFPFMEDL@?$GAvector?5destructor?5iterator?8@ 10003258     libvcruntime:undname.obj
 0001:00002278       ??_C@_0CE@IKBNEHA@?$GAvector?5vbase?5constructor?5itera@ 10003278     libvcruntime:undname.obj
 0001:0000229c       ??_C@_0BL@NILFHHPC@?$GAvirtual?5displacement?5map?8@ 1000329c     libvcruntime:undname.obj
 0001:000022b8       ??_C@_0CB@JONCMFFK@?$GAeh?5vector?5constructor?5iterator@ 100032b8     libvcruntime:undname.obj
 0001:000022dc       ??_C@_0CA@GCEOPDGL@?$GAeh?5vector?5destructor?5iterator?8@ 100032dc     libvcruntime:undname.obj
 0001:000022fc       ??_C@_0CH@OOJPLCPH@?$GAeh?5vector?5vbase?5constructor?5it@ 100032fc     libvcruntime:undname.obj
 0001:00002324       ??_C@_0BL@LLKPOHJI@?$GAcopy?5constructor?5closure?8@ 10003324     libvcruntime:undname.obj
 0001:00002340       ??_C@_0BA@KBCDOMBN@?$GAudt?5returning?8@ 10003340     libvcruntime:undname.obj
 0001:00002350       ??_C@_03KLGMFNMG@?$GAEH@   10003350     libvcruntime:undname.obj
 0001:00002354       ??_C@_05KHLCHHI@?$GARTTI@  10003354     libvcruntime:undname.obj
 0001:0000235c       ??_C@_0BA@KKLDJDLB@?$GAlocal?5vftable?8@ 1000335c     libvcruntime:undname.obj
 0001:0000236c       ??_C@_0CE@IIHCMGGL@?$GAlocal?5vftable?5constructor?5clos@ 1000336c     libvcruntime:undname.obj
 0001:00002390       ??_C@_06FHBGPFGH@?5new?$FL?$FN@ 10003390     libvcruntime:undname.obj
 0001:00002398       ??_C@_09LBNFPBCA@?5delete?$FL?$FN@ 10003398     libvcruntime:undname.obj
 0001:000023a4       ??_C@_0P@HJKNJFNN@?$GAomni?5callsig?8@ 100033a4     libvcruntime:undname.obj
 0001:000023b4       ??_C@_0BL@CNOONJFP@?$GAplacement?5delete?5closure?8@ 100033b4     libvcruntime:undname.obj
 0001:000023d0       ??_C@_0BN@CKNJLHMB@?$GAplacement?5delete?$FL?$FN?5closure?8@ 100033d0     libvcruntime:undname.obj
 0001:000023f0       ??_C@_0CG@CFDHKGGD@?$GAmanaged?5vector?5constructor?5ite@ 100033f0     libvcruntime:undname.obj
 0001:00002418       ??_C@_0CF@IMGKMJNO@?$GAmanaged?5vector?5destructor?5iter@ 10003418     libvcruntime:undname.obj
 0001:00002440       ??_C@_0CG@HLDDJMAG@?$GAeh?5vector?5copy?5constructor?5ite@ 10003440     libvcruntime:undname.obj
 0001:00002468       ??_C@_0CM@FCBBDIGB@?$GAeh?5vector?5vbase?5copy?5construct@ 10003468     libvcruntime:undname.obj
 0001:00002494       ??_C@_0BL@CLIPGLGB@?$GAdynamic?5initializer?5for?5?8@ 10003494     libvcruntime:undname.obj
 0001:000024b0       ??_C@_0CB@PDBIFEP@?$GAdynamic?5atexit?5destructor?5for?5@ 100034b0     libvcruntime:undname.obj
 0001:000024d4       ??_C@_0CD@CGAJBKEJ@?$GAvector?5copy?5constructor?5iterat@ 100034d4     libvcruntime:undname.obj
 0001:000024f8       ??_C@_0CJ@GJELGAMM@?$GAvector?5vbase?5copy?5constructor?5@ 100034f8     libvcruntime:undname.obj
 0001:00002524       ??_C@_0CL@FGIJHLCE@?$GAmanaged?5vector?5copy?5constructo@ 10003524     libvcruntime:undname.obj
 0001:00002550       ??_C@_0BM@PMGGMLDN@?$GAlocal?5static?5thread?5guard?8@ 10003550     libvcruntime:undname.obj
 0001:0000256c       ??_C@_0N@BDNMDMOL@operator?5?$CC?$CC?5@ 1000356c     libvcruntime:undname.obj
 0001:0000257c       ??_C@_0BC@GGEBGALA@operator?5co_await@ 1000357c     libvcruntime:undname.obj
 0001:00002590       ??_C@_0BC@DAFEJGAK@?5Type?5Descriptor?8@ 10003590     libvcruntime:undname.obj
 0001:000025a4       ??_C@_0BM@LDKODKLH@?5Base?5Class?5Descriptor?5at?5?$CI@ 100035a4     libvcruntime:undname.obj
 0001:000025c0       ??_C@_0BD@LGICGFMM@?5Base?5Class?5Array?8@ 100035c0     libvcruntime:undname.obj
 0001:000025d4       ??_C@_0BN@MECKDCOJ@?5Class?5Hierarchy?5Descriptor?8@ 100035d4     libvcruntime:undname.obj
 0001:000025f4       ??_C@_0BK@CFCOFLF@?5Complete?5Object?5Locator?8@ 100035f4     libvcruntime:undname.obj
 0001:00002610       __pDestructExceptionObject 10003610     libvcruntime:ehhelpers.obj
 0001:00002618       ___acrt_exception_action_table 10003618     libucrt:exception_filter.obj
 0001:000026a8       ___acrt_signal_action_table_count 100036a8     libucrt:exception_filter.obj
 0001:000026ac       ___acrt_signal_action_first_fpe_index 100036ac     libucrt:exception_filter.obj
 0001:000026b0       ___acrt_signal_action_fpe_count 100036b0     libucrt:exception_filter.obj
 0001:000026b4       ??_C@_1BI@BGOHAHKC@?$AAm?$AAs?$AAc?$AAo?$AAr?$AAe?$AAe?$AA?4?$AAd?$AAl?$AAl?$AA?$AA@ 100036b4     libucrt:exit.obj
 0001:000026cc       ??_C@_0P@MIGLKIOC@CorExitProcess?$AA@ 100036cc     libucrt:exit.obj
 0001:000028c8       ___lc_time_c               100038c8     libucrt:nlsdata.obj
 0001:00002a2c       ??_C@_03KOEHGMDN@Sun?$AA@  10003a2c     libucrt:nlsdata.obj
 0001:00002a30       ??_C@_03PDAGKDH@Mon?$AA@   10003a30     libucrt:nlsdata.obj
 0001:00002a34       ??_C@_03NAGEINEP@Tue?$AA@  10003a34     libucrt:nlsdata.obj
 0001:00002a38       ??_C@_03MHOMLAJA@Wed?$AA@  10003a38     libucrt:nlsdata.obj
 0001:00002a3c       ??_C@_03IOFIKPDN@Thu?$AA@  10003a3c     libucrt:nlsdata.obj
 0001:00002a40       ??_C@_03IDIOELNC@Fri?$AA@  10003a40     libucrt:nlsdata.obj
 0001:00002a44       ??_C@_03FEFJNEK@Sat?$AA@   10003a44     libucrt:nlsdata.obj
 0001:00002a48       ??_C@_06OOPIFAJ@Sunday?$AA@ 10003a48     libucrt:nlsdata.obj
 0001:00002a50       ??_C@_06JLEDEDGH@Monday?$AA@ 10003a50     libucrt:nlsdata.obj
 0001:00002a58       ??_C@_07BAAGCFCM@Tuesday?$AA@ 10003a58     libucrt:nlsdata.obj
 0001:00002a60       ??_C@_09DLIGFAKA@Wednesday?$AA@ 10003a60     libucrt:nlsdata.obj
 0001:00002a6c       ??_C@_08HACCIKIA@Thursday?$AA@ 10003a6c     libucrt:nlsdata.obj
 0001:00002a78       ??_C@_06JECMNKMI@Friday?$AA@ 10003a78     libucrt:nlsdata.obj
 0001:00002a80       ??_C@_08INBOOONO@Saturday?$AA@ 10003a80     libucrt:nlsdata.obj
 0001:00002a8c       ??_C@_03JIHJHPIE@Jan?$AA@  10003a8c     libucrt:nlsdata.obj
 0001:00002a90       ??_C@_03HJBDCHOM@Feb?$AA@  10003a90     libucrt:nlsdata.obj
 0001:00002a94       ??_C@_03ODNJBKGA@Mar?$AA@  10003a94     libucrt:nlsdata.obj
 0001:00002a98       ??_C@_03LEOLGMJP@Apr?$AA@  10003a98     libucrt:nlsdata.obj
 0001:00002a9c       ??_C@_03CNMDKL@May?$AA@    10003a9c     libucrt:nlsdata.obj
 0001:00002aa0       ??_C@_03IDFGHECI@Jun?$AA@  10003aa0     libucrt:nlsdata.obj
 0001:00002aa4       ??_C@_03LBGABGKK@Jul?$AA@  10003aa4     libucrt:nlsdata.obj
 0001:00002aa8       ??_C@_03IFJFEIGA@Aug?$AA@  10003aa8     libucrt:nlsdata.obj
 0001:00002aac       ??_C@_03GGCAPAJC@Sep?$AA@  10003aac     libucrt:nlsdata.obj
 0001:00002ab0       ??_C@_03BMAOKBAD@Oct?$AA@  10003ab0     libucrt:nlsdata.obj
 0001:00002ab4       ??_C@_03JPJOFNIA@Nov?$AA@  10003ab4     libucrt:nlsdata.obj
 0001:00002ab8       ??_C@_03MKABNOCG@Dec?$AA@  10003ab8     libucrt:nlsdata.obj
 0001:00002abc       ??_C@_07CGJPFGJA@January?$AA@ 10003abc     libucrt:nlsdata.obj
 0001:00002ac4       ??_C@_08GNJGEPFN@February?$AA@ 10003ac4     libucrt:nlsdata.obj
 0001:00002ad0       ??_C@_05HPCKOFNC@March?$AA@ 10003ad0     libucrt:nlsdata.obj
 0001:00002ad8       ??_C@_05DMJDNLEJ@April?$AA@ 10003ad8     libucrt:nlsdata.obj
 0001:00002ae0       ??_C@_04CNLMGBGM@June?$AA@ 10003ae0     libucrt:nlsdata.obj
 0001:00002ae8       ??_C@_04MIEPOIFP@July?$AA@ 10003ae8     libucrt:nlsdata.obj
 0001:00002af0       ??_C@_06LBBHFDDG@August?$AA@ 10003af0     libucrt:nlsdata.obj
 0001:00002af8       ??_C@_09BHHEALKD@September?$AA@ 10003af8     libucrt:nlsdata.obj
 0001:00002b04       ??_C@_07JJNFCEND@October?$AA@ 10003b04     libucrt:nlsdata.obj
 0001:00002b0c       ??_C@_08HCHEGEOA@November?$AA@ 10003b0c     libucrt:nlsdata.obj
 0001:00002b18       ??_C@_08EDHMEBNP@December?$AA@ 10003b18     libucrt:nlsdata.obj
 0001:00002b24       ??_C@_02DEDBPAFC@AM?$AA@   10003b24     libucrt:nlsdata.obj
 0001:00002b28       ??_C@_02CJNFDJBF@PM?$AA@   10003b28     libucrt:nlsdata.obj
 0001:00002b2c       ??_C@_08BPBNCDIB@MM?1dd?1yy?$AA@ 10003b2c     libucrt:nlsdata.obj
 0001:00002b38       ??_C@_0BE@CKGJFCPC@dddd?0?5MMMM?5dd?0?5yyyy?$AA@ 10003b38     libucrt:nlsdata.obj
 0001:00002b4c       ??_C@_08JCCMCCIL@HH?3mm?3ss?$AA@ 10003b4c     libucrt:nlsdata.obj
 0001:00002b58       ??_C@_17MBGCMIPB@?$AAS?$AAu?$AAn?$AA?$AA@ 10003b58     libucrt:nlsdata.obj
 0001:00002b60       ??_C@_17KBOMKBF@?$AAM?$AAo?$AAn?$AA?$AA@ 10003b60     libucrt:nlsdata.obj
 0001:00002b68       ??_C@_17BMKGEGOJ@?$AAT?$AAu?$AAe?$AA?$AA@ 10003b68     libucrt:nlsdata.obj
 0001:00002b70       ??_C@_17CJEDCEPE@?$AAW?$AAe?$AAd?$AA?$AA@ 10003b70     libucrt:nlsdata.obj
 0001:00002b78       ??_C@_17PDPHAADD@?$AAT?$AAh?$AAu?$AA?$AA@ 10003b78     libucrt:nlsdata.obj
 0001:00002b80       ??_C@_17HFOLPPLP@?$AAF?$AAr?$AAi?$AA?$AA@ 10003b80     libucrt:nlsdata.obj
 0001:00002b88       ??_C@_17GGIBDPIH@?$AAS?$AAa?$AAt?$AA?$AA@ 10003b88     libucrt:nlsdata.obj
 0001:00002b90       ??_C@_1O@IHNHDHPB@?$AAS?$AAu?$AAn?$AAd?$AAa?$AAy?$AA?$AA@ 10003b90     libucrt:nlsdata.obj
 0001:00002ba0       ??_C@_1O@MMNBFLIA@?$AAM?$AAo?$AAn?$AAd?$AAa?$AAy?$AA?$AA@ 10003ba0     libucrt:nlsdata.obj
 0001:00002bb0       ??_C@_1BA@ENFBFFEK@?$AAT?$AAu?$AAe?$AAs?$AAd?$AAa?$AAy?$AA?$AA@ 10003bb0     libucrt:nlsdata.obj
 0001:00002bc0       ??_C@_1BE@EBOGMDOH@?$AAW?$AAe?$AAd?$AAn?$AAe?$AAs?$AAd?$AAa?$AAy?$AA?$AA@ 10003bc0     libucrt:nlsdata.obj
 0001:00002bd4       ??_C@_1BC@HHMNLIHE@?$AAT?$AAh?$AAu?$AAr?$AAs?$AAd?$AAa?$AAy?$AA?$AA@ 10003bd4     libucrt:nlsdata.obj
 0001:00002be8       ??_C@_1O@PDICJHAG@?$AAF?$AAr?$AAi?$AAd?$AAa?$AAy?$AA?$AA@ 10003be8     libucrt:nlsdata.obj
 0001:00002bf8       ??_C@_1BC@ENMNNPAJ@?$AAS?$AAa?$AAt?$AAu?$AAr?$AAd?$AAa?$AAy?$AA?$AA@ 10003bf8     libucrt:nlsdata.obj
 0001:00002c0c       ??_C@_17DKNBKCHM@?$AAJ?$AAa?$AAn?$AA?$AA@ 10003c0c     libucrt:nlsdata.obj
 0001:00002c14       ??_C@_17LMDJEKJN@?$AAF?$AAe?$AAb?$AA?$AA@ 10003c14     libucrt:nlsdata.obj
 0001:00002c1c       ??_C@_17CKNLEDEC@?$AAM?$AAa?$AAr?$AA?$AA@ 10003c1c     libucrt:nlsdata.obj
 0001:00002c24       ??_C@_17LFPOIHDD@?$AAA?$AAp?$AAr?$AA?$AA@ 10003c24     libucrt:nlsdata.obj
 0001:00002c2c       ??_C@_17PNNKMEED@?$AAM?$AAa?$AAy?$AA?$AA@ 10003c2c     libucrt:nlsdata.obj
 0001:00002c34       ??_C@_17KCJGOCPB@?$AAJ?$AAu?$AAn?$AA?$AA@ 10003c34     libucrt:nlsdata.obj
 0001:00002c3c       ??_C@_17IJPCKHK@?$AAJ?$AAu?$AAl?$AA?$AA@ 10003c3c     libucrt:nlsdata.obj
 0001:00002c44       ??_C@_17ICPELBCN@?$AAA?$AAu?$AAg?$AA?$AA@ 10003c44     libucrt:nlsdata.obj
 0001:00002c4c       ??_C@_17HCHCOKMG@?$AAS?$AAe?$AAp?$AA?$AA@ 10003c4c     libucrt:nlsdata.obj
 0001:00002c54       ??_C@_17FNLKOI@?$AAO?$AAc?$AAt?$AA?$AA@ 10003c54     libucrt:nlsdata.obj
 0001:00002c5c       ??_C@_17BBDMLCIG@?$AAN?$AAo?$AAv?$AA?$AA@ 10003c5c     libucrt:nlsdata.obj
 0001:00002c64       ??_C@_17EGKACKIF@?$AAD?$AAe?$AAc?$AA?$AA@ 10003c64     libucrt:nlsdata.obj
 0001:00002c6c       ??_C@_1BA@EFMEIEBA@?$AAJ?$AAa?$AAn?$AAu?$AAa?$AAr?$AAy?$AA?$AA@ 10003c6c     libucrt:nlsdata.obj
 0001:00002c7c       ??_C@_1BC@JGDDFFAM@?$AAF?$AAe?$AAb?$AAr?$AAu?$AAa?$AAr?$AAy?$AA?$AA@ 10003c7c     libucrt:nlsdata.obj
 0001:00002c90       ??_C@_1M@IKEENEDF@?$AAM?$AAa?$AAr?$AAc?$AAh?$AA?$AA@ 10003c90     libucrt:nlsdata.obj
 0001:00002c9c       ??_C@_1M@GJNLMHFD@?$AAA?$AAp?$AAr?$AAi?$AAl?$AA?$AA@ 10003c9c     libucrt:nlsdata.obj
 0001:00002ca8       ??_C@_19EPFLPGAP@?$AAJ?$AAu?$AAn?$AAe?$AA?$AA@ 10003ca8     libucrt:nlsdata.obj
 0001:00002cb4       ??_C@_19BIFMLPCD@?$AAJ?$AAu?$AAl?$AAy?$AA?$AA@ 10003cb4     libucrt:nlsdata.obj
 0001:00002cc0       ??_C@_1O@PAHLKOAC@?$AAA?$AAu?$AAg?$AAu?$AAs?$AAt?$AA?$AA@ 10003cc0     libucrt:nlsdata.obj
 0001:00002cd0       ??_C@_1BE@DKAAMBJL@?$AAS?$AAe?$AAp?$AAt?$AAe?$AAm?$AAb?$AAe?$AAr?$AA?$AA@ 10003cd0     libucrt:nlsdata.obj
 0001:00002ce4       ??_C@_1BA@EPANDLNG@?$AAO?$AAc?$AAt?$AAo?$AAb?$AAe?$AAr?$AA?$AA@ 10003ce4     libucrt:nlsdata.obj
 0001:00002cf4       ??_C@_1BC@BGLIFPF@?$AAN?$AAo?$AAv?$AAe?$AAm?$AAb?$AAe?$AAr?$AA?$AA@ 10003cf4     libucrt:nlsdata.obj
 0001:00002d08       ??_C@_1BC@FEMKIFH@?$AAD?$AAe?$AAc?$AAe?$AAm?$AAb?$AAe?$AAr?$AA?$AA@ 10003d08     libucrt:nlsdata.obj
 0001:00002d1c       ??_C@_15ODEHAHHF@?$AAA?$AAM?$AA?$AA@ 10003d1c     libucrt:nlsdata.obj
 0001:00002d24       ??_C@_15CLMNNGEL@?$AAP?$AAM?$AA?$AA@ 10003d24     libucrt:nlsdata.obj
 0001:00002d2c       ??_C@_1BC@IEBCMHCM@?$AAM?$AAM?$AA?1?$AAd?$AAd?$AA?1?$AAy?$AAy?$AA?$AA@ 10003d2c     libucrt:nlsdata.obj
 0001:00002d40       ??_C@_1CI@KNAKOEBC@?$AAd?$AAd?$AAd?$AAd?$AA?0?$AA?5?$AAM?$AAM?$AAM?$AAM?$AA?5?$AAd?$AAd?$AA?0?$AA?5?$AAy?$AAy?$AAy?$AAy?$AA?$AA@ 10003d40     libucrt:nlsdata.obj
 0001:00002d68       ??_C@_1BC@GDGBMEMK@?$AAH?$AAH?$AA?3?$AAm?$AAm?$AA?3?$AAs?$AAs?$AA?$AA@ 10003d68     libucrt:nlsdata.obj
 0001:00002d7c       ??_C@_1M@BMHNFIME@?$AAe?$AAn?$AA?9?$AAU?$AAS?$AA?$AA@ 10003d7c     libucrt:nlsdata.obj
 0001:00002d88       ___newctype                10003d88     libucrt:ctype.obj
 0001:00003088       ___newclmap                10004088     libucrt:ctype.obj
 0001:00003208       ___newcumap                10004208     libucrt:ctype.obj
 0001:00003388       __wctype                   10004388     libucrt:ctype.obj
 0001:0000359c       ??_C@_1M@HPNHIDJI@?$AAj?$AAa?$AA?9?$AAJ?$AAP?$AA?$AA@ 1000459c     libucrt:mbctype.obj
 0001:000035a8       ??_C@_1M@BIBDDEMK@?$AAz?$AAh?$AA?9?$AAC?$AAN?$AA?$AA@ 100045a8     libucrt:mbctype.obj
 0001:000035b4       ??_C@_1M@JLOOOEGK@?$AAk?$AAo?$AA?9?$AAK?$AAR?$AA?$AA@ 100045b4     libucrt:mbctype.obj
 0001:000035c0       ??_C@_1M@CLNBBOPM@?$AAz?$AAh?$AA?9?$AAT?$AAW?$AA?$AA@ 100045c0     libucrt:mbctype.obj
 0001:00003620       ??_C@_1EA@JGEFHKEI@?$AAa?$AAp?$AAi?$AA?9?$AAm?$AAs?$AA?9?$AAw?$AAi?$AAn?$AA?9?$AAc?$AAo?$AAr?$AAe?$AA?9?$AAd?$AAa?$AAt?$AAe?$AAt?$AAi?$AAm?$AAe?$AA?9?$AAl?$AA1?$AA?9?$AA1?$AA?9?$AA1?$AA?$AA@ 10004620     libucrt:winapi_thunks.obj
 0001:00003660       ??_C@_1DM@KHCHBNEB@?$AAa?$AAp?$AAi?$AA?9?$AAm?$AAs?$AA?9?$AAw?$AAi?$AAn?$AA?9?$AAc?$AAo?$AAr?$AAe?$AA?9?$AAf?$AAi?$AAb?$AAe?$AAr?$AAs?$AA?9?$AAl?$AA1?$AA?9?$AA1?$AA?9?$AA1?$AA?$AA@ 10004660     libucrt:winapi_thunks.obj
 0001:0000369c       ??_C@_1DI@IJCEHOCB@?$AAa?$AAp?$AAi?$AA?9?$AAm?$AAs?$AA?9?$AAw?$AAi?$AAn?$AA?9?$AAc?$AAo?$AAr?$AAe?$AA?9?$AAf?$AAi?$AAl?$AAe?$AA?9?$AAl?$AA1?$AA?9?$AA2?$AA?9?$AA2?$AA?$AA@ 1000469c     libucrt:winapi_thunks.obj
 0001:000036d8       ??_C@_1EI@MPIAOHOC@?$AAa?$AAp?$AAi?$AA?9?$AAm?$AAs?$AA?9?$AAw?$AAi?$AAn?$AA?9?$AAc?$AAo?$AAr?$AAe?$AA?9?$AAl?$AAo?$AAc?$AAa?$AAl?$AAi?$AAz?$AAa?$AAt?$AAi?$AAo?$AAn?$AA?9?$AAl?$AA1?$AA?9@ 100046d8     libucrt:winapi_thunks.obj
 0001:00003720       ??_C@_1FK@FPHCKFIE@?$AAa?$AAp?$AAi?$AA?9?$AAm?$AAs?$AA?9?$AAw?$AAi?$AAn?$AA?9?$AAc?$AAo?$AAr?$AAe?$AA?9?$AAl?$AAo?$AAc?$AAa?$AAl?$AAi?$AAz?$AAa?$AAt?$AAi?$AAo?$AAn?$AA?9?$AAo?$AAb?$AAs@ 10004720     libucrt:winapi_thunks.obj
 0001:00003780       ??_C@_1EM@DILCGIIO@?$AAa?$AAp?$AAi?$AA?9?$AAm?$AAs?$AA?9?$AAw?$AAi?$AAn?$AA?9?$AAc?$AAo?$AAr?$AAe?$AA?9?$AAp?$AAr?$AAo?$AAc?$AAe?$AAs?$AAs?$AAt?$AAh?$AAr?$AAe?$AAa?$AAd?$AAs?$AA?9?$AAl@ 10004780     libucrt:winapi_thunks.obj
 0001:000037cc       ??_C@_1DM@LNCGDDPN@?$AAa?$AAp?$AAi?$AA?9?$AAm?$AAs?$AA?9?$AAw?$AAi?$AAn?$AA?9?$AAc?$AAo?$AAr?$AAe?$AA?9?$AAs?$AAt?$AAr?$AAi?$AAn?$AAg?$AA?9?$AAl?$AA1?$AA?9?$AA1?$AA?9?$AA0?$AA?$AA@ 100047cc     libucrt:winapi_thunks.obj
 0001:00003808       ??_C@_1DK@LPPGFMPP@?$AAa?$AAp?$AAi?$AA?9?$AAm?$AAs?$AA?9?$AAw?$AAi?$AAn?$AA?9?$AAc?$AAo?$AAr?$AAe?$AA?9?$AAs?$AAy?$AAn?$AAc?$AAh?$AA?9?$AAl?$AA1?$AA?9?$AA2?$AA?9?$AA0?$AA?$AA@ 10004808     libucrt:winapi_thunks.obj
 0001:00003844       ??_C@_1DO@FPAPJEMD@?$AAa?$AAp?$AAi?$AA?9?$AAm?$AAs?$AA?9?$AAw?$AAi?$AAn?$AA?9?$AAc?$AAo?$AAr?$AAe?$AA?9?$AAs?$AAy?$AAs?$AAi?$AAn?$AAf?$AAo?$AA?9?$AAl?$AA1?$AA?9?$AA2?$AA?9?$AA1?$AA?$AA@ 10004844     libucrt:winapi_thunks.obj
 0001:00003884       ??_C@_1DK@NDHNAHIO@?$AAa?$AAp?$AAi?$AA?9?$AAm?$AAs?$AA?9?$AAw?$AAi?$AAn?$AA?9?$AAc?$AAo?$AAr?$AAe?$AA?9?$AAw?$AAi?$AAn?$AAr?$AAt?$AA?9?$AAl?$AA1?$AA?9?$AA1?$AA?9?$AA0?$AA?$AA@ 10004884     libucrt:winapi_thunks.obj
 0001:000038c0       ??_C@_1DM@KGHDGBCM@?$AAa?$AAp?$AAi?$AA?9?$AAm?$AAs?$AA?9?$AAw?$AAi?$AAn?$AA?9?$AAc?$AAo?$AAr?$AAe?$AA?9?$AAx?$AAs?$AAt?$AAa?$AAt?$AAe?$AA?9?$AAl?$AA2?$AA?9?$AA1?$AA?9?$AA0?$AA?$AA@ 100048c0     libucrt:winapi_thunks.obj
 0001:00003900       ??_C@_1EO@IJIOEFOH@?$AAa?$AAp?$AAi?$AA?9?$AAm?$AAs?$AA?9?$AAw?$AAi?$AAn?$AA?9?$AAr?$AAt?$AAc?$AAo?$AAr?$AAe?$AA?9?$AAn?$AAt?$AAu?$AAs?$AAe?$AAr?$AA?9?$AAw?$AAi?$AAn?$AAd?$AAo?$AAw?$AA?9@ 10004900     libucrt:winapi_thunks.obj
 0001:00003950       ??_C@_1FG@HHGEKANL@?$AAa?$AAp?$AAi?$AA?9?$AAm?$AAs?$AA?9?$AAw?$AAi?$AAn?$AA?9?$AAs?$AAe?$AAc?$AAu?$AAr?$AAi?$AAt?$AAy?$AA?9?$AAs?$AAy?$AAs?$AAt?$AAe?$AAm?$AAf?$AAu?$AAn?$AAc?$AAt?$AAi@ 10004950     libucrt:winapi_thunks.obj
 0001:000039a8       ??_C@_1EG@DBIOJECG@?$AAe?$AAx?$AAt?$AA?9?$AAm?$AAs?$AA?9?$AAw?$AAi?$AAn?$AA?9?$AAn?$AAt?$AAu?$AAs?$AAe?$AAr?$AA?9?$AAd?$AAi?$AAa?$AAl?$AAo?$AAg?$AAb?$AAo?$AAx?$AA?9?$AAl?$AA1?$AA?9?$AA1@ 100049a8     libucrt:winapi_thunks.obj
 0001:000039f0       ??_C@_1EO@FIHMJCLF@?$AAe?$AAx?$AAt?$AA?9?$AAm?$AAs?$AA?9?$AAw?$AAi?$AAn?$AA?9?$AAn?$AAt?$AAu?$AAs?$AAe?$AAr?$AA?9?$AAw?$AAi?$AAn?$AAd?$AAo?$AAw?$AAs?$AAt?$AAa?$AAt?$AAi?$AAo?$AAn?$AA?9@ 100049f0     libucrt:winapi_thunks.obj
 0001:00003a40       ??_C@_1BC@DNHGCMLG@?$AAa?$AAd?$AAv?$AAa?$AAp?$AAi?$AA3?$AA2?$AA?$AA@ 10004a40     libucrt:winapi_thunks.obj
 0001:00003a54       ??_C@_1BC@GDMECMAK@?$AAk?$AAe?$AAr?$AAn?$AAe?$AAl?$AA3?$AA2?$AA?$AA@ 10004a54     libucrt:winapi_thunks.obj
 0001:00003a68       ??_C@_1M@OAIMIKLP@?$AAn?$AAt?$AAd?$AAl?$AAl?$AA?$AA@ 10004a68     libucrt:winapi_thunks.obj
 0001:00003a78       ??_C@_1EG@DPGNFKGC@?$AAa?$AAp?$AAi?$AA?9?$AAm?$AAs?$AA?9?$AAw?$AAi?$AAn?$AA?9?$AAa?$AAp?$AAp?$AAm?$AAo?$AAd?$AAe?$AAl?$AA?9?$AAr?$AAu?$AAn?$AAt?$AAi?$AAm?$AAe?$AA?9?$AAl?$AA1?$AA?9?$AA1@ 10004a78     libucrt:winapi_thunks.obj
 0001:00003ac0       ??_C@_1O@BCCLBEOE@?$AAu?$AAs?$AAe?$AAr?$AA3?$AA2?$AA?$AA@ 10004ac0     libucrt:winapi_thunks.obj
 0001:00003ad0       ??_C@_1BA@PFFKHIOG@?$AAa?$AAp?$AAi?$AA?9?$AAm?$AAs?$AA?9?$AA?$AA@ 10004ad0     libucrt:winapi_thunks.obj
 0001:00003ae0       ??_C@_1BA@IAIFMGEF@?$AAe?$AAx?$AAt?$AA?9?$AAm?$AAs?$AA?9?$AA?$AA@ 10004ae0     libucrt:winapi_thunks.obj
 0001:00003af4       ??_C@_0BA@FHFNEAED@AreFileApisANSI?$AA@ 10004af4     libucrt:winapi_thunks.obj
 0001:00003b0c       ??_C@_08KNHFBNJ@FlsAlloc?$AA@ 10004b0c     libucrt:winapi_thunks.obj
 0001:00003b20       ??_C@_07PEJMOBNF@FlsFree?$AA@ 10004b20     libucrt:winapi_thunks.obj
 0001:00003b30       ??_C@_0M@GDNOONDI@FlsGetValue?$AA@ 10004b30     libucrt:winapi_thunks.obj
 0001:00003b44       ??_C@_0M@JCPCPOEF@FlsSetValue?$AA@ 10004b44     libucrt:winapi_thunks.obj
 0001:00003b58       ??_C@_0BM@HCFOFFN@InitializeCriticalSectionEx?$AA@ 10004b58     libucrt:winapi_thunks.obj
 0001:00003b7c       ??_C@_0O@KKBNKAPF@LCMapStringEx?$AA@ 10004b7c     libucrt:winapi_thunks.obj
 0001:00003b94       ??_C@_0BB@HBDEELFH@LocaleNameToLCID?$AA@ 10004b94     libucrt:winapi_thunks.obj
 0001:00003bac       ??_C@_0CF@OJOFEIGO@AppPolicyGetProcessTerminationMe@ 10004bac     libucrt:winapi_thunks.obj
 0001:00003bd4       ??_C@_15PJPFLCCM@?$AAu?$AAk?$AA?$AA@ 10004bd4     libucrt:get_qualified_locale.obj
 0001:00004300       ??_C@_15EMKDOKLE@?$AAa?$AAr?$AA?$AA@ 10005300     libucrt:lcidtoname_downlevel.obj
 0001:00004308       ??_C@_15KNPADPLH@?$AAb?$AAg?$AA?$AA@ 10005308     libucrt:lcidtoname_downlevel.obj
 0001:00004310       ??_C@_15EDMHLDMO@?$AAc?$AAa?$AA?$AA@ 10005310     libucrt:lcidtoname_downlevel.obj
 0001:00004318       ??_C@_1O@BPEAJADD@?$AAz?$AAh?$AA?9?$AAC?$AAH?$AAS?$AA?$AA@ 10005318     libucrt:lcidtoname_downlevel.obj
 0001:00004328       ??_C@_15LJNHCMNK@?$AAc?$AAs?$AA?$AA@ 10005328     libucrt:lcidtoname_downlevel.obj
 0001:00004330       ??_C@_15FOMCIDHG@?$AAd?$AAa?$AA?$AA@ 10005330     libucrt:lcidtoname_downlevel.obj
 0001:00004338       ??_C@_15NBKABECB@?$AAd?$AAe?$AA?$AA@ 10005338     libucrt:lcidtoname_downlevel.obj
 0001:00004340       ??_C@_15GHPEIIAO@?$AAe?$AAl?$AA?$AA@ 10005340     libucrt:lcidtoname_downlevel.obj
 0001:00004348       ??_C@_15MNPNEAIF@?$AAe?$AAn?$AA?$AA@ 10005348     libucrt:lcidtoname_downlevel.obj
 0001:00004350       ??_C@_15GPIOMPMH@?$AAe?$AAs?$AA?$AA@ 10005350     libucrt:lcidtoname_downlevel.obj
 0001:00004358       ??_C@_15NGLOAKJC@?$AAf?$AAi?$AA?$AA@ 10005358     libucrt:lcidtoname_downlevel.obj
 0001:00004360       ??_C@_15FBKGNKAM@?$AAf?$AAr?$AA?$AA@ 10005360     libucrt:lcidtoname_downlevel.obj
 0001:00004368       ??_C@_15KGGCNEFK@?$AAh?$AAe?$AA?$AA@ 10005368     libucrt:lcidtoname_downlevel.obj
 0001:00004370       ??_C@_15PGHLIDMF@?$AAh?$AAu?$AA?$AA@ 10005370     libucrt:lcidtoname_downlevel.obj
 0001:00004378       ??_C@_15BIEMAPLM@?$AAi?$AAs?$AA?$AA@ 10005378     libucrt:lcidtoname_downlevel.obj
 0001:00004380       ??_C@_15IFJLDHAF@?$AAi?$AAt?$AA?$AA@ 10005380     libucrt:lcidtoname_downlevel.obj
 0001:00004388       ??_C@_15GEMIOCAG@?$AAj?$AAa?$AA?$AA@ 10005388     libucrt:lcidtoname_downlevel.obj
 0001:00004390       ??_C@_15EPELEGJA@?$AAk?$AAo?$AA?$AA@ 10005390     libucrt:lcidtoname_downlevel.obj
 0001:00004398       ??_C@_15NDDHIMN@?$AAn?$AAl?$AA?$AA@ 10005398     libucrt:lcidtoname_downlevel.obj
 0001:000043a0       ??_C@_15BPIGNHCD@?$AAn?$AAo?$AA?$AA@ 100053a0     libucrt:lcidtoname_downlevel.obj
 0001:000043a8       ??_C@_15DEOPBLCG@?$AAp?$AAl?$AA?$AA@ 100053a8     libucrt:lcidtoname_downlevel.obj
 0001:000043b0       ??_C@_15KBECGEFG@?$AAp?$AAt?$AA?$AA@ 100053b0     libucrt:lcidtoname_downlevel.obj
 0001:000043b8       ??_C@_15GLJCBFMD@?$AAr?$AAo?$AA?$AA@ 100053b8     libucrt:lcidtoname_downlevel.obj
 0001:000043c0       ??_C@_15FEDGKCDI@?$AAr?$AAu?$AA?$AA@ 100053c0     libucrt:lcidtoname_downlevel.obj
 0001:000043c8       ??_C@_15GLKMLLHM@?$AAh?$AAr?$AA?$AA@ 100053c8     libucrt:lcidtoname_downlevel.obj
 0001:000043d0       ??_C@_15CPKMFBDB@?$AAs?$AAk?$AA?$AA@ 100053d0     libucrt:lcidtoname_downlevel.obj
 0001:000043d8       ??_C@_15BAAIOGMK@?$AAs?$AAq?$AA?$AA@ 100053d8     libucrt:lcidtoname_downlevel.obj
 0001:000043e0       ??_C@_15INNPNOHD@?$AAs?$AAv?$AA?$AA@ 100053e0     libucrt:lcidtoname_downlevel.obj
 0001:000043e8       ??_C@_15CABMMOGH@?$AAt?$AAh?$AA?$AA@ 100053e8     libucrt:lcidtoname_downlevel.obj
 0001:000043f0       ??_C@_15BPLIHJJM@?$AAt?$AAr?$AA?$AA@ 100053f0     libucrt:lcidtoname_downlevel.obj
 0001:000043f8       ??_C@_15NEOEKKDJ@?$AAu?$AAr?$AA?$AA@ 100053f8     libucrt:lcidtoname_downlevel.obj
 0001:00004400       ??_C@_15NFICGAJK@?$AAi?$AAd?$AA?$AA@ 10005400     libucrt:lcidtoname_downlevel.obj
 0001:00004408       ??_C@_15HPJPHDM@?$AAb?$AAe?$AA?$AA@ 10005408     libucrt:lcidtoname_downlevel.obj
 0001:00004410       ??_C@_15LCHLGJII@?$AAs?$AAl?$AA?$AA@ 10005410     libucrt:lcidtoname_downlevel.obj
 0001:00004418       ??_C@_15PCFJPHHO@?$AAe?$AAt?$AA?$AA@ 10005418     libucrt:lcidtoname_downlevel.obj
 0001:00004420       ??_C@_15HPFPGODN@?$AAl?$AAv?$AA?$AA@ 10005420     libucrt:lcidtoname_downlevel.obj
 0001:00004428       ??_C@_15NFFGKGLG@?$AAl?$AAt?$AA?$AA@ 10005428     libucrt:lcidtoname_downlevel.obj
 0001:00004430       ??_C@_15BDAKCCHN@?$AAf?$AAa?$AA?$AA@ 10005430     libucrt:lcidtoname_downlevel.obj
 0001:00004438       ??_C@_15NFGIAIAJ@?$AAv?$AAi?$AA?$AA@ 10005438     libucrt:lcidtoname_downlevel.obj
 0001:00004440       ??_C@_15LMKNDMHN@?$AAh?$AAy?$AA?$AA@ 10005440     libucrt:lcidtoname_downlevel.obj
 0001:00004448       ??_C@_15IJBHMCFL@?$AAa?$AAz?$AA?$AA@ 10005448     libucrt:lcidtoname_downlevel.obj
 0001:00004450       ??_C@_15EKOFJABL@?$AAe?$AAu?$AA?$AA@ 10005450     libucrt:lcidtoname_downlevel.obj
 0001:00004458       ??_C@_15BGHADCNK@?$AAm?$AAk?$AA?$AA@ 10005458     libucrt:lcidtoname_downlevel.obj
 0001:00004460       ??_C@_15JDNICKHM@?$AAa?$AAf?$AA?$AA@ 10005460     libucrt:lcidtoname_downlevel.obj
 0001:00004468       ??_C@_15KPJEDBKD@?$AAk?$AAa?$AA?$AA@ 10005468     libucrt:lcidtoname_downlevel.obj
 0001:00004470       ??_C@_15PDNFFFEO@?$AAf?$AAo?$AA?$AA@ 10005470     libucrt:lcidtoname_downlevel.obj
 0001:00004478       ??_C@_15OMLEGLOC@?$AAh?$AAi?$AA?$AA@ 10005478     libucrt:lcidtoname_downlevel.obj
 0001:00004480       ??_C@_15IDNNENKK@?$AAm?$AAs?$AA?$AA@ 10005480     libucrt:lcidtoname_downlevel.obj
 0001:00004488       ??_C@_15MACJNBMH@?$AAk?$AAk?$AA?$AA@ 10005488     libucrt:lcidtoname_downlevel.obj
 0001:00004490       ??_C@_15DKDJEOND@?$AAk?$AAy?$AA?$AA@ 10005490     libucrt:lcidtoname_downlevel.obj
 0001:00004498       ??_C@_15DFGDLJBG@?$AAs?$AAw?$AA?$AA@ 10005498     libucrt:lcidtoname_downlevel.obj
 0001:000044a0       ??_C@_15BBFAICNG@?$AAu?$AAz?$AA?$AA@ 100054a0     libucrt:lcidtoname_downlevel.obj
 0001:000044a8       ??_C@_15DKNDCGEA@?$AAt?$AAt?$AA?$AA@ 100054a8     libucrt:lcidtoname_downlevel.obj
 0001:000044b0       ??_C@_15MGIFMDPL@?$AAp?$AAa?$AA?$AA@ 100054b0     libucrt:lcidtoname_downlevel.obj
 0001:000044b8       ??_C@_15HCNDBBA@?$AAg?$AAu?$AA?$AA@ 100054b8     libucrt:lcidtoname_downlevel.obj
 0001:000044c0       ??_C@_15FNBEIBON@?$AAt?$AAa?$AA?$AA@ 100054c0     libucrt:lcidtoname_downlevel.obj
 0001:000044c8       ??_C@_15NCHGBGLK@?$AAt?$AAe?$AA?$AA@ 100054c8     libucrt:lcidtoname_downlevel.obj
 0001:000044d0       ??_C@_15PHPHCBPF@?$AAk?$AAn?$AA?$AA@ 100054d0     libucrt:lcidtoname_downlevel.obj
 0001:000044d8       ??_C@_15DLGBCKMP@?$AAm?$AAr?$AA?$AA@ 100054d8     libucrt:lcidtoname_downlevel.obj
 0001:000044e0       ??_C@_15EABBLBFF@?$AAs?$AAa?$AA?$AA@ 100054e0     libucrt:lcidtoname_downlevel.obj
 0001:000044e8       ??_C@_15CBKOMCOI@?$AAm?$AAn?$AA?$AA@ 100054e8     libucrt:lcidtoname_downlevel.obj
 0001:000044f0       ??_C@_15CKDMCJAF@?$AAg?$AAl?$AA?$AA@ 100054f0     libucrt:lcidtoname_downlevel.obj
 0001:000044f8       ??_C@_17CNJFBPG@?$AAk?$AAo?$AAk?$AA?$AA@ 100054f8     libucrt:lcidtoname_downlevel.obj
 0001:00004500       ??_C@_17FFBJICPL@?$AAs?$AAy?$AAr?$AA?$AA@ 10005500     libucrt:lcidtoname_downlevel.obj
 0001:00004508       ??_C@_17KPNDCPAF@?$AAd?$AAi?$AAv?$AA?$AA@ 10005508     libucrt:lcidtoname_downlevel.obj
 0001:00004510       ??_C@_11LOCGONAA@?$AA?$AA@ 10005510     libucrt:lcidtoname_downlevel.obj
 0001:00004514       ??_C@_1M@OKAHONE@?$AAa?$AAr?$AA?9?$AAS?$AAA?$AA?$AA@ 10005514     libucrt:lcidtoname_downlevel.obj
 0001:00004520       ??_C@_1M@FFFIGIGK@?$AAb?$AAg?$AA?9?$AAB?$AAG?$AA?$AA@ 10005520     libucrt:lcidtoname_downlevel.obj
 0001:0000452c       ??_C@_1M@BJNKEDC@?$AAc?$AAa?$AA?9?$AAE?$AAS?$AA?$AA@ 1000552c     libucrt:lcidtoname_downlevel.obj
 0001:00004538       ??_C@_1M@IJJHFJHA@?$AAc?$AAs?$AA?9?$AAC?$AAZ?$AA?$AA@ 10005538     libucrt:lcidtoname_downlevel.obj
 0001:00004544       ??_C@_1M@CLPEOBGI@?$AAd?$AAa?$AA?9?$AAD?$AAK?$AA?$AA@ 10005544     libucrt:lcidtoname_downlevel.obj
 0001:00004550       ??_C@_1M@MCMADGCB@?$AAd?$AAe?$AA?9?$AAD?$AAE?$AA?$AA@ 10005550     libucrt:lcidtoname_downlevel.obj
 0001:0000455c       ??_C@_1M@OOCKEMAM@?$AAe?$AAl?$AA?9?$AAG?$AAR?$AA?$AA@ 1000555c     libucrt:lcidtoname_downlevel.obj
 0001:00004568       ??_C@_1M@DDNJFGID@?$AAf?$AAi?$AA?9?$AAF?$AAI?$AA?$AA@ 10005568     libucrt:lcidtoname_downlevel.obj
 0001:00004574       ??_C@_1M@GLIPPMAC@?$AAf?$AAr?$AA?9?$AAF?$AAR?$AA?$AA@ 10005574     libucrt:lcidtoname_downlevel.obj
 0001:00004580       ??_C@_1M@GFMCHPE@?$AAh?$AAe?$AA?9?$AAI?$AAL?$AA?$AA@ 10005580     libucrt:lcidtoname_downlevel.obj
 0001:0000458c       ??_C@_1M@MHLPGNKM@?$AAh?$AAu?$AA?9?$AAH?$AAU?$AA?$AA@ 1000558c     libucrt:lcidtoname_downlevel.obj
 0001:00004598       ??_C@_1M@LPDDNNPN@?$AAi?$AAs?$AA?9?$AAI?$AAS?$AA?$AA@ 10005598     libucrt:lcidtoname_downlevel.obj
 0001:000045a4       ??_C@_1M@MADIPODN@?$AAi?$AAt?$AA?9?$AAI?$AAT?$AA?$AA@ 100055a4     libucrt:lcidtoname_downlevel.obj
 0001:000045b0       ??_C@_1M@IHBJJGG@?$AAn?$AAl?$AA?9?$AAN?$AAL?$AA?$AA@ 100055b0     libucrt:lcidtoname_downlevel.obj
 0001:000045bc       ??_C@_1M@EANAGDL@?$AAn?$AAb?$AA?9?$AAN?$AAO?$AA?$AA@ 100055bc     libucrt:lcidtoname_downlevel.obj
 0001:000045c8       ??_C@_1M@NEIEMEGP@?$AAp?$AAl?$AA?9?$AAP?$AAL?$AA?$AA@ 100055c8     libucrt:lcidtoname_downlevel.obj
 0001:000045d4       ??_C@_1M@BOCFIGEP@?$AAp?$AAt?$AA?9?$AAB?$AAR?$AA?$AA@ 100055d4     libucrt:lcidtoname_downlevel.obj
 0001:000045e0       ??_C@_1M@IMPFOPBG@?$AAr?$AAo?$AA?9?$AAR?$AAO?$AA?$AA@ 100055e0     libucrt:lcidtoname_downlevel.obj
 0001:000045ec       ??_C@_1M@IDNNEJMM@?$AAr?$AAu?$AA?9?$AAR?$AAU?$AA?$AA@ 100055ec     libucrt:lcidtoname_downlevel.obj
 0001:000045f8       ??_C@_1M@LILEEOGM@?$AAh?$AAr?$AA?9?$AAH?$AAR?$AA?$AA@ 100055f8     libucrt:lcidtoname_downlevel.obj
 0001:00004604       ??_C@_1M@FKIFEHPB@?$AAs?$AAk?$AA?9?$AAS?$AAK?$AA?$AA@ 10005604     libucrt:lcidtoname_downlevel.obj
 0001:00004610       ??_C@_1M@LJMAMNPJ@?$AAs?$AAq?$AA?9?$AAA?$AAL?$AA?$AA@ 10005610     libucrt:lcidtoname_downlevel.obj
 0001:0000461c       ??_C@_1M@GIAKDKJK@?$AAs?$AAv?$AA?9?$AAS?$AAE?$AA?$AA@ 1000561c     libucrt:lcidtoname_downlevel.obj
 0001:00004628       ??_C@_1M@MKJKIKCL@?$AAt?$AAh?$AA?9?$AAT?$AAH?$AA?$AA@ 10005628     libucrt:lcidtoname_downlevel.obj
 0001:00004634       ??_C@_1M@MFLCCMPB@?$AAt?$AAr?$AA?9?$AAT?$AAR?$AA?$AA@ 10005634     libucrt:lcidtoname_downlevel.obj
 0001:00004640       ??_C@_1M@OIJHDKJN@?$AAu?$AAr?$AA?9?$AAP?$AAK?$AA?$AA@ 10005640     libucrt:lcidtoname_downlevel.obj
 0001:0000464c       ??_C@_1M@LHIPCIEK@?$AAi?$AAd?$AA?9?$AAI?$AAD?$AA?$AA@ 1000564c     libucrt:lcidtoname_downlevel.obj
 0001:00004658       ??_C@_1M@MFMOBGI@?$AAu?$AAk?$AA?9?$AAU?$AAA?$AA?$AA@ 10005658     libucrt:lcidtoname_downlevel.obj
 0001:00004664       ??_C@_1M@OBGLJIPL@?$AAb?$AAe?$AA?9?$AAB?$AAY?$AA?$AA@ 10005664     libucrt:lcidtoname_downlevel.obj
 0001:00004670       ??_C@_1M@BCFAJEAD@?$AAs?$AAl?$AA?9?$AAS?$AAI?$AA?$AA@ 10005670     libucrt:lcidtoname_downlevel.obj
 0001:0000467c       ??_C@_1M@FKFFEDDN@?$AAe?$AAt?$AA?9?$AAE?$AAE?$AA?$AA@ 1000567c     libucrt:lcidtoname_downlevel.obj
 0001:00004688       ??_C@_1M@KGKKAACI@?$AAl?$AAv?$AA?9?$AAL?$AAV?$AA?$AA@ 10005688     libucrt:lcidtoname_downlevel.obj
 0001:00004694       ??_C@_1M@IFGBIJO@?$AAl?$AAt?$AA?9?$AAL?$AAT?$AA?$AA@ 10005694     libucrt:lcidtoname_downlevel.obj
 0001:000046a0       ??_C@_1M@FGEAHEDM@?$AAf?$AAa?$AA?9?$AAI?$AAR?$AA?$AA@ 100056a0     libucrt:lcidtoname_downlevel.obj
 0001:000046ac       ??_C@_1M@KBMAIBFN@?$AAv?$AAi?$AA?9?$AAV?$AAN?$AA?$AA@ 100056ac     libucrt:lcidtoname_downlevel.obj
 0001:000046b8       ??_C@_1M@GPCBKDJK@?$AAh?$AAy?$AA?9?$AAA?$AAM?$AA?$AA@ 100056b8     libucrt:lcidtoname_downlevel.obj
 0001:000046c4       ??_C@_1BG@BECMDDJB@?$AAa?$AAz?$AA?9?$AAA?$AAZ?$AA?9?$AAL?$AAa?$AAt?$AAn?$AA?$AA@ 100056c4     libucrt:lcidtoname_downlevel.obj
 0001:000046dc       ??_C@_1M@MAOFCAEA@?$AAe?$AAu?$AA?9?$AAE?$AAS?$AA?$AA@ 100056dc     libucrt:lcidtoname_downlevel.obj
 0001:000046e8       ??_C@_1M@IGHABKPI@?$AAm?$AAk?$AA?9?$AAM?$AAK?$AA?$AA@ 100056e8     libucrt:lcidtoname_downlevel.obj
 0001:000046f4       ??_C@_1M@IAIGNEJG@?$AAt?$AAn?$AA?9?$AAZ?$AAA?$AA?$AA@ 100056f4     libucrt:lcidtoname_downlevel.obj
 0001:00004700       ??_C@_1M@IIJCOJFA@?$AAx?$AAh?$AA?9?$AAZ?$AAA?$AA?$AA@ 10005700     libucrt:lcidtoname_downlevel.obj
 0001:0000470c       ??_C@_1M@LGPJHNJH@?$AAz?$AAu?$AA?9?$AAZ?$AAA?$AA?$AA@ 1000570c     libucrt:lcidtoname_downlevel.obj
 0001:00004718       ??_C@_1M@HOKAOIO@?$AAa?$AAf?$AA?9?$AAZ?$AAA?$AA?$AA@ 10005718     libucrt:lcidtoname_downlevel.obj
 0001:00004724       ??_C@_1M@DPCLHLIE@?$AAk?$AAa?$AA?9?$AAG?$AAE?$AA?$AA@ 10005724     libucrt:lcidtoname_downlevel.obj
 0001:00004730       ??_C@_1M@BLKMHJBI@?$AAf?$AAo?$AA?9?$AAF?$AAO?$AA?$AA@ 10005730     libucrt:lcidtoname_downlevel.obj
 0001:0000473c       ??_C@_1M@LGGJAPPB@?$AAh?$AAi?$AA?9?$AAI?$AAN?$AA?$AA@ 1000573c     libucrt:lcidtoname_downlevel.obj
 0001:00004748       ??_C@_1M@FIKPIHFE@?$AAm?$AAt?$AA?9?$AAM?$AAT?$AA?$AA@ 10005748     libucrt:lcidtoname_downlevel.obj
 0001:00004754       ??_C@_1M@HEGGPBFA@?$AAs?$AAe?$AA?9?$AAN?$AAO?$AA?$AA@ 10005754     libucrt:lcidtoname_downlevel.obj
 0001:00004760       ??_C@_1M@EIBJEEPA@?$AAm?$AAs?$AA?9?$AAM?$AAY?$AA?$AA@ 10005760     libucrt:lcidtoname_downlevel.obj
 0001:0000476c       ??_C@_1M@FHLBGMPP@?$AAk?$AAk?$AA?9?$AAK?$AAZ?$AA?$AA@ 1000576c     libucrt:lcidtoname_downlevel.obj
 0001:00004778       ??_C@_1M@NGJJLCGI@?$AAk?$AAy?$AA?9?$AAK?$AAG?$AA?$AA@ 10005778     libucrt:lcidtoname_downlevel.obj
 0001:00004784       ??_C@_1M@GIENNBFC@?$AAs?$AAw?$AA?9?$AAK?$AAE?$AA?$AA@ 10005784     libucrt:lcidtoname_downlevel.obj
 0001:00004790       ??_C@_1BG@NDGMJIMJ@?$AAu?$AAz?$AA?9?$AAU?$AAZ?$AA?9?$AAL?$AAa?$AAt?$AAn?$AA?$AA@ 10005790     libucrt:lcidtoname_downlevel.obj
 0001:000047a8       ??_C@_1M@IDCCIHBC@?$AAt?$AAt?$AA?9?$AAR?$AAU?$AA?$AA@ 100057a8     libucrt:lcidtoname_downlevel.obj
 0001:000047b4       ??_C@_1M@LOICPMOJ@?$AAb?$AAn?$AA?9?$AAI?$AAN?$AA?$AA@ 100057b4     libucrt:lcidtoname_downlevel.obj
 0001:000047c0       ??_C@_1M@KPKKNEAH@?$AAp?$AAa?$AA?9?$AAI?$AAN?$AA?$AA@ 100057c0     libucrt:lcidtoname_downlevel.obj
 0001:000047cc       ??_C@_1M@PJGPPBOG@?$AAg?$AAu?$AA?9?$AAI?$AAN?$AA?$AA@ 100057cc     libucrt:lcidtoname_downlevel.obj
 0001:000047d8       ??_C@_1M@KMKMOPHI@?$AAt?$AAa?$AA?9?$AAI?$AAN?$AA?$AA@ 100057d8     libucrt:lcidtoname_downlevel.obj
 0001:000047e4       ??_C@_1M@KFEHEPAC@?$AAt?$AAe?$AA?9?$AAI?$AAN?$AA?$AA@ 100057e4     libucrt:lcidtoname_downlevel.obj
 0001:000047f0       ??_C@_1M@CDCLMGHI@?$AAk?$AAn?$AA?9?$AAI?$AAN?$AA?$AA@ 100057f0     libucrt:lcidtoname_downlevel.obj
 0001:000047fc       ??_C@_1M@MIODLDKF@?$AAm?$AAl?$AA?9?$AAI?$AAN?$AA?$AA@ 100057fc     libucrt:lcidtoname_downlevel.obj
 0001:00004808       ??_C@_1M@PBIEACPO@?$AAm?$AAr?$AA?9?$AAI?$AAN?$AA?$AA@ 10005808     libucrt:lcidtoname_downlevel.obj
 0001:00004814       ??_C@_1M@NIDEAGPH@?$AAs?$AAa?$AA?9?$AAI?$AAN?$AA?$AA@ 10005814     libucrt:lcidtoname_downlevel.obj
 0001:00004820       ??_C@_1M@FHIHCBIO@?$AAm?$AAn?$AA?9?$AAM?$AAN?$AA?$AA@ 10005820     libucrt:lcidtoname_downlevel.obj
 0001:0000482c       ??_C@_1M@JAIJPENP@?$AAc?$AAy?$AA?9?$AAG?$AAB?$AA?$AA@ 1000582c     libucrt:lcidtoname_downlevel.obj
 0001:00004838       ??_C@_1M@PHGFBEPN@?$AAg?$AAl?$AA?9?$AAE?$AAS?$AA?$AA@ 10005838     libucrt:lcidtoname_downlevel.obj
 0001:00004844       ??_C@_1O@KPIPDNCP@?$AAk?$AAo?$AAk?$AA?9?$AAI?$AAN?$AA?$AA@ 10005844     libucrt:lcidtoname_downlevel.obj
 0001:00004854       ??_C@_1O@KNHJLDJA@?$AAs?$AAy?$AAr?$AA?9?$AAS?$AAY?$AA?$AA@ 10005854     libucrt:lcidtoname_downlevel.obj
 0001:00004864       ??_C@_1O@MKEKBLAH@?$AAd?$AAi?$AAv?$AA?9?$AAM?$AAV?$AA?$AA@ 10005864     libucrt:lcidtoname_downlevel.obj
 0001:00004874       ??_C@_1O@OHDCKDDF@?$AAq?$AAu?$AAz?$AA?9?$AAB?$AAO?$AA?$AA@ 10005874     libucrt:lcidtoname_downlevel.obj
 0001:00004884       ??_C@_1M@LEPJNLFD@?$AAn?$AAs?$AA?9?$AAZ?$AAA?$AA?$AA@ 10005884     libucrt:lcidtoname_downlevel.obj
 0001:00004890       ??_C@_1M@OMLEIIJB@?$AAm?$AAi?$AA?9?$AAN?$AAZ?$AA?$AA@ 10005890     libucrt:lcidtoname_downlevel.obj
 0001:0000489c       ??_C@_1M@PMPEAILG@?$AAa?$AAr?$AA?9?$AAI?$AAQ?$AA?$AA@ 1000589c     libucrt:lcidtoname_downlevel.obj
 0001:000048a8       ??_C@_1M@CNKPNOEE@?$AAd?$AAe?$AA?9?$AAC?$AAH?$AA?$AA@ 100058a8     libucrt:lcidtoname_downlevel.obj
 0001:000048b4       ??_C@_1M@LKMGMLKO@?$AAe?$AAn?$AA?9?$AAG?$AAB?$AA?$AA@ 100058b4     libucrt:lcidtoname_downlevel.obj
 0001:000048c0       ??_C@_1M@PGKJFFGL@?$AAe?$AAs?$AA?9?$AAM?$AAX?$AA?$AA@ 100058c0     libucrt:lcidtoname_downlevel.obj
 0001:000048cc       ??_C@_1M@DNNANBDC@?$AAf?$AAr?$AA?9?$AAB?$AAE?$AA?$AA@ 100058cc     libucrt:lcidtoname_downlevel.obj
 0001:000048d8       ??_C@_1M@HLGMDFHM@?$AAi?$AAt?$AA?9?$AAC?$AAH?$AA?$AA@ 100058d8     libucrt:lcidtoname_downlevel.obj
 0001:000048e4       ??_C@_1M@CLLBGJH@?$AAn?$AAl?$AA?9?$AAB?$AAE?$AA?$AA@ 100058e4     libucrt:lcidtoname_downlevel.obj
 0001:000048f0       ??_C@_1M@BODBOGLF@?$AAn?$AAn?$AA?9?$AAN?$AAO?$AA?$AA@ 100058f0     libucrt:lcidtoname_downlevel.obj
 0001:000048fc       ??_C@_1M@HFFAHKAD@?$AAp?$AAt?$AA?9?$AAP?$AAT?$AA?$AA@ 100058fc     libucrt:lcidtoname_downlevel.obj
 0001:00004908       ??_C@_1BG@LNOAKHIE@?$AAs?$AAr?$AA?9?$AAS?$AAP?$AA?9?$AAL?$AAa?$AAt?$AAn?$AA?$AA@ 10005908     libucrt:lcidtoname_downlevel.obj
 0001:00004920       ??_C@_1M@HBMHBGAK@?$AAs?$AAv?$AA?9?$AAF?$AAI?$AA?$AA@ 10005920     libucrt:lcidtoname_downlevel.obj
 0001:0000492c       ??_C@_1BG@DGCJGJBE@?$AAa?$AAz?$AA?9?$AAA?$AAZ?$AA?9?$AAC?$AAy?$AAr?$AAl?$AA?$AA@ 1000592c     libucrt:lcidtoname_downlevel.obj
 0001:00004944       ??_C@_1M@KEJDAAHB@?$AAs?$AAe?$AA?9?$AAS?$AAE?$AA?$AA@ 10005944     libucrt:lcidtoname_downlevel.obj
 0001:00004950       ??_C@_1M@HEIBJJAD@?$AAm?$AAs?$AA?9?$AAB?$AAN?$AA?$AA@ 10005950     libucrt:lcidtoname_downlevel.obj
 0001:0000495c       ??_C@_1BG@PBGJMCEM@?$AAu?$AAz?$AA?9?$AAU?$AAZ?$AA?9?$AAC?$AAy?$AAr?$AAl?$AA?$AA@ 1000595c     libucrt:lcidtoname_downlevel.obj
 0001:00004974       ??_C@_1O@LAOBCMDF@?$AAq?$AAu?$AAz?$AA?9?$AAE?$AAC?$AA?$AA@ 10005974     libucrt:lcidtoname_downlevel.obj
 0001:00004984       ??_C@_1M@POEEMAIO@?$AAa?$AAr?$AA?9?$AAE?$AAG?$AA?$AA@ 10005984     libucrt:lcidtoname_downlevel.obj
 0001:00004990       ??_C@_1M@EFAKDEDL@?$AAz?$AAh?$AA?9?$AAH?$AAK?$AA?$AA@ 10005990     libucrt:lcidtoname_downlevel.obj
 0001:0000499c       ??_C@_1M@HKKIJHGI@?$AAd?$AAe?$AA?9?$AAA?$AAT?$AA?$AA@ 1000599c     libucrt:lcidtoname_downlevel.obj
 0001:000049a8       ??_C@_1M@KBFBEHJF@?$AAe?$AAn?$AA?9?$AAA?$AAU?$AA?$AA@ 100059a8     libucrt:lcidtoname_downlevel.obj
 0001:000049b4       ??_C@_1M@MNPLFAAH@?$AAe?$AAs?$AA?9?$AAE?$AAS?$AA?$AA@ 100059b4     libucrt:lcidtoname_downlevel.obj
 0001:000049c0       ??_C@_1M@HJOOJFMA@?$AAf?$AAr?$AA?9?$AAC?$AAA?$AA?$AA@ 100059c0     libucrt:lcidtoname_downlevel.obj
 0001:000049cc       ??_C@_1BG@JPOFPNAB@?$AAs?$AAr?$AA?9?$AAS?$AAP?$AA?9?$AAC?$AAy?$AAr?$AAl?$AA?$AA@ 100059cc     libucrt:lcidtoname_downlevel.obj
 0001:000049e4       ??_C@_1M@LNFOCMOB@?$AAs?$AAe?$AA?9?$AAF?$AAI?$AA?$AA@ 100059e4     libucrt:lcidtoname_downlevel.obj
 0001:000049f0       ??_C@_1O@MGJBOAMB@?$AAq?$AAu?$AAz?$AA?9?$AAP?$AAE?$AA?$AA@ 100059f0     libucrt:lcidtoname_downlevel.obj
 0001:00004a00       ??_C@_1M@GJINLBOK@?$AAa?$AAr?$AA?9?$AAL?$AAY?$AA?$AA@ 10005a00     libucrt:lcidtoname_downlevel.obj
 0001:00004a0c       ??_C@_1M@GGMNHJNL@?$AAz?$AAh?$AA?9?$AAS?$AAG?$AA?$AA@ 10005a0c     libucrt:lcidtoname_downlevel.obj
 0001:00004a18       ??_C@_1M@HOIKODND@?$AAd?$AAe?$AA?9?$AAL?$AAU?$AA?$AA@ 10005a18     libucrt:lcidtoname_downlevel.obj
 0001:00004a24       ??_C@_1M@DDOCCGFG@?$AAe?$AAn?$AA?9?$AAC?$AAA?$AA?$AA@ 10005a24     libucrt:lcidtoname_downlevel.obj
 0001:00004a30       ??_C@_1M@BNOEMJLF@?$AAe?$AAs?$AA?9?$AAG?$AAT?$AA?$AA@ 10005a30     libucrt:lcidtoname_downlevel.obj
 0001:00004a3c       ??_C@_1M@EOGNKEK@?$AAf?$AAr?$AA?9?$AAC?$AAH?$AA?$AA@ 10005a3c     libucrt:lcidtoname_downlevel.obj
 0001:00004a48       ??_C@_1M@FLIDJFHL@?$AAh?$AAr?$AA?9?$AAB?$AAA?$AA?$AA@ 10005a48     libucrt:lcidtoname_downlevel.obj
 0001:00004a54       ??_C@_1O@FMCELNAJ@?$AAs?$AAm?$AAj?$AA?9?$AAN?$AAO?$AA?$AA@ 10005a54     libucrt:lcidtoname_downlevel.obj
 0001:00004a64       ??_C@_1M@JHGLJMGJ@?$AAa?$AAr?$AA?9?$AAD?$AAZ?$AA?$AA@ 10005a64     libucrt:lcidtoname_downlevel.obj
 0001:00004a70       ??_C@_1M@JKKFDCNP@?$AAz?$AAh?$AA?9?$AAM?$AAO?$AA?$AA@ 10005a70     libucrt:lcidtoname_downlevel.obj
 0001:00004a7c       ??_C@_1M@GEEFALPE@?$AAd?$AAe?$AA?9?$AAL?$AAI?$AA?$AA@ 10005a7c     libucrt:lcidtoname_downlevel.obj
 0001:00004a88       ??_C@_1M@IGEOFBG@?$AAe?$AAn?$AA?9?$AAN?$AAZ?$AA?$AA@ 10005a88     libucrt:lcidtoname_downlevel.obj
 0001:00004a94       ??_C@_1M@KDBONEHP@?$AAe?$AAs?$AA?9?$AAC?$AAR?$AA?$AA@ 10005a94     libucrt:lcidtoname_downlevel.obj
 0001:00004aa0       ??_C@_1M@FHMDOHNN@?$AAf?$AAr?$AA?9?$AAL?$AAU?$AA?$AA@ 10005aa0     libucrt:lcidtoname_downlevel.obj
 0001:00004aac       ??_C@_1BG@NFKKMAFG@?$AAb?$AAs?$AA?9?$AAB?$AAA?$AA?9?$AAL?$AAa?$AAt?$AAn?$AA?$AA@ 10005aac     libucrt:lcidtoname_downlevel.obj
 0001:00004ac4       ??_C@_1O@IMNBEMCI@?$AAs?$AAm?$AAj?$AA?9?$AAS?$AAE?$AA?$AA@ 10005ac4     libucrt:lcidtoname_downlevel.obj
 0001:00004ad4       ??_C@_1M@DHHMBNDP@?$AAa?$AAr?$AA?9?$AAM?$AAA?$AA?$AA@ 10005ad4     libucrt:lcidtoname_downlevel.obj
 0001:00004ae0       ??_C@_1M@BNBLJCGH@?$AAe?$AAn?$AA?9?$AAI?$AAE?$AA?$AA@ 10005ae0     libucrt:lcidtoname_downlevel.obj
 0001:00004aec       ??_C@_1M@GEPAFMDL@?$AAe?$AAs?$AA?9?$AAP?$AAA?$AA?$AA@ 10005aec     libucrt:lcidtoname_downlevel.obj
 0001:00004af8       ??_C@_1M@OJONDMDL@?$AAf?$AAr?$AA?9?$AAM?$AAC?$AA?$AA@ 10005af8     libucrt:lcidtoname_downlevel.obj
 0001:00004b04       ??_C@_1BG@OBCNFJB@?$AAs?$AAr?$AA?9?$AAB?$AAA?$AA?9?$AAL?$AAa?$AAt?$AAn?$AA?$AA@ 10005b04     libucrt:lcidtoname_downlevel.obj
 0001:00004b1c       ??_C@_1O@KEMEEGPO@?$AAs?$AAm?$AAa?$AA?9?$AAN?$AAO?$AA?$AA@ 10005b1c     libucrt:lcidtoname_downlevel.obj
 0001:00004b2c       ??_C@_1M@ELMGFODK@?$AAa?$AAr?$AA?9?$AAT?$AAN?$AA?$AA@ 10005b2c     libucrt:lcidtoname_downlevel.obj
 0001:00004b38       ??_C@_1M@BHDLHFAF@?$AAe?$AAn?$AA?9?$AAZ?$AAA?$AA?$AA@ 10005b38     libucrt:lcidtoname_downlevel.obj
 0001:00004b44       ??_C@_1M@BMGIGLIF@?$AAe?$AAs?$AA?9?$AAD?$AAO?$AA?$AA@ 10005b44     libucrt:lcidtoname_downlevel.obj
 0001:00004b50       ??_C@_1BG@CMBHIPBE@?$AAs?$AAr?$AA?9?$AAB?$AAA?$AA?9?$AAC?$AAy?$AAr?$AAl?$AA?$AA@ 10005b50     libucrt:lcidtoname_downlevel.obj
 0001:00004b68       ??_C@_1O@HEDBLHNP@?$AAs?$AAm?$AAa?$AA?9?$AAS?$AAE?$AA?$AA@ 10005b68     libucrt:lcidtoname_downlevel.obj
 0001:00004b78       ??_C@_1M@DAGCADIM@?$AAa?$AAr?$AA?9?$AAO?$AAM?$AA?$AA@ 10005b78     libucrt:lcidtoname_downlevel.obj
 0001:00004b84       ??_C@_1M@FODLMICG@?$AAe?$AAn?$AA?9?$AAJ?$AAM?$AA?$AA@ 10005b84     libucrt:lcidtoname_downlevel.obj
 0001:00004b90       ??_C@_1M@DNMLCIHB@?$AAe?$AAs?$AA?9?$AAV?$AAE?$AA?$AA@ 10005b90     libucrt:lcidtoname_downlevel.obj
 0001:00004b9c       ??_C@_1O@EOKHMKJK@?$AAs?$AAm?$AAs?$AA?9?$AAF?$AAI?$AA?$AA@ 10005b9c     libucrt:lcidtoname_downlevel.obj
 0001:00004bac       ??_C@_1M@CAFJMKOF@?$AAa?$AAr?$AA?9?$AAY?$AAE?$AA?$AA@ 10005bac     libucrt:lcidtoname_downlevel.obj
 0001:00004bb8       ??_C@_1M@CBFHIJLI@?$AAe?$AAn?$AA?9?$AAC?$AAB?$AA?$AA@ 10005bb8     libucrt:lcidtoname_downlevel.obj
 0001:00004bc4       ??_C@_1M@BGNFLDN@?$AAe?$AAs?$AA?9?$AAC?$AAO?$AA?$AA@ 10005bc4     libucrt:lcidtoname_downlevel.obj
 0001:00004bd0       ??_C@_1O@JMPHMAMC@?$AAs?$AAm?$AAn?$AA?9?$AAF?$AAI?$AA?$AA@ 10005bd0     libucrt:lcidtoname_downlevel.obj
 0001:00004be0       ??_C@_1M@JLANABKE@?$AAa?$AAr?$AA?9?$AAS?$AAY?$AA?$AA@ 10005be0     libucrt:lcidtoname_downlevel.obj
 0001:00004bec       ??_C@_1M@HPKGCFGN@?$AAe?$AAn?$AA?9?$AAB?$AAZ?$AA?$AA@ 10005bec     libucrt:lcidtoname_downlevel.obj
 0001:00004bf8       ??_C@_1M@OLJCMLGM@?$AAe?$AAs?$AA?9?$AAP?$AAE?$AA?$AA@ 10005bf8     libucrt:lcidtoname_downlevel.obj
 0001:00004c04       ??_C@_1M@MKKGFKLE@?$AAa?$AAr?$AA?9?$AAJ?$AAO?$AA?$AA@ 10005c04     libucrt:lcidtoname_downlevel.obj
 0001:00004c10       ??_C@_1M@EKPGLDNI@?$AAe?$AAn?$AA?9?$AAT?$AAT?$AA?$AA@ 10005c10     libucrt:lcidtoname_downlevel.obj
 0001:00004c1c       ??_C@_1M@OONGHFHE@?$AAe?$AAs?$AA?9?$AAA?$AAR?$AA?$AA@ 10005c1c     libucrt:lcidtoname_downlevel.obj
 0001:00004c28       ??_C@_1M@OOJFGBHE@?$AAa?$AAr?$AA?9?$AAL?$AAB?$AA?$AA@ 10005c28     libucrt:lcidtoname_downlevel.obj
 0001:00004c34       ??_C@_1M@GCEJHNEG@?$AAe?$AAn?$AA?9?$AAZ?$AAW?$AA?$AA@ 10005c34     libucrt:lcidtoname_downlevel.obj
 0001:00004c40       ??_C@_1M@JNOCAHJI@?$AAe?$AAs?$AA?9?$AAE?$AAC?$AA?$AA@ 10005c40     libucrt:lcidtoname_downlevel.obj
 0001:00004c4c       ??_C@_1M@JEFHPGGB@?$AAa?$AAr?$AA?9?$AAK?$AAW?$AA?$AA@ 10005c4c     libucrt:lcidtoname_downlevel.obj
 0001:00004c58       ??_C@_1M@MLKIBJOJ@?$AAe?$AAn?$AA?9?$AAP?$AAH?$AA?$AA@ 10005c58     libucrt:lcidtoname_downlevel.obj
 0001:00004c64       ??_C@_1M@BDNIPEND@?$AAe?$AAs?$AA?9?$AAC?$AAL?$AA?$AA@ 10005c64     libucrt:lcidtoname_downlevel.obj
 0001:00004c70       ??_C@_1M@MPNMEKBD@?$AAa?$AAr?$AA?9?$AAA?$AAE?$AA?$AA@ 10005c70     libucrt:lcidtoname_downlevel.obj
 0001:00004c7c       ??_C@_1M@KBJALCPI@?$AAe?$AAs?$AA?9?$AAU?$AAY?$AA?$AA@ 10005c7c     libucrt:lcidtoname_downlevel.obj
 0001:00004c88       ??_C@_1M@LLCCOAGA@?$AAa?$AAr?$AA?9?$AAB?$AAH?$AA?$AA@ 10005c88     libucrt:lcidtoname_downlevel.obj
 0001:00004c94       ??_C@_1M@PBFNCDEL@?$AAe?$AAs?$AA?9?$AAP?$AAY?$AA?$AA@ 10005c94     libucrt:lcidtoname_downlevel.obj
 0001:00004ca0       ??_C@_1M@EDGINPNP@?$AAa?$AAr?$AA?9?$AAQ?$AAA?$AA?$AA@ 10005ca0     libucrt:lcidtoname_downlevel.obj
 0001:00004cac       ??_C@_1M@MKDBIIJI@?$AAe?$AAs?$AA?9?$AAB?$AAO?$AA?$AA@ 10005cac     libucrt:lcidtoname_downlevel.obj
 0001:00004cb8       ??_C@_1M@CPKKEBLD@?$AAe?$AAs?$AA?9?$AAS?$AAV?$AA?$AA@ 10005cb8     libucrt:lcidtoname_downlevel.obj
 0001:00004cc4       ??_C@_1M@NDBGMMJL@?$AAe?$AAs?$AA?9?$AAH?$AAN?$AA?$AA@ 10005cc4     libucrt:lcidtoname_downlevel.obj
 0001:00004cd0       ??_C@_1M@JIJIBHDP@?$AAe?$AAs?$AA?9?$AAN?$AAI?$AA?$AA@ 10005cd0     libucrt:lcidtoname_downlevel.obj
 0001:00004cdc       ??_C@_1M@CGFMKEEK@?$AAe?$AAs?$AA?9?$AAP?$AAR?$AA?$AA@ 10005cdc     libucrt:lcidtoname_downlevel.obj
 0001:00004ce8       ??_C@_1O@ICJHKIIK@?$AAz?$AAh?$AA?9?$AAC?$AAH?$AAT?$AA?$AA@ 10005ce8     libucrt:lcidtoname_downlevel.obj
 0001:00004cf8       ??_C@_15CLNEJCE@?$AAs?$AAr?$AA?$AA@ 10005cf8     libucrt:lcidtoname_downlevel.obj
 0001:00005420       ??_C@_1M@KAHEKEIG@?$AAa?$AAf?$AA?9?$AAz?$AAa?$AA?$AA@ 10006420     libucrt:lcidtoname_downlevel.obj
 0001:0000542c       ??_C@_1M@GIECOABL@?$AAa?$AAr?$AA?9?$AAa?$AAe?$AA?$AA@ 1000642c     libucrt:lcidtoname_downlevel.obj
 0001:00005438       ??_C@_1M@BMLMEKGI@?$AAa?$AAr?$AA?9?$AAb?$AAh?$AA?$AA@ 10006438     libucrt:lcidtoname_downlevel.obj
 0001:00005444       ??_C@_1M@DAPFDGGB@?$AAa?$AAr?$AA?9?$AAd?$AAz?$AA?$AA@ 10006444     libucrt:lcidtoname_downlevel.obj
 0001:00005450       ??_C@_1M@FJNKGKIG@?$AAa?$AAr?$AA?9?$AAe?$AAg?$AA?$AA@ 10006450     libucrt:lcidtoname_downlevel.obj
 0001:0000545c       ??_C@_1M@FLGKKCLO@?$AAa?$AAr?$AA?9?$AAi?$AAq?$AA?$AA@ 1000645c     libucrt:lcidtoname_downlevel.obj
 0001:00005468       ??_C@_1M@GNDIPALM@?$AAa?$AAr?$AA?9?$AAj?$AAo?$AA?$AA@ 10006468     libucrt:lcidtoname_downlevel.obj
 0001:00005474       ??_C@_1M@DDMJFMGJ@?$AAa?$AAr?$AA?9?$AAk?$AAw?$AA?$AA@ 10006474     libucrt:lcidtoname_downlevel.obj
 0001:00005480       ??_C@_1M@EJALMLHM@?$AAa?$AAr?$AA?9?$AAl?$AAb?$AA?$AA@ 10006480     libucrt:lcidtoname_downlevel.obj
 0001:0000548c       ??_C@_1M@MOBDBLOC@?$AAa?$AAr?$AA?9?$AAl?$AAy?$AA?$AA@ 1000648c     libucrt:lcidtoname_downlevel.obj
 0001:00005498       ??_C@_1M@JAOCLHDH@?$AAa?$AAr?$AA?9?$AAm?$AAa?$AA?$AA@ 10006498     libucrt:lcidtoname_downlevel.obj
 0001:000054a4       ??_C@_1M@JHPMKJIE@?$AAa?$AAr?$AA?9?$AAo?$AAm?$AA?$AA@ 100064a4     libucrt:lcidtoname_downlevel.obj
 0001:000054b0       ??_C@_1M@OEPGHFNH@?$AAa?$AAr?$AA?9?$AAq?$AAa?$AA?$AA@ 100064b0     libucrt:lcidtoname_downlevel.obj
 0001:000054bc       ??_C@_1M@KJDONENM@?$AAa?$AAr?$AA?9?$AAs?$AAa?$AA?$AA@ 100064bc     libucrt:lcidtoname_downlevel.obj
 0001:000054c8       ??_C@_1M@DMJDKLKM@?$AAa?$AAr?$AA?9?$AAs?$AAy?$AA?$AA@ 100064c8     libucrt:lcidtoname_downlevel.obj
 0001:000054d4       ??_C@_1M@OMFIPEDC@?$AAa?$AAr?$AA?9?$AAt?$AAn?$AA?$AA@ 100064d4     libucrt:lcidtoname_downlevel.obj
 0001:000054e0       ??_C@_1M@IHMHGAON@?$AAa?$AAr?$AA?9?$AAy?$AAe?$AA?$AA@ 100064e0     libucrt:lcidtoname_downlevel.obj
 0001:000054ec       ??_C@_1BG@KDCPGJGB@?$AAa?$AAz?$AA?9?$AAa?$AAz?$AA?9?$AAc?$AAy?$AAr?$AAl?$AA?$AA@ 100064ec     libucrt:lcidtoname_downlevel.obj
 0001:00005504       ??_C@_1BG@IBCKDDOE@?$AAa?$AAz?$AA?9?$AAa?$AAz?$AA?9?$AAl?$AAa?$AAt?$AAn?$AA?$AA@ 10006504     libucrt:lcidtoname_downlevel.obj
 0001:0000551c       ??_C@_1M@EGPFDCPD@?$AAb?$AAe?$AA?9?$AAb?$AAy?$AA?$AA@ 1000651c     libucrt:lcidtoname_downlevel.obj
 0001:00005528       ??_C@_1M@PCMGMCGC@?$AAb?$AAg?$AA?9?$AAb?$AAg?$AA?$AA@ 10006528     libucrt:lcidtoname_downlevel.obj
 0001:00005534       ??_C@_1M@BJBMFGOB@?$AAb?$AAn?$AA?9?$AAi?$AAn?$AA?$AA@ 10006534     libucrt:lcidtoname_downlevel.obj
 0001:00005540       ??_C@_1BG@EAKMMACD@?$AAb?$AAs?$AA?9?$AAb?$AAa?$AA?9?$AAl?$AAa?$AAt?$AAn?$AA?$AA@ 10006540     libucrt:lcidtoname_downlevel.obj
 0001:00005558       ??_C@_1M@KGADAODK@?$AAc?$AAa?$AA?9?$AAe?$AAs?$AA?$AA@ 10006558     libucrt:lcidtoname_downlevel.obj
 0001:00005564       ??_C@_1M@COAJPDHI@?$AAc?$AAs?$AA?9?$AAc?$AAz?$AA?$AA@ 10006564     libucrt:lcidtoname_downlevel.obj
 0001:00005570       ??_C@_1M@DHBHFONH@?$AAc?$AAy?$AA?9?$AAg?$AAb?$AA?$AA@ 10006570     libucrt:lcidtoname_downlevel.obj
 0001:0000557c       ??_C@_1M@IMGKELGA@?$AAd?$AAa?$AA?9?$AAd?$AAk?$AA?$AA@ 1000657c     libucrt:lcidtoname_downlevel.obj
 0001:00005588       ??_C@_1M@NNDGDNGA@?$AAd?$AAe?$AA?9?$AAa?$AAt?$AA?$AA@ 10006588     libucrt:lcidtoname_downlevel.obj
 0001:00005594       ??_C@_1M@IKDBHEEM@?$AAd?$AAe?$AA?9?$AAc?$AAh?$AA?$AA@ 10006594     libucrt:lcidtoname_downlevel.obj
 0001:000055a0       ??_C@_1M@GFFOJMCJ@?$AAd?$AAe?$AA?9?$AAd?$AAe?$AA?$AA@ 100065a0     libucrt:lcidtoname_downlevel.obj
 0001:000055ac       ??_C@_1M@MDNLKBPM@?$AAd?$AAe?$AA?9?$AAl?$AAi?$AA?$AA@ 100065ac     libucrt:lcidtoname_downlevel.obj
 0001:000055b8       ??_C@_1M@NJBEEJNL@?$AAd?$AAe?$AA?9?$AAl?$AAu?$AA?$AA@ 100065b8     libucrt:lcidtoname_downlevel.obj
 0001:000055c4       ??_C@_1O@GNNELBAP@?$AAd?$AAi?$AAv?$AA?9?$AAm?$AAv?$AA?$AA@ 100065c4     libucrt:lcidtoname_downlevel.obj
 0001:000055d4       ??_C@_1M@EJLEOGAE@?$AAe?$AAl?$AA?9?$AAg?$AAr?$AA?$AA@ 100065d4     libucrt:lcidtoname_downlevel.obj
 0001:000055e0       ??_C@_1M@GMPONJN@?$AAe?$AAn?$AA?9?$AAa?$AAu?$AA?$AA@ 100065e0     libucrt:lcidtoname_downlevel.obj
 0001:000055ec       ??_C@_1M@NIDIIPGF@?$AAe?$AAn?$AA?9?$AAb?$AAz?$AA?$AA@ 100065ec     libucrt:lcidtoname_downlevel.obj
 0001:000055f8       ??_C@_1M@JEHMIMFO@?$AAe?$AAn?$AA?9?$AAc?$AAa?$AA?$AA@ 100065f8     libucrt:lcidtoname_downlevel.obj
 0001:00005604       ??_C@_1M@IGMJCDLA@?$AAe?$AAn?$AA?9?$AAc?$AAb?$AA?$AA@ 10006604     libucrt:lcidtoname_downlevel.obj
 0001:00005610       ??_C@_1M@BNFIGBKG@?$AAe?$AAn?$AA?9?$AAg?$AAb?$AA?$AA@ 10006610     libucrt:lcidtoname_downlevel.obj
 0001:0000561c       ??_C@_1M@LKIFDIGP@?$AAe?$AAn?$AA?9?$AAi?$AAe?$AA?$AA@ 1000661c     libucrt:lcidtoname_downlevel.obj
 0001:00005628       ??_C@_1M@PJKFGCCO@?$AAe?$AAn?$AA?9?$AAj?$AAm?$AA?$AA@ 10006628     libucrt:lcidtoname_downlevel.obj
 0001:00005634       ??_C@_1M@KPPKEPBO@?$AAe?$AAn?$AA?9?$AAn?$AAz?$AA?$AA@ 10006634     libucrt:lcidtoname_downlevel.obj
 0001:00005640       ??_C@_1M@GMDGLDOB@?$AAe?$AAn?$AA?9?$AAp?$AAh?$AA?$AA@ 10006640     libucrt:lcidtoname_downlevel.obj
 0001:0000564c       ??_C@_1M@ONGIBJNA@?$AAe?$AAn?$AA?9?$AAt?$AAt?$AA?$AA@ 1000664c     libucrt:lcidtoname_downlevel.obj
 0001:00005658       ??_C@_1M@LLODPCMM@?$AAe?$AAn?$AA?9?$AAu?$AAs?$AA?$AA@ 10006658     libucrt:lcidtoname_downlevel.obj
 0001:00005664       ??_C@_1M@LAKFNPAN@?$AAe?$AAn?$AA?9?$AAz?$AAa?$AA?$AA@ 10006664     libucrt:lcidtoname_downlevel.obj
 0001:00005670       ??_C@_1M@MFNHNHEO@?$AAe?$AAn?$AA?9?$AAz?$AAw?$AA?$AA@ 10006670     libucrt:lcidtoname_downlevel.obj
 0001:0000567c       ??_C@_1M@EJEINPHM@?$AAe?$AAs?$AA?9?$AAa?$AAr?$AA?$AA@ 1000667c     libucrt:lcidtoname_downlevel.obj
 0001:00005688       ??_C@_1M@GNKPCCJA@?$AAe?$AAs?$AA?9?$AAb?$AAo?$AA?$AA@ 10006688     libucrt:lcidtoname_downlevel.obj
 0001:00005694       ??_C@_1M@LEEGFONL@?$AAe?$AAs?$AA?9?$AAc?$AAl?$AA?$AA@ 10006694     libucrt:lcidtoname_downlevel.obj
 0001:000056a0       ??_C@_1M@KGPDPBDF@?$AAe?$AAs?$AA?9?$AAc?$AAo?$AA?$AA@ 100066a0     libucrt:lcidtoname_downlevel.obj
 0001:000056ac       ??_C@_1M@EIAHOHH@?$AAe?$AAs?$AA?9?$AAc?$AAr?$AA?$AA@ 100066ac     libucrt:lcidtoname_downlevel.obj
 0001:000056b8       ??_C@_1M@LLPGMBIN@?$AAe?$AAs?$AA?9?$AAd?$AAo?$AA?$AA@ 100066b8     libucrt:lcidtoname_downlevel.obj
 0001:000056c4       ??_C@_1M@DKHMKNJA@?$AAe?$AAs?$AA?9?$AAe?$AAc?$AA?$AA@ 100066c4     libucrt:lcidtoname_downlevel.obj
 0001:000056d0       ??_C@_1M@GKGFPKAP@?$AAe?$AAs?$AA?9?$AAe?$AAs?$AA?$AA@ 100066d0     libucrt:lcidtoname_downlevel.obj
 0001:000056dc       ??_C@_1M@LKHKGDLN@?$AAe?$AAs?$AA?9?$AAg?$AAt?$AA?$AA@ 100066dc     libucrt:lcidtoname_downlevel.obj
 0001:000056e8       ??_C@_1M@HEIIGGJD@?$AAe?$AAs?$AA?9?$AAh?$AAn?$AA?$AA@ 100066e8     libucrt:lcidtoname_downlevel.obj
 0001:000056f4       ??_C@_1M@FBDHPPGD@?$AAe?$AAs?$AA?9?$AAm?$AAx?$AA?$AA@ 100066f4     libucrt:lcidtoname_downlevel.obj
 0001:00005700       ??_C@_1M@DPAGLNDH@?$AAe?$AAs?$AA?9?$AAn?$AAi?$AA?$AA@ 10006700     libucrt:lcidtoname_downlevel.obj
 0001:0000570c       ??_C@_1M@MDGOPGDD@?$AAe?$AAs?$AA?9?$AAp?$AAa?$AA?$AA@ 1000670c     libucrt:lcidtoname_downlevel.obj
 0001:00005718       ??_C@_1M@EMAMGBGE@?$AAe?$AAs?$AA?9?$AAp?$AAe?$AA?$AA@ 10006718     libucrt:lcidtoname_downlevel.obj
 0001:00005724       ??_C@_1M@IBMCAOEC@?$AAe?$AAs?$AA?9?$AAp?$AAr?$AA?$AA@ 10006724     libucrt:lcidtoname_downlevel.obj
 0001:00005730       ??_C@_1M@FGMDIJED@?$AAe?$AAs?$AA?9?$AAp?$AAy?$AA?$AA@ 10006730     libucrt:lcidtoname_downlevel.obj
 0001:0000573c       ??_C@_1M@IIDEOLLL@?$AAe?$AAs?$AA?9?$AAs?$AAv?$AA?$AA@ 1000673c     libucrt:lcidtoname_downlevel.obj
 0001:00005748       ??_C@_1M@GAOBIPA@?$AAe?$AAs?$AA?9?$AAu?$AAy?$AA?$AA@ 10006748     libucrt:lcidtoname_downlevel.obj
 0001:00005754       ??_C@_1M@JKFFICHJ@?$AAe?$AAs?$AA?9?$AAv?$AAe?$AA?$AA@ 10006754     libucrt:lcidtoname_downlevel.obj
 0001:00005760       ??_C@_1M@PNMLOJDF@?$AAe?$AAt?$AA?9?$AAe?$AAe?$AA?$AA@ 10006760     libucrt:lcidtoname_downlevel.obj
 0001:0000576c       ??_C@_1M@GHHLIKEI@?$AAe?$AAu?$AA?9?$AAe?$AAs?$AA?$AA@ 1000676c     libucrt:lcidtoname_downlevel.obj
 0001:00005778       ??_C@_1M@PBNONODE@?$AAf?$AAa?$AA?9?$AAi?$AAr?$AA?$AA@ 10006778     libucrt:lcidtoname_downlevel.obj
 0001:00005784       ??_C@_1M@JEEHPMIL@?$AAf?$AAi?$AA?9?$AAf?$AAi?$AA?$AA@ 10006784     libucrt:lcidtoname_downlevel.obj
 0001:00005790       ??_C@_1M@LMDCNDBA@?$AAf?$AAo?$AA?9?$AAf?$AAo?$AA?$AA@ 10006790     libucrt:lcidtoname_downlevel.obj
 0001:0000579c       ??_C@_1M@JKEOHLDK@?$AAf?$AAr?$AA?9?$AAb?$AAe?$AA?$AA@ 1000679c     libucrt:lcidtoname_downlevel.obj
 0001:000057a8       ??_C@_1M@NOHADPMI@?$AAf?$AAr?$AA?9?$AAc?$AAa?$AA?$AA@ 100067a8     libucrt:lcidtoname_downlevel.obj
 0001:000057b4       ??_C@_1M@KDHIHAEC@?$AAf?$AAr?$AA?9?$AAc?$AAh?$AA?$AA@ 100067b4     libucrt:lcidtoname_downlevel.obj
 0001:000057c0       ??_C@_1M@MMBBFGAK@?$AAf?$AAr?$AA?9?$AAf?$AAr?$AA?$AA@ 100067c0     libucrt:lcidtoname_downlevel.obj
 0001:000057cc       ??_C@_1M@PAFNENNF@?$AAf?$AAr?$AA?9?$AAl?$AAu?$AA?$AA@ 100067cc     libucrt:lcidtoname_downlevel.obj
 0001:000057d8       ??_C@_1M@EOHDJGDD@?$AAf?$AAr?$AA?9?$AAm?$AAc?$AA?$AA@ 100067d8     libucrt:lcidtoname_downlevel.obj
 0001:000057e4       ??_C@_1M@FAPLLOPF@?$AAg?$AAl?$AA?9?$AAe?$AAs?$AA?$AA@ 100067e4     libucrt:lcidtoname_downlevel.obj
 0001:000057f0       ??_C@_1M@FOPBFLOO@?$AAg?$AAu?$AA?9?$AAi?$AAn?$AA?$AA@ 100067f0     libucrt:lcidtoname_downlevel.obj
 0001:000057fc       ??_C@_1M@KBMCINPM@?$AAh?$AAe?$AA?9?$AAi?$AAl?$AA?$AA@ 100067fc     libucrt:lcidtoname_downlevel.obj
 0001:00005808       ??_C@_1M@BBPHKFPJ@?$AAh?$AAi?$AA?9?$AAi?$AAn?$AA?$AA@ 10006808     libucrt:lcidtoname_downlevel.obj
 0001:00005814       ??_C@_1M@PMBNDPHD@?$AAh?$AAr?$AA?9?$AAb?$AAa?$AA?$AA@ 10006814     libucrt:lcidtoname_downlevel.obj
 0001:00005820       ??_C@_1M@BPCKOEGE@?$AAh?$AAr?$AA?9?$AAh?$AAr?$AA?$AA@ 10006820     libucrt:lcidtoname_downlevel.obj
 0001:0000582c       ??_C@_1M@GACBMHKE@?$AAh?$AAu?$AA?9?$AAh?$AAu?$AA?$AA@ 1000682c     libucrt:lcidtoname_downlevel.obj
 0001:00005838       ??_C@_1M@MILPAJJC@?$AAh?$AAy?$AA?9?$AAa?$AAm?$AA?$AA@ 10006838     libucrt:lcidtoname_downlevel.obj
 0001:00005844       ??_C@_1M@BABBICEC@?$AAi?$AAd?$AA?9?$AAi?$AAd?$AA?$AA@ 10006844     libucrt:lcidtoname_downlevel.obj
 0001:00005850       ??_C@_1M@BIKNHHPF@?$AAi?$AAs?$AA?9?$AAi?$AAs?$AA?$AA@ 10006850     libucrt:lcidtoname_downlevel.obj
 0001:0000585c       ??_C@_1M@NMPCJPHE@?$AAi?$AAt?$AA?9?$AAc?$AAh?$AA?$AA@ 1000685c     libucrt:lcidtoname_downlevel.obj
 0001:00005868       ??_C@_1M@GHKGFEDF@?$AAi?$AAt?$AA?9?$AAi?$AAt?$AA?$AA@ 10006868     libucrt:lcidtoname_downlevel.obj
 0001:00005874       ??_C@_1M@NIEJCJJA@?$AAj?$AAa?$AA?9?$AAj?$AAp?$AA?$AA@ 10006874     libucrt:lcidtoname_downlevel.obj
 0001:00005880       ??_C@_1M@JILFNBIM@?$AAk?$AAa?$AA?9?$AAg?$AAe?$AA?$AA@ 10006880     libucrt:lcidtoname_downlevel.obj
 0001:0000588c       ??_C@_1M@PACPMGPH@?$AAk?$AAk?$AA?9?$AAk?$AAz?$AA?$AA@ 1000688c     libucrt:lcidtoname_downlevel.obj
 0001:00005898       ??_C@_1M@IELFGMHA@?$AAk?$AAn?$AA?9?$AAi?$AAn?$AA?$AA@ 10006898     libucrt:lcidtoname_downlevel.obj
 0001:000058a4       ??_C@_1O@IBBJHCH@?$AAk?$AAo?$AAk?$AA?9?$AAi?$AAn?$AA?$AA@ 100068a4     libucrt:lcidtoname_downlevel.obj
 0001:000058b4       ??_C@_1M@DMHAEOGC@?$AAk?$AAo?$AA?9?$AAk?$AAr?$AA?$AA@ 100068b4     libucrt:lcidtoname_downlevel.obj
 0001:000058c0       ??_C@_1M@HBAHBIGA@?$AAk?$AAy?$AA?9?$AAk?$AAg?$AA?$AA@ 100068c0     libucrt:lcidtoname_downlevel.obj
 0001:000058cc       ??_C@_1M@KPMILCJG@?$AAl?$AAt?$AA?9?$AAl?$AAt?$AA?$AA@ 100068cc     libucrt:lcidtoname_downlevel.obj
 0001:000058d8       ??_C@_1M@BDEKKCA@?$AAl?$AAv?$AA?9?$AAl?$AAv?$AA?$AA@ 100068d8     libucrt:lcidtoname_downlevel.obj
 0001:000058e4       ??_C@_1M@ELCKCCJJ@?$AAm?$AAi?$AA?9?$AAn?$AAz?$AA?$AA@ 100068e4     libucrt:lcidtoname_downlevel.obj
 0001:000058f0       ??_C@_1M@CBOOLAPA@?$AAm?$AAk?$AA?9?$AAm?$AAk?$AA?$AA@ 100068f0     libucrt:lcidtoname_downlevel.obj
 0001:000058fc       ??_C@_1M@GPHNBJKN@?$AAm?$AAl?$AA?9?$AAi?$AAn?$AA?$AA@ 100068fc     libucrt:lcidtoname_downlevel.obj
 0001:00005908       ??_C@_1M@PABJILIG@?$AAm?$AAn?$AA?9?$AAm?$AAn?$AA?$AA@ 10006908     libucrt:lcidtoname_downlevel.obj
 0001:00005914       ??_C@_1M@FGBKKIPG@?$AAm?$AAr?$AA?9?$AAi?$AAn?$AA?$AA@ 10006914     libucrt:lcidtoname_downlevel.obj
 0001:00005920       ??_C@_1M@NDBPDDAL@?$AAm?$AAs?$AA?9?$AAb?$AAn?$AA?$AA@ 10006920     libucrt:lcidtoname_downlevel.obj
 0001:0000592c       ??_C@_1M@OPIHOOPI@?$AAm?$AAs?$AA?9?$AAm?$AAy?$AA?$AA@ 1000692c     libucrt:lcidtoname_downlevel.obj
 0001:00005938       ??_C@_1M@PPDBCNFM@?$AAm?$AAt?$AA?9?$AAm?$AAt?$AA?$AA@ 10006938     libucrt:lcidtoname_downlevel.obj
 0001:00005944       ??_C@_1M@KDJDKMDD@?$AAn?$AAb?$AA?9?$AAn?$AAo?$AA?$AA@ 10006944     libucrt:lcidtoname_downlevel.obj
 0001:00005950       ??_C@_1M@KFCFLMJP@?$AAn?$AAl?$AA?9?$AAb?$AAe?$AA?$AA@ 10006950     libucrt:lcidtoname_downlevel.obj
 0001:0000595c       ??_C@_1M@KPOPDDGO@?$AAn?$AAl?$AA?9?$AAn?$AAl?$AA?$AA@ 1000695c     libucrt:lcidtoname_downlevel.obj
 0001:00005968       ??_C@_1M@LJKPEMLN@?$AAn?$AAn?$AA?9?$AAn?$AAo?$AA?$AA@ 10006968     libucrt:lcidtoname_downlevel.obj
 0001:00005974       ??_C@_1M@BDGHHBFL@?$AAn?$AAs?$AA?9?$AAz?$AAa?$AA?$AA@ 10006974     libucrt:lcidtoname_downlevel.obj
 0001:00005980       ??_C@_1M@IDEHOAP@?$AAp?$AAa?$AA?9?$AAi?$AAn?$AA?$AA@ 10006980     libucrt:lcidtoname_downlevel.obj
 0001:0000598c       ??_C@_1M@HDBKGOGH@?$AAp?$AAl?$AA?9?$AAp?$AAl?$AA?$AA@ 1000698c     libucrt:lcidtoname_downlevel.obj
 0001:00005998       ??_C@_1M@LJLLCMEH@?$AAp?$AAt?$AA?9?$AAb?$AAr?$AA?$AA@ 10006998     libucrt:lcidtoname_downlevel.obj
 0001:000059a4       ??_C@_1M@NCMONAAL@?$AAp?$AAt?$AA?9?$AAp?$AAt?$AA?$AA@ 100069a4     libucrt:lcidtoname_downlevel.obj
 0001:000059b0       ??_C@_1O@EAKMAJDN@?$AAq?$AAu?$AAz?$AA?9?$AAb?$AAo?$AA?$AA@ 100069b0     libucrt:lcidtoname_downlevel.obj
 0001:000059c0       ??_C@_1O@BHHPIGDN@?$AAq?$AAu?$AAz?$AA?9?$AAe?$AAc?$AA?$AA@ 100069c0     libucrt:lcidtoname_downlevel.obj
 0001:000059d0       ??_C@_1O@GBAPEKMJ@?$AAq?$AAu?$AAz?$AA?9?$AAp?$AAe?$AA?$AA@ 100069d0     libucrt:lcidtoname_downlevel.obj
 0001:000059e0       ??_C@_1M@CLGLEFBO@?$AAr?$AAo?$AA?9?$AAr?$AAo?$AA?$AA@ 100069e0     libucrt:lcidtoname_downlevel.obj
 0001:000059ec       ??_C@_1M@CEEDODME@?$AAr?$AAu?$AA?9?$AAr?$AAu?$AA?$AA@ 100069ec     libucrt:lcidtoname_downlevel.obj
 0001:000059f8       ??_C@_1M@HPKKKMPP@?$AAs?$AAa?$AA?9?$AAi?$AAn?$AA?$AA@ 100069f8     libucrt:lcidtoname_downlevel.obj
 0001:00005a04       ??_C@_1M@BKMAIGOJ@?$AAs?$AAe?$AA?9?$AAf?$AAi?$AA?$AA@ 10006a04     libucrt:lcidtoname_downlevel.obj
 0001:00005a10       ??_C@_1M@NDPIFLFI@?$AAs?$AAe?$AA?9?$AAn?$AAo?$AA?$AA@ 10006a10     libucrt:lcidtoname_downlevel.obj
 0001:00005a1c       ??_C@_1M@DANKKHJ@?$AAs?$AAe?$AA?9?$AAs?$AAe?$AA?$AA@ 10006a1c     libucrt:lcidtoname_downlevel.obj
 0001:00005a28       ??_C@_1M@PNBLONPJ@?$AAs?$AAk?$AA?9?$AAs?$AAk?$AA?$AA@ 10006a28     libucrt:lcidtoname_downlevel.obj
 0001:00005a34       ??_C@_1M@LFMODOAL@?$AAs?$AAl?$AA?9?$AAs?$AAi?$AA?$AA@ 10006a34     libucrt:lcidtoname_downlevel.obj
 0001:00005a40       ??_C@_1O@DFKOMPG@?$AAs?$AAm?$AAa?$AA?9?$AAn?$AAo?$AA?$AA@ 10006a40     libucrt:lcidtoname_downlevel.obj
 0001:00005a50       ??_C@_1O@NDKPBNNH@?$AAs?$AAm?$AAa?$AA?9?$AAs?$AAe?$AA?$AA@ 10006a50     libucrt:lcidtoname_downlevel.obj
 0001:00005a60       ??_C@_1O@PLLKBHAB@?$AAs?$AAm?$AAj?$AA?9?$AAn?$AAo?$AA?$AA@ 10006a60     libucrt:lcidtoname_downlevel.obj
 0001:00005a70       ??_C@_1O@CLEPOGCA@?$AAs?$AAm?$AAj?$AA?9?$AAs?$AAe?$AA?$AA@ 10006a70     libucrt:lcidtoname_downlevel.obj
 0001:00005a80       ??_C@_1O@DLGJGKMK@?$AAs?$AAm?$AAn?$AA?9?$AAf?$AAi?$AA?$AA@ 10006a80     libucrt:lcidtoname_downlevel.obj
 0001:00005a90       ??_C@_1O@OJDJGAJC@?$AAs?$AAm?$AAs?$AA?9?$AAf?$AAi?$AA?$AA@ 10006a90     libucrt:lcidtoname_downlevel.obj
 0001:00005aa0       ??_C@_1M@BOFOGHPB@?$AAs?$AAq?$AA?9?$AAa?$AAl?$AA?$AA@ 10006aa0     libucrt:lcidtoname_downlevel.obj
 0001:00005aac       ??_C@_1BG@LJBBIPGB@?$AAs?$AAr?$AA?9?$AAb?$AAa?$AA?9?$AAc?$AAy?$AAr?$AAl?$AA?$AA@ 10006aac     libucrt:lcidtoname_downlevel.obj
 0001:00005ac4       ??_C@_1BG@JLBENFOE@?$AAs?$AAr?$AA?9?$AAb?$AAa?$AA?9?$AAl?$AAa?$AAt?$AAn?$AA?$AA@ 10006ac4     libucrt:lcidtoname_downlevel.obj
 0001:00005adc       ??_C@_1BG@KODPNHE@?$AAs?$AAr?$AA?9?$AAs?$AAp?$AA?9?$AAc?$AAy?$AAr?$AAl?$AA?$AA@ 10006adc     libucrt:lcidtoname_downlevel.obj
 0001:00005af4       ??_C@_1BG@CIOGKHPB@?$AAs?$AAr?$AA?9?$AAs?$AAp?$AA?9?$AAl?$AAa?$AAt?$AAn?$AA?$AA@ 10006af4     libucrt:lcidtoname_downlevel.obj
 0001:00005b0c       ??_C@_1M@NGFJLMAC@?$AAs?$AAv?$AA?9?$AAf?$AAi?$AA?$AA@ 10006b0c     libucrt:lcidtoname_downlevel.obj
 0001:00005b18       ??_C@_1M@MPJEJAJC@?$AAs?$AAv?$AA?9?$AAs?$AAe?$AA?$AA@ 10006b18     libucrt:lcidtoname_downlevel.obj
 0001:00005b24       ??_C@_1M@MPNDHLFK@?$AAs?$AAw?$AA?9?$AAk?$AAe?$AA?$AA@ 10006b24     libucrt:lcidtoname_downlevel.obj
 0001:00005b30       ??_C@_1O@KOHBJJI@?$AAs?$AAy?$AAr?$AA?9?$AAs?$AAy?$AA?$AA@ 10006b30     libucrt:lcidtoname_downlevel.obj
 0001:00005b40       ??_C@_1M@LDCEFHA@?$AAt?$AAa?$AA?9?$AAi?$AAn?$AA?$AA@ 10006b40     libucrt:lcidtoname_downlevel.obj
 0001:00005b4c       ??_C@_1M@CNJOFAK@?$AAt?$AAe?$AA?9?$AAi?$AAn?$AA?$AA@ 10006b4c     libucrt:lcidtoname_downlevel.obj
 0001:00005b58       ??_C@_1M@GNAECACD@?$AAt?$AAh?$AA?9?$AAt?$AAh?$AA?$AA@ 10006b58     libucrt:lcidtoname_downlevel.obj
 0001:00005b64       ??_C@_1M@CHBIHOJO@?$AAt?$AAn?$AA?9?$AAz?$AAa?$AA?$AA@ 10006b64     libucrt:lcidtoname_downlevel.obj
 0001:00005b70       ??_C@_1M@GCCMIGPJ@?$AAt?$AAr?$AA?9?$AAt?$AAr?$AA?$AA@ 10006b70     libucrt:lcidtoname_downlevel.obj
 0001:00005b7c       ??_C@_1M@CELMCNBK@?$AAt?$AAt?$AA?9?$AAr?$AAu?$AA?$AA@ 10006b7c     libucrt:lcidtoname_downlevel.obj
 0001:00005b88       ??_C@_1M@KLMCELGA@?$AAu?$AAk?$AA?9?$AAu?$AAa?$AA?$AA@ 10006b88     libucrt:lcidtoname_downlevel.obj
 0001:00005b94       ??_C@_1M@EPAJJAJF@?$AAu?$AAr?$AA?9?$AAp?$AAk?$AA?$AA@ 10006b94     libucrt:lcidtoname_downlevel.obj
 0001:00005ba0       ??_C@_1BG@GEGPMCDJ@?$AAu?$AAz?$AA?9?$AAu?$AAz?$AA?9?$AAc?$AAy?$AAr?$AAl?$AA?$AA@ 10006ba0     libucrt:lcidtoname_downlevel.obj
 0001:00005bb8       ??_C@_1BG@EGGKJILM@?$AAu?$AAz?$AA?9?$AAu?$AAz?$AA?9?$AAl?$AAa?$AAt?$AAn?$AA?$AA@ 10006bb8     libucrt:lcidtoname_downlevel.obj
 0001:00005bd0       ??_C@_1M@GFOCLFF@?$AAv?$AAi?$AA?9?$AAv?$AAn?$AA?$AA@ 10006bd0     libucrt:lcidtoname_downlevel.obj
 0001:00005bdc       ??_C@_1M@CPAMEDFI@?$AAx?$AAh?$AA?9?$AAz?$AAa?$AA?$AA@ 10006bdc     libucrt:lcidtoname_downlevel.obj
 0001:00005be8       ??_C@_1O@EBKIFIGN@?$AAz?$AAh?$AA?9?$AAc?$AAh?$AAs?$AA?$AA@ 10006be8     libucrt:lcidtoname_downlevel.obj
 0001:00005bf8       ??_C@_1O@NMHPGANE@?$AAz?$AAh?$AA?9?$AAc?$AAh?$AAt?$AA?$AA@ 10006bf8     libucrt:lcidtoname_downlevel.obj
 0001:00005c08       ??_C@_1M@LPINJOMC@?$AAz?$AAh?$AA?9?$AAc?$AAn?$AA?$AA@ 10006c08     libucrt:lcidtoname_downlevel.obj
 0001:00005c14       ??_C@_1M@OCJEJODD@?$AAz?$AAh?$AA?9?$AAh?$AAk?$AA?$AA@ 10006c14     libucrt:lcidtoname_downlevel.obj
 0001:00005c20       ??_C@_1M@DNDLJINH@?$AAz?$AAh?$AA?9?$AAm?$AAo?$AA?$AA@ 10006c20     libucrt:lcidtoname_downlevel.obj
 0001:00005c2c       ??_C@_1M@MBFDNDND@?$AAz?$AAh?$AA?9?$AAs?$AAg?$AA?$AA@ 10006c2c     libucrt:lcidtoname_downlevel.obj
 0001:00005c38       ??_C@_1M@IMEPLEPE@?$AAz?$AAh?$AA?9?$AAt?$AAw?$AA?$AA@ 10006c38     libucrt:lcidtoname_downlevel.obj
 0001:00005c44       ??_C@_1M@BBGHNHJP@?$AAz?$AAu?$AA?9?$AAz?$AAa?$AA?$AA@ 10006c44     libucrt:lcidtoname_downlevel.obj
 0001:00005c50       ??_C@_00CNPNBAHC@?$AA@     10006c50     libucrt:mbrtowc.obj
 0001:00005cb8       ??_C@_1BA@BALFACEM@?$AAC?$AAO?$AAN?$AAO?$AAU?$AAT?$AA$?$AA?$AA@ 10006cb8     libucrt:initcon.obj
 0001:00005dd0       __infinity                 10006dd0     libucrt:87tran.obj
 0001:00005dda       __minfinity                10006dda     libucrt:87tran.obj
 0001:00005de4       __logemax                  10006de4     libucrt:87tran.obj
 0001:00005e0a       __OP_EXPjmptab             10006e0a     libucrt:87tran.obj
 0001:00005e30       __indefinite               10006e30     libucrt:87disp.obj
 0001:00005e3a       __piby2                    10006e3a     libucrt:87disp.obj
 0001:00005e44       __piby4                    10006e44     libucrt:87disp.obj
 0001:00005e78       __DEFAULT_CW_in_mem        10006e78     libucrt:common.obj
 0001:00005e7a       __pi_by_2_to_61            10006e7a     libucrt:common.obj
 0001:00005eb4       ??_C@_03MGHMBJCF@log?$AA@  10006eb4     libucrt:libm_error.obj
 0001:00005eb8       ??_C@_05HGHHAHAP@log10?$AA@ 10006eb8     libucrt:libm_error.obj
 0001:00005ec0       ??_C@_03KHJOGHMM@exp?$AA@  10006ec0     libucrt:libm_error.obj
 0001:00005ec4       ??_C@_03JGHBODFD@pow?$AA@  10006ec4     libucrt:libm_error.obj
 0001:00005ec8       ??_C@_04FIHNOPOL@asin?$AA@ 10006ec8     libucrt:libm_error.obj
 0001:00005ed0       ??_C@_04PDIFKINK@acos?$AA@ 10006ed0     libucrt:libm_error.obj
 0001:00005ed8       ??_C@_04EIAKFFMI@sqrt?$AA@ 10006ed8     libucrt:libm_error.obj
 0001:00005ee0       __real@3ff0000000000000    10006ee0     libucrt:libm_error.obj
 0001:00005f00       ___acrt_log10_table_t      10006f00     libucrt:log10_tables.obj
 0001:00006310       ___acrt_log10_table_cb     10007310     libucrt:log10_tables.obj
 0001:00006720       __real@3fe0000000000000    10007720     libucrt:powhlp.obj
 0001:00006810       ??_C@_04COOMCNPB@sinh?$AA@ 10007810     libucrt:fpexcept.obj
 0001:00006818       ??_C@_04HPJJNFIM@cosh?$AA@ 10007818     libucrt:fpexcept.obj
 0001:00006820       ??_C@_04FJHINJAO@tanh?$AA@ 10007820     libucrt:fpexcept.obj
 0001:00006828       ??_C@_04MLLJIGOK@atan?$AA@ 10007828     libucrt:fpexcept.obj
 0001:00006830       ??_C@_05KNGEOGJB@atan2?$AA@ 10007830     libucrt:fpexcept.obj
 0001:00006838       ??_C@_03BLEJJJBH@sin?$AA@  10007838     libucrt:fpexcept.obj
 0001:0000683c       ??_C@_03LALBNOCG@cos?$AA@  1000783c     libucrt:fpexcept.obj
 0001:00006840       ??_C@_03IIINPABG@tan?$AA@  10007840     libucrt:fpexcept.obj
 0001:00006844       ??_C@_04GFPJNGEK@ceil?$AA@ 10007844     libucrt:fpexcept.obj
 0001:0000684c       ??_C@_05PBJFFIGL@floor?$AA@ 1000784c     libucrt:fpexcept.obj
 0001:00006854       ??_C@_04ODHECPBC@fabs?$AA@ 10007854     libucrt:fpexcept.obj
 0001:0000685c       ??_C@_04EHEDPDJG@modf?$AA@ 1000785c     libucrt:fpexcept.obj
 0001:00006864       ??_C@_05CEJMAHNP@ldexp?$AA@ 10007864     libucrt:fpexcept.obj
 0001:0000686c       ??_C@_05KBKMEMPO@_cabs?$AA@ 1000786c     libucrt:fpexcept.obj
 0001:00006874       ??_C@_06MEIMCGCF@_hypot?$AA@ 10007874     libucrt:fpexcept.obj
 0001:0000687c       ??_C@_04KEPJIHGP@fmod?$AA@ 1000787c     libucrt:fpexcept.obj
 0001:00006884       ??_C@_05GKKHEGJL@frexp?$AA@ 10007884     libucrt:fpexcept.obj
 0001:0000688c       ??_C@_03MJLDFKDL@_y0?$AA@  1000788c     libucrt:fpexcept.obj
 0001:00006890       ??_C@_03NAKIGLHK@_y1?$AA@  10007890     libucrt:fpexcept.obj
 0001:00006894       ??_C@_03ONILCKOB@_yn?$AA@  10007894     libucrt:fpexcept.obj
 0001:00006898       ??_C@_05JGDBENOH@_logb?$AA@ 10007898     libucrt:fpexcept.obj
 0001:000068a0       ??_C@_0L@KDOEJCKC@_nextafter?$AA@ 100078a0     libucrt:fpexcept.obj
 0001:000068b0       __d_inf                    100078b0     libucrt:util.obj
 0001:000068b8       __d_max                    100078b8     libucrt:util.obj
 0001:000068c0       __d_mzero                  100078c0     libucrt:util.obj
 0001:000068f0       __load_config_used         100078f0     LIBCMT:loadcfg.obj
 0001:00006990       ??_R4exception@std@@6B@    10007990     LIBCMT:throw_bad_alloc.obj
 0001:000069a4       ??_R3exception@std@@8      100079a4     LIBCMT:throw_bad_alloc.obj
 0001:000069b4       ??_R2exception@std@@8      100079b4     LIBCMT:throw_bad_alloc.obj
 0001:000069bc       ??_R1A@?0A@EA@exception@std@@8 100079bc     LIBCMT:throw_bad_alloc.obj
 0001:000069d8       ??_R4bad_alloc@std@@6B@    100079d8     LIBCMT:throw_bad_alloc.obj
 0001:000069ec       ??_R3bad_alloc@std@@8      100079ec     LIBCMT:throw_bad_alloc.obj
 0001:000069fc       ??_R2bad_alloc@std@@8      100079fc     LIBCMT:throw_bad_alloc.obj
 0001:00006a08       ??_R1A@?0A@EA@bad_alloc@std@@8 10007a08     LIBCMT:throw_bad_alloc.obj
 0001:00006a24       ??_R4bad_array_new_length@std@@6B@ 10007a24     LIBCMT:throw_bad_alloc.obj
 0001:00006a38       ??_R3bad_array_new_length@std@@8 10007a38     LIBCMT:throw_bad_alloc.obj
 0001:00006a48       ??_R2bad_array_new_length@std@@8 10007a48     LIBCMT:throw_bad_alloc.obj
 0001:00006a58       ??_R1A@?0A@EA@bad_array_new_length@std@@8 10007a58     LIBCMT:throw_bad_alloc.obj
 0001:00006a74       ??_R4type_info@@6B@        10007a74     LIBCMT:std_type_info_static.obj
 0001:00006a88       ??_R3type_info@@8          10007a88     LIBCMT:std_type_info_static.obj
 0001:00006a98       ??_R2type_info@@8          10007a98     LIBCMT:std_type_info_static.obj
 0001:00006aa0       ??_R1A@?0A@EA@type_info@@8 10007aa0     LIBCMT:std_type_info_static.obj
 0001:00006ac0       ___safe_se_handler_table   10007ac0     <linker-defined>
 0001:00006d68       ___rtc_iaa                 10007d68     LIBCMT:initsect.obj
 0001:00006d6c       ___rtc_izz                 10007d6c     LIBCMT:initsect.obj
 0001:00006d70       ___rtc_taa                 10007d70     LIBCMT:initsect.obj
 0001:00006d74       ___rtc_tzz                 10007d74     LIBCMT:initsect.obj
 0001:00006d80       __alloca_probe             10007d80 f   chkstk.obj
 0001:00006d80       __chkstk                   10007d80 f   chkstk.obj
 0001:00006db0       ?fputc@@YAHHPAX@Z          10007db0 f   fileio.obj
 0001:00007040       ?PrintHandleInfo@@YA_NKPAX_NPAVPerfThread@@@Z 10008040 f   handles.obj
 0001:000077d0       ??0PluginDialogBuilder@@QAE@ABUPluginStartupInfo@@ABU_GUID@@1HPB_WP6GHPAXHH3@Z3_K@Z 100087d0 f i PCFG.OBJ
 0001:000078d0       ??1?$DialogBuilderBase@UFarDialogItem@@@@MAE@XZ 100088d0 f i PCFG.OBJ
 0001:00007910       ??1PluginDialogBuilder@@UAE@XZ 10008910 f i PCFG.OBJ
 0001:00007930       ??_G?$DialogBuilderBase@UFarDialogItem@@@@MAEPAXI@Z 10008930 f i PCFG.OBJ
 0001:00007930       ??_E?$DialogBuilderBase@UFarDialogItem@@@@MAEPAXI@Z 10008930 f i PCFG.OBJ
 0001:00007950       ??_E?$DialogItemBinding@UFarDialogItem@@@@UAEPAXI@Z 10008950 f i PCFG.OBJ
 0001:00007950       ??_G?$DialogItemBinding@UFarDialogItem@@@@UAEPAXI@Z 10008950 f i PCFG.OBJ
 0001:00007980       ??_GPluginEditFieldBinding@@UAEPAXI@Z 10008980 f i Pclass.obj
 0001:00007980       ??_EPluginCheckBoxBinding@@UAEPAXI@Z 10008980 f i PCFG.OBJ
 0001:00007980       ??_EPluginEditFieldBinding@@UAEPAXI@Z 10008980 f i Pclass.obj
 0001:00007980       ??_GPluginCheckBoxBinding@@UAEPAXI@Z 10008980 f i PCFG.OBJ
 0001:000079b0       ??_EPluginDialogBuilder@@UAEPAXI@Z 100089b0 f i PCFG.OBJ
 0001:000079b0       ??_GPluginDialogBuilder@@UAEPAXI@Z 100089b0 f i PCFG.OBJ
 0001:000079f0       ??_EPluginIntEditFieldBinding@@UAEPAXI@Z 100089f0 f i PCFG.OBJ
 0001:000079f0       ??_GPluginIntEditFieldBinding@@UAEPAXI@Z 100089f0 f i PCFG.OBJ
 0001:000079f0       ??_GPluginUIntEditFieldBinding@@UAEPAXI@Z 100089f0 f i PCFG.OBJ
 0001:000079f0       ??_EPluginUIntEditFieldBinding@@UAEPAXI@Z 100089f0 f i PCFG.OBJ
 0001:00007a20       ??_GPluginRadioButtonBinding@@UAEPAXI@Z 10008a20 f i PCFG.OBJ
 0001:00007a20       ??_EPluginRadioButtonBinding@@UAEPAXI@Z 10008a20 f i PCFG.OBJ
 0001:00007a50       ?AddButtons@?$DialogBuilderBase@UFarDialogItem@@@@QAEXHPBHHH@Z 10008a50 f i PCFG.OBJ
 0001:00007c80       ?AddDialogItem@?$DialogBuilderBase@UFarDialogItem@@@@IAEPAUFarDialogItem@@W4FARDIALOGITEMTYPES@@PB_W@Z 10008c80 f i PCFG.OBJ
 0001:00007da0       ?AddUIntEditField@?$DialogBuilderBase@UFarDialogItem@@@@UAEPAUFarDialogItem@@PAIH@Z 10008da0 f i PCFG.OBJ
 0001:00007da0       ?AddIntEditField@?$DialogBuilderBase@UFarDialogItem@@@@UAEPAUFarDialogItem@@PAHH@Z 10008da0 f i PCFG.OBJ
 0001:00007da0       ?CreateCheckBoxBinding@?$DialogBuilderBase@UFarDialogItem@@@@MAEPAU?$DialogItemBinding@UFarDialogItem@@@@PAHH@Z 10008da0 f i PCFG.OBJ
 0001:00007db0       ?AddIntEditField@PluginDialogBuilder@@UAEPAUFarDialogItem@@PAHH@Z 10008db0 f i PCFG.OBJ
 0001:00007ed0       ?AddUIntEditField@PluginDialogBuilder@@UAEPAUFarDialogItem@@PAIH@Z 10008ed0 f i PCFG.OBJ
 0001:00007ff0       ?Config@@YAHXZ             10008ff0 f   PCFG.OBJ
 0001:00008610       ?CreateCheckBoxBinding@PluginDialogBuilder@@MAEPAU?$DialogItemBinding@UFarDialogItem@@@@PAHH@Z 10009610 f i PCFG.OBJ
 0001:00008670       ?CreateRadioButtonBinding@?$DialogBuilderBase@UFarDialogItem@@@@MAEPAU?$DialogItemBinding@UFarDialogItem@@@@PAH@Z 10009670 f i PCFG.OBJ
 0001:00008670       ?GetLangString@?$DialogBuilderBase@UFarDialogItem@@@@MAEPB_WH@Z 10009670 f i PCFG.OBJ
 0001:00008680       ?CreateRadioButtonBinding@PluginDialogBuilder@@MAEPAU?$DialogItemBinding@UFarDialogItem@@@@PAH@Z 10009680 f i PCFG.OBJ
 0001:000086d0       ?DoShowDialog@?$DialogBuilderBase@UFarDialogItem@@@@MAEHXZ 100096d0 f i PCFG.OBJ
 0001:000086e0       ?DoShowDialog@PluginDialogBuilder@@MAEHXZ 100096e0 f i PCFG.OBJ
 0001:00008730       ?GetLangString@PluginDialogBuilder@@MAEPB_WH@Z 10009730 f i PCFG.OBJ
 0001:00008750       ?InitDialogItem@?$DialogBuilderBase@UFarDialogItem@@@@MAEXPAUFarDialogItem@@PB_W@Z 10009750 f i PCFG.OBJ
 0001:00008750       ?SaveValue@?$DialogItemBinding@UFarDialogItem@@@@UAEXPAUFarDialogItem@@H@Z 10009750 f i PCFG.OBJ
 0001:00008760       ?InitDialogItem@PluginDialogBuilder@@MAEXPAUFarDialogItem@@PB_W@Z 10009760 f i PCFG.OBJ
 0001:00008780       ?ItemWidth@?$DialogBuilderBase@UFarDialogItem@@@@IAEHABUFarDialogItem@@@Z 10009780 f i PCFG.OBJ
 0001:000087f0       ?Read@_Opt@@SAXXZ          100097f0 f   PCFG.OBJ
 0001:00008b20       ?SaveValue@PluginCheckBoxBinding@@UAEXPAUFarDialogItem@@H@Z 10009b20 f i PCFG.OBJ
 0001:00008b70       ?SaveValue@PluginIntEditFieldBinding@@UAEXPAUFarDialogItem@@H@Z 10009b70 f i PCFG.OBJ
 0001:00008ba0       ?SaveValue@PluginRadioButtonBinding@@UAEXPAUFarDialogItem@@H@Z 10009ba0 f i PCFG.OBJ
 0001:00008bd0       ?SaveValue@PluginUIntEditFieldBinding@@UAEXPAUFarDialogItem@@H@Z 10009bd0 f i PCFG.OBJ
 0001:00008c00       ?ShowDialog@?$DialogBuilderBase@UFarDialogItem@@@@QAE_NXZ 10009c00 f i PCFG.OBJ
 0001:00008cf0       ?TextWidth@?$DialogBuilderBase@UFarDialogItem@@@@MAEHABUFarDialogItem@@@Z 10009cf0 f i PCFG.OBJ
 0001:00008d00       ?TextWidth@PluginDialogBuilder@@MAEHABUFarDialogItem@@@Z 10009d00 f i PCFG.OBJ
 0001:00008d10       ?UpdateBorderSize@?$DialogBuilderBase@UFarDialogItem@@@@IAEXXZ 10009d10 f i PCFG.OBJ
 0001:00008e70       ?Write@_Opt@@SAXXZ         10009e70 f   PCFG.OBJ
 0001:000090b0       ??0Plist@@QAE@XZ           1000a0b0 f   Pclass.obj
 0001:00009240       ??0ui64Table@@QAE@XZ       1000a240 f   Pclass.obj
 0001:00009280       ??1Plist@@QAE@XZ           1000a280 f   Pclass.obj
 0001:000092d0       ?AddEditField@PluginDialogBuilder@@QAEPAUFarDialogItem@@PA_WHHPB_W_N@Z 1000a2d0 f i Pclass.obj
 0001:000093a0       ?Compare@Plist@@QAEHPBUPluginPanelItem@@0I@Z 1000a3a0 f   Pclass.obj
 0001:00009530       ?Connect@Plist@@QAE_NPB_W00@Z 1000a530 f   Pclass.obj
 0001:00009720       ?ConnectWMI@Plist@@AAE_NXZ 1000a720 f   Pclass.obj
 0001:000097a0       ?DeleteFiles@Plist@@QAEHPAUPluginPanelItem@@H_K@Z 1000a7a0 f   Pclass.obj
 0001:00009a80       ?DisconnectWMI@Plist@@AAEXXZ 1000aa80 f   Pclass.obj
 0001:00009ab0       ?EnumWndProc@@YGHPAUHWND__@@J@Z 1000aab0 f   Pclass.obj
 0001:00009b30       ?FreeFindData@Plist@@QAEXPAUPluginPanelItem@@H@Z 1000ab30 f   Pclass.obj
 0001:00009b90       ?GeneratePanelModes@Plist@@AAEXXZ 1000ab90 f   Pclass.obj
 0001:0000a180       ?GetFiles@Plist@@QAEHPAUPluginPanelItem@@HHPAPB_W_KAAU_Opt@@@Z 1000b180 f   Pclass.obj
 0001:0000af90       ?GetFindData@Plist@@QAEHAAPAUPluginPanelItem@@AAI_K@Z 1000bf90 f   Pclass.obj
 0001:0000b700       ?GetOpenPanelInfo@Plist@@QAEXPAUOpenPanelInfo@@@Z 1000c700 f   Pclass.obj
 0001:0000b870       ?GetVersionInfo@Plist@@SA_NPA_WAAPAEAAPA_W2@Z 1000c870 f   Pclass.obj
 0001:0000b9a0       ?InitializePanelModes@Plist@@SAXXZ 1000c9a0 f   Pclass.obj
 0001:0000bda0       ?PrintOwnerInfo@Plist@@AAEXPAXK@Z 1000cda0 f   Pclass.obj
 0001:0000bf90       ?PrintTitle@Plist@@SAPA_WH@Z 1000cf90 f   Pclass.obj
 0001:0000bfe0       ?ProcessEvent@Plist@@QAEHHPAX@Z 1000cfe0 f   Pclass.obj
 0001:0000c170       ?ProcessKey@Plist@@QAEHPBU_INPUT_RECORD@@@Z 1000d170 f   Pclass.obj
 0001:0000d580       ?Reread@Plist@@AAEXXZ      1000e580 f   Pclass.obj
 0001:0000d600       ?SavePanelModes@Plist@@SAXXZ 1000e600 f   Pclass.obj
 0001:0000d840       ?SaveValue@PluginEditFieldBinding@@UAEXPAUFarDialogItem@@H@Z 1000e840 f i Pclass.obj
 0001:0000d870       ?TranslateMode@Plist@@CA_NPB_WPA_W@Z 1000e870 f   Pclass.obj
 0001:0000dac0       ?WmiError@Plist@@AAEXXZ    1000eac0 f   Pclass.obj
 0001:0000db00       ??0PerfThread@@QAE@AAVPlist@@PB_W11@Z 1000eb00 f   perfthread.obj
 0001:0000dee0       ??1PerfThread@@QAE@XZ      1000eee0 f   perfthread.obj
 0001:0000df60       ?GetProcessData@PerfThread@@QBEPAUProcessPerfData@@KK@Z 1000ef60 f   perfthread.obj
 0001:0000dfc0       ?Refresh@PerfThread@@AAEXXZ 1000efc0 f   perfthread.obj
 0001:0000e730       ?SyncReread@PerfThread@@QAEXXZ 1000f730 f   perfthread.obj
 0001:0000e760       ?ThreadProc@PerfThread@@AAGKXZ 1000f760 f   perfthread.obj
 0001:0000e950       ?ThreadProc@PerfThread@@CGKPAX@Z 1000f950 f   perfthread.obj
 0001:0000e9a0       ?CreateToken@DebugToken@@SA_NXZ 1000f9a0 f   Plist.obj
 0001:0000ea60       ?DumpNTCounters@@YAXPAXAAVPerfThread@@KK@Z 1000fa60 f   Plist.obj
 0001:0000ed20       ?Enable@DebugToken@@QAE_NXZ 1000fd20 f   Plist.obj
 0001:0000edb0       ?GetInternalProcessData@@YAHPAXPAU_LDR_MODULE@@AAPAU_RTL_USER_PROCESS_PARAMETERS@@AAPAD_N@Z 1000fdb0 f   Plist.obj
 0001:0000ee90       ?GetList@@YAHAAPAUPluginPanelItem@@AAIAAVPerfThread@@@Z 1000fe90 f   Plist.obj
 0001:0000f150       ?GetOpenProcessData@@YAXPAXPA_WK1K1KPAPA_W2@Z 10010150 f   Plist.obj
 0001:0000f450       ?GetPData@@YA_NAAUProcessData@@AAUProcessPerfData@@@Z 10010450 f   Plist.obj
 0001:0000f4d0       ?KillProcess@@YAHKPAUHWND__@@@Z 100104d0 f   Plist.obj
 0001:0000f5c0       ?OpenProcessForced@@YAPAXPAVDebugToken@@KKH@Z 100105c0 f   Plist.obj
 0001:0000f610       ?PrintModules@@YAXPAXKAAU_Opt@@@Z 10010610 f   Plist.obj
 0001:0000f8f0       ?PrintNTCurDirAndEnv@@YAXPAX0H@Z 100108f0 f   Plist.obj
 0001:0000fa40       ?PrintTime@@YAPA_WK_N@Z    10010a40 f   Plist.obj
 0001:0000fad0       ?PrintTime@@YAPA_W_K_N@Z   10010ad0 f   Plist.obj
 0001:0000fb40       ?Revert@DebugToken@@QAE_NXZ 10010b40 f   Plist.obj
 0001:0000fb80       ?ConvertDate@@YAXABU_FILETIME@@PA_W1@Z 10010b80 f   Pmix.obj
 0001:0000fc10       ?GetMsg@@YAPB_WH@Z         10010c10 f   Pmix.obj
 0001:0000fc20       ?WinError@@YAHPA_W@Z       10010c20 f   Pmix.obj
 0001:0000fd80       ??0WMIConnection@@QAE@XZ   10010d80 f   WMI.obj
 0001:0000fdb0       ??1WMIConnection@@QAE@XZ   10010db0 f   WMI.obj
 0001:0000fdd0       ?Connect@WMIConnection@@QAE_NPB_W00@Z 10010dd0 f   WMI.obj
 0001:0000ff20       ?Disconnect@WMIConnection@@QAEXXZ 10010f20 f   WMI.obj
 0001:0000ff40       ?ExecMethod@WMIConnection@@AAEHKPB_W0K@Z 10010f40 f   WMI.obj
 0001:00010130       ?GetProcessExecutablePath@WMIConnection@@QAEXKPA_W@Z 10011130 f   WMI.obj
 0001:000101f0       ?GetProcessOwner@WMIConnection@@QAEXKPA_W0@Z 100111f0 f   WMI.obj
 0001:00010340       ?GetProcessPriority@WMIConnection@@QAEKK@Z 10011340 f   WMI.obj
 0001:00010400       ?GetProcessSessionId@WMIConnection@@QAEHK@Z 10011400 f   WMI.obj
 0001:000104c0       ?GetProcessUserSid@WMIConnection@@QAEXKPA_W@Z 100114c0 f   WMI.obj
 0001:000105b0       ?SetProcessPriority@WMIConnection@@QAEHKK@Z 100115b0 f   WMI.obj
 0001:000105d0       ?TerminateProcess@WMIConnection@@QAEHK@Z 100115d0 f   WMI.obj
 0001:00010630       ?Message@@YAHIPA_WPAPB_WHH@Z 10011630 f   Proclist.obj
 0001:000107b0       _ClosePanelW@4             100117b0 f   Proclist.obj
 0001:000107e0       _CompareW@4                100117e0 f   Proclist.obj
 0001:00010800       _ConfigureW@4              10011800 f   Proclist.obj
 0001:00010810       _DeleteFilesW@4            10011810 f   Proclist.obj
 0001:00010830       _ExitFARW@4                10011830 f   Proclist.obj
 0001:00010860       _FreeFindDataW@4           10011860 f   Proclist.obj
 0001:00010880       _GetFilesW@4               10011880 f   Proclist.obj
 0001:000108b0       _GetFindDataW@4            100118b0 f   Proclist.obj
 0001:000108d0       _GetGlobalInfoW@4          100118d0 f   Proclist.obj
 0001:00010960       _GetOpenPanelInfoW@4       10011960 f   Proclist.obj
 0001:00010970       _GetPluginInfoW@4          10011970 f   Proclist.obj
 0001:00010a20       _OpenW@4                   10011a20 f   Proclist.obj
 0001:00010aa0       _ProcessPanelEventW@4      10011aa0 f   Proclist.obj
 0001:00010ac0       _ProcessPanelInputW@4      10011ac0 f   Proclist.obj
 0001:00010ae0       _SetStartupInfoW@4         10011ae0 f   Proclist.obj
 0001:00010f30       _DecodePointerWrapper@4    10011f30 f   vc_crt_fix_impl.obj
 0001:00010f80       _EncodePointerWrapper@4    10011f80 f   vc_crt_fix_impl.obj
 0001:00010fd0       _GetLogicalProcessorInformationWrapper@8 10011fd0 f   vc_crt_fix_impl.obj
 0001:00011020       _GetModuleHandleExWWrapper@12 10012020 f   vc_crt_fix_impl.obj
 0001:00011070       _GetNumaHighestNodeNumberWrapper@4 10012070 f   vc_crt_fix_impl.obj
 0001:000110c0       _InitializeSListHeadWrapper@4 100120c0 f   vc_crt_fix_impl.obj
 0001:00011110       _InterlockedFlushSListWrapper@4 10012110 f   vc_crt_fix_impl.obj
 0001:00011160       _InterlockedPopEntrySListWrapper@4 10012160 f   vc_crt_fix_impl.obj
 0001:000111b0       _InterlockedPushEntrySListWrapper@8 100121b0 f   vc_crt_fix_impl.obj
 0001:00011200       _InterlockedPushListSListExWrapper@16 10012200 f   vc_crt_fix_impl.obj
 0001:00011250       _QueryDepthSListWrapper@4  10012250 f   vc_crt_fix_impl.obj
 0001:000112a0       _RtlFirstEntrySListWrapper@4 100122a0 f   vc_crt_fix_impl.obj
 0001:000112f0       _SetThreadStackGuaranteeWrapper@4 100122f0 f   vc_crt_fix_impl.obj
 0001:00011333       _WNetAddConnection2W@16    10012333 f   mpr:MPR.dll
 0001:00011339       _WNetCancelConnection2W@12 10012339 f   mpr:MPR.dll
 0001:0001133f       _GetFileVersionInfoSizeW@8 1001233f f   version:VERSION.dll
 0001:00011345       _GetFileVersionInfoW@16    10012345 f   version:VERSION.dll
 0001:0001134b       _VerQueryValueW@16         1001234b f   version:VERSION.dll
 0001:00011351       ??_U@YAPAXI@Z              10012351 f   LIBCMT:new_array.obj
 0001:0001135a       ??_V@YAXPAX@Z              1001235a f   LIBCMT:delete_array.obj
 0001:0001135f       ??2@YAPAXI@Z               1001235f f   LIBCMT:new_scalar.obj
 0001:0001138f       ??3@YAXPAXI@Z              1001238f f   LIBCMT:delete_scalar_size.obj
 0001:000113a0       __aulldiv                  100123a0 f   LIBCMT:ulldiv.obj
 0001:00011410       __alldiv                   10012410 f   LIBCMT:lldiv.obj
 0001:000114c0       __allmul                   100124c0 f   LIBCMT:llmul.obj
 0001:00011500       __aullrem                  10012500 f   LIBCMT:ullrem.obj
 0001:00011575       ??$__crt_fast_encode_pointer@PAP6AXXZ@@YAPAP6AXXZQAP6AXXZ@Z 10012575 f i LIBCMT:utility.obj
 0001:00011575       ??$__crt_fast_encode_pointer@PAX@@YAPAXQAX@Z 10012575 f i libvcruntime:winapi_downlevel.obj
 0001:000115d6       ___scrt_acquire_startup_lock 100125d6 f   LIBCMT:utility.obj
 0001:00011608       ___scrt_dllmain_after_initialize_c 10012608 f   LIBCMT:utility.obj
 0001:00011633       ___scrt_dllmain_before_initialize_c 10012633 f   LIBCMT:utility.obj
 0001:00011641       ___scrt_dllmain_crt_thread_attach 10012641 f   LIBCMT:utility.obj
 0001:00011660       ___scrt_dllmain_crt_thread_detach 10012660 f   LIBCMT:utility.obj
 0001:0001166d       ___scrt_dllmain_exception_filter 1001266d f   LIBCMT:utility.obj
 0001:000116a1       ___scrt_dllmain_uninitialize_c 100126a1 f   LIBCMT:utility.obj
 0001:000116c4       ___scrt_dllmain_uninitialize_critical 100126c4 f   LIBCMT:utility.obj
 0001:000116d1       ___scrt_initialize_crt     100126d1 f   LIBCMT:utility.obj
 0001:0001170a       ___scrt_initialize_onexit_tables 1001270a f   LIBCMT:utility.obj
 0001:000117af       ___scrt_is_nonwritable_in_current_image 100127af f   LIBCMT:utility.obj
 0001:00011843       ___scrt_release_startup_lock 10012843 f   LIBCMT:utility.obj
 0001:00011860       ___scrt_uninitialize_crt   10012860 f   LIBCMT:utility.obj
 0001:00011888       __onexit                   10012888 f   LIBCMT:utility.obj
 0001:000118c3       _atexit                    100128c3 f   LIBCMT:utility.obj
 0001:00011bf8       __DllMainCRTStartup@12     10012bf8 f   LIBCMT:dll_dllmain.obj
 0001:00011c1b       ??3@YAXPAX@Z               10012c1b f   LIBCMT:delete_scalar.obj
 0001:00011c20       ??0bad_alloc@std@@QAE@ABV01@@Z 10012c20 f i LIBCMT:throw_bad_alloc.obj
 0001:00011c3b       ??0bad_alloc@std@@QAE@XZ   10012c3b f i LIBCMT:throw_bad_alloc.obj
 0001:00011c53       ??0bad_array_new_length@std@@QAE@ABV01@@Z 10012c53 f i LIBCMT:throw_bad_alloc.obj
 0001:00011c6e       ??0bad_array_new_length@std@@QAE@XZ 10012c6e f i LIBCMT:throw_bad_alloc.obj
 0001:00011c86       ??0exception@std@@QAE@ABV01@@Z 10012c86 f i LIBCMT:throw_bad_alloc.obj
 0001:00011cb2       ??1bad_alloc@std@@UAE@XZ   10012cb2 f i LIBCMT:throw_bad_alloc.obj
 0001:00011cb2       ??1bad_array_new_length@std@@UAE@XZ 10012cb2 f i LIBCMT:throw_bad_alloc.obj
 0001:00011cc3       ??_Gexception@std@@UAEPAXI@Z 10012cc3 f i LIBCMT:throw_bad_alloc.obj
 0001:00011cc3       ??_Gbad_array_new_length@std@@UAEPAXI@Z 10012cc3 f i LIBCMT:throw_bad_alloc.obj
 0001:00011cc3       ??_Ebad_alloc@std@@UAEPAXI@Z 10012cc3 f i LIBCMT:throw_bad_alloc.obj
 0001:00011cc3       ??_Ebad_array_new_length@std@@UAEPAXI@Z 10012cc3 f i LIBCMT:throw_bad_alloc.obj
 0001:00011cc3       ??_Eexception@std@@UAEPAXI@Z 10012cc3 f i LIBCMT:throw_bad_alloc.obj
 0001:00011cc3       ??_Gbad_alloc@std@@UAEPAXI@Z 10012cc3 f i LIBCMT:throw_bad_alloc.obj
 0001:00011cf0       ?__scrt_throw_std_bad_alloc@@YAXXZ 10012cf0 f   LIBCMT:throw_bad_alloc.obj
 0001:00011d0d       ?__scrt_throw_std_bad_array_new_length@@YAXXZ 10012d0d f   LIBCMT:throw_bad_alloc.obj
 0001:00011d2a       ?what@exception@std@@UBEPBDXZ 10012d2a f i LIBCMT:throw_bad_alloc.obj
 0001:00011d37       ___isa_available_init      10012d37 f   LIBCMT:cpu_disp.obj
 0001:00011ece       __get_startup_argv_mode    10012ece f   LIBCMT:argv_mode.obj
 0001:00011ed2       ___scrt_is_ucrt_dll_in_use 10012ed2 f   LIBCMT:ucrt_detection.obj
 0001:00011ede       ___scrt_fastfail           10012ede f   LIBCMT:utility_desktop.obj
 0001:00011ff8       __crt_debugger_hook        10012ff8 f   LIBCMT:utility_desktop.obj
 0001:00012000       __SEH_prolog4              10013000 f   LIBCMT:sehprolg4.obj
 0001:00012046       __SEH_epilog4              10013046 f   LIBCMT:sehprolg4.obj
 0001:0001205b       @_guard_check_icall_nop@4  1001305b f i LIBCMT:guard_support.obj
 0001:000120a9       ___security_init_cookie    100130a9 f   LIBCMT:gs_support.obj
 0001:000120f4       _DllMain@12                100130f4 f   LIBCMT:dll_dllmain_stub.obj
 0001:000120fa       ?__scrt_initialize_type_info@@YAXXZ 100130fa f   LIBCMT:tncleanup.obj
 0001:00012106       ?__scrt_uninitialize_type_info@@YAXXZ 10013106 f   LIBCMT:tncleanup.obj
 0001:00012112       ___local_stdio_printf_options 10013112 f i LIBCMT:default_local_stdio_options.obj
 0001:00012118       ___local_stdio_scanf_options 10013118 f i LIBCMT:default_local_stdio_options.obj
 0001:0001211e       ___scrt_initialize_default_local_stdio_options 1001311e f   LIBCMT:default_local_stdio_options.obj
 0001:0001213b       ___scrt_get_dyn_tls_init_callback 1001313b f   LIBCMT:dyn_tls_init.obj
 0001:00012141       __RTC_Initialize           10013141 f   LIBCMT:initsect.obj
 0001:0001216d       __RTC_Terminate            1001316d f   LIBCMT:initsect.obj
 0001:00012199       ??_Gtype_info@@UAEPAXI@Z   10013199 f i LIBCMT:std_type_info_static.obj
 0001:00012199       ??_Etype_info@@UAEPAXI@Z   10013199 f i LIBCMT:std_type_info_static.obj
 0001:000121bc       @__security_check_cookie@4 100131bc f   LIBCMT:secchk.obj
 0001:000121cd       ___raise_securityfailure   100131cd f   LIBCMT:gs_report.obj
 0001:000121f5       ___report_gsfailure        100131f5 f   LIBCMT:gs_report.obj
 0001:000122f0       _memset                    100132f0 f   libvcruntime:memset.obj
 0001:0001244a       _wcschr                    1001344a f   libvcruntime:wcschr.obj
 0001:00012511       _wcsrchr                   10013511 f   libvcruntime:wcsrchr.obj
 0001:000125c0       _memcpy                    100135c0 f   libvcruntime:memcpy.obj
 0001:00012b40       _memmove                   10013b40 f   libvcruntime:memmove.obj
 0001:000130b4       ___vcrt_initialize         100140b4 f   libvcruntime:initialization.obj
 0001:000130dd       ___vcrt_thread_attach      100140dd f   libvcruntime:initialization.obj
 0001:000130e8       ___vcrt_thread_detach      100140e8 f   libvcruntime:initialization.obj
 0001:000130f3       ___vcrt_uninitialize       100140f3 f   libvcruntime:initialization.obj
 0001:00013112       ___vcrt_uninitialize_critical 10014112 f   libvcruntime:initialization.obj
 0001:00013160       __except_handler4          10014160 f   libvcruntime:chandler4.obj
 0001:000132b7       ___std_exception_copy      100142b7 f   libvcruntime:std_exception.obj
 0001:0001331a       ___std_exception_destroy   1001431a f   libvcruntime:std_exception.obj
 0001:00013339       __CxxThrowException@8      10014339 f   libvcruntime:throw.obj
 0001:000133a6       ___std_type_info_destroy_list 100143a6 f   libvcruntime:std_type_info.obj
 0001:000133c9       ___vcrt_freefls@4          100143c9 f   libvcruntime:per_thread_data.obj
 0001:000133e5       ___vcrt_freeptd            100143e5 f   libvcruntime:per_thread_data.obj
 0001:0001341b       ___vcrt_getptd_noexit      1001441b f   libvcruntime:per_thread_data.obj
 0001:000134ad       ___vcrt_initialize_ptd     100144ad f   libvcruntime:per_thread_data.obj
 0001:000134e0       ___vcrt_uninitialize_ptd   100144e0 f   libvcruntime:per_thread_data.obj
 0001:000134fb       ___vcrt_initialize_locks   100144fb f   libvcruntime:locks.obj
 0001:00013537       ___vcrt_uninitialize_locks 10014537 f   libvcruntime:locks.obj
 0001:00013699       ___vcrt_FlsAlloc           10014699 f   libvcruntime:winapi_downlevel.obj
 0001:000136d4       ___vcrt_FlsFree            100146d4 f   libvcruntime:winapi_downlevel.obj
 0001:0001370f       ___vcrt_FlsGetValue        1001470f f   libvcruntime:winapi_downlevel.obj
 0001:0001374a       ___vcrt_FlsSetValue        1001474a f   libvcruntime:winapi_downlevel.obj
 0001:00013788       ___vcrt_InitializeCriticalSectionEx 10014788 f   libvcruntime:winapi_downlevel.obj
 0001:000137cf       ___vcrt_initialize_winapi_thunks 100147cf f   libvcruntime:winapi_downlevel.obj
 0001:000137f8       ___vcrt_uninitialize_winapi_thunks 100147f8 f   libvcruntime:winapi_downlevel.obj
 0001:0001382a       ___vcrt_initialize_pure_virtual_call_handler 1001482a f   libvcruntime:purevirt_data.obj
 0001:00013840       __local_unwind4            10014840 f   libvcruntime:exsup4.obj
 0001:00013918       __seh_longjmp_unwind4@4    10014918 f   libvcruntime:exsup4.obj
 0001:00013940       @_EH4_CallFilterFunc@8     10014940 f   libvcruntime:exsup4.obj
 0001:00013958       @_EH4_TransferToHandler@8  10014958 f   libvcruntime:exsup4.obj
 0001:00013974       @_EH4_GlobalUnwind2@8      10014974 f   libvcruntime:exsup4.obj
 0001:00013990       @_EH4_LocalUnwind@16       10014990 f   libvcruntime:exsup4.obj
 0001:000139a7       ___except_validate_context_record 100149a7 f   libvcruntime:jbcxrval.obj
 0001:000139d7       ___except_validate_jump_buffer 100149d7 f   libvcruntime:jbcxrval.obj
 0001:00013a10       __global_unwind2           10014a10 f   libvcruntime:exsup.obj
 0001:00013a76       __local_unwind2            10014a76 f   libvcruntime:exsup.obj
 0001:00013afa       __abnormal_termination     10014afa f   libvcruntime:exsup.obj
 0001:00013b20       __NLG_Notify1              10014b20 f   libvcruntime:exsup.obj
 0001:00013b2c       __NLG_Notify               10014b2c f   libvcruntime:exsup.obj
 0001:00013b43       __NLG_Dispatch2            10014b43     libvcruntime:exsup.obj
 0001:00013b43       __NLG_Dispatch             10014b43     libvcruntime:exsup.obj
 0001:00013b4b       __NLG_Call                 10014b4b f   libvcruntime:exsup.obj
 0001:00013b4d       __NLG_Return2              10014b4d     libvcruntime:exsup.obj
 0001:00013b50       __CallSettingFrame@12      10014b50 f   libvcruntime:lowhelpr.obj
 0001:00013b77       __NLG_Return               10014b77     libvcruntime:lowhelpr.obj
 0001:00013b9c       ___DestructExceptionObject 10014b9c f   libvcruntime:ehhelpers.obj
 0001:00013c3c       ?_CallMemberFunction0@@YGXQAX0@Z 10014c3c f i libvcruntime:ehhelpers.obj
 0001:00013c49       ??0_LocaleUpdate@@QAE@QAU__crt_locale_pointers@@@Z 10014c49 f i libucrt:memicmp.obj
 0001:00013ccc       __memicmp                  10014ccc f   libucrt:memicmp.obj
 0001:00013d2e       __memicmp_l                10014d2e f   libucrt:memicmp.obj
 0001:00013dde       _free                      10014dde f   libucrt:free.obj
 0001:00013dfb       _malloc                    10014dfb f   libucrt:malloc.obj
 0001:00013e06       ??$is_overflow_condition@K@__crt_strtox@@YA_NIK@Z 10014e06 f i libucrt:strtox.obj
 0001:00013e37       ??$make_c_string_character_source@_WPAPA_W@__crt_strtox@@YA?AV?$c_string_character_source@_W@0@QB_WQAPA_W@Z 10014e37 f i libucrt:strtox.obj
 0001:00013e52       ??$parse_integer@KV?$c_string_character_source@_W@__crt_strtox@@@__crt_strtox@@YAKQAU__crt_locale_pointers@@V?$c_string_character_source@_W@0@H_N@Z 10014e52 f i libucrt:strtox.obj
 0001:00014494       ?unget@?$c_string_character_source@_W@__crt_strtox@@QAEX_W@Z 10015494 f i libucrt:strtox.obj
 0001:000144c2       ?validate@?$c_string_character_source@_W@__crt_strtox@@QBE_NXZ 100154c2 f i libucrt:strtox.obj
 0001:000144dd       ___acrt_locale_get_ctype_array_value 100154dd f i libucrt:strtox.obj
 0001:000144ff       __chvalidchk_l             100154ff f i libucrt:strtox.obj
 0001:00014527       __ischartype_l             10015527 f i libucrt:strtox.obj
 0001:0001455a       _wcstol                    1001555a f   libucrt:strtox.obj
 0001:00014664       __ui64tow                  10015664 f   libucrt:xtoa.obj
 0001:00014686       _wcscspn                   10015686 f   libucrt:wcscspn.obj
 0001:000146e1       _wcsncat                   100156e1 f   libucrt:wcsncat.obj
 0001:00014726       _wcspbrk                   10015726 f   libucrt:wcspbrk.obj
 0001:00014774       _wcstok                    10015774 f   libucrt:wcstok.obj
 0001:00014799       __isleadbyte_l             10015799 f i libucrt:_wctype.obj
 0001:000147d5       _iswdigit                  100157d5 f i libucrt:_wctype.obj
 0001:000147e8       ___acrt_initialize_new_handler 100157e8 f   libucrt:new_handler.obj
 0001:000147f7       __callnewh                 100157f7 f   libucrt:new_handler.obj
 0001:00014824       __query_new_handler        10015824 f   libucrt:new_handler.obj
 0001:00014876       __seh_filter_dll           10015876 f   libucrt:exception_filter.obj
 0001:00014896       __seh_filter_exe           10015896 f   libucrt:exception_filter.obj
 0001:00014c56       ___acrt_initialize_thread_local_exit_callback 10015c56 f   libucrt:exit.obj
 0001:00014c65       __cexit                    10015c65 f   libucrt:exit.obj
 0001:00014c74       __exit                     10015c74 f   libucrt:exit.obj
 0001:00014c8a       __is_c_termination_complete 10015c8a f   libucrt:exit.obj
 0001:00014f42       ___acrt_allocate_buffer_for_argv 10015f42 f   libucrt:argv_parsing.obj
 0001:00014f91       __configure_narrow_argv    10015f91 f   libucrt:argv_parsing.obj
 0001:000150f0       ??$uninitialize@A6AXAAPAPA_W@Z@?$dual_state_global@PAPA_W@__crt_state_management@@QAEXA6AXAAPAPA_W@Z@Z 100160f0 f i libucrt:environment_initialization.obj
 0001:000150f0       ??$uninitialize@A6AXAAPAPAD@Z@?$dual_state_global@PAPAD@__crt_state_management@@QAEXA6AXAAPAPAD@Z@Z 100160f0 f i libucrt:environment_initialization.obj
 0001:0001514f       ___dcrt_uninitialize_environments_nolock 1001614f f   libucrt:environment_initialization.obj
 0001:00015186       __initialize_narrow_environment 10016186 f   libucrt:environment_initialization.obj
 0001:0001522d       ??$__crt_fast_encode_pointer@P6AHXZ@@YAP6AHXZQ6AHXZ@Z 1001622d f i libucrt:onexit.obj
 0001:00015453       __crt_atexit               10016453 f   libucrt:onexit.obj
 0001:00015469       __execute_onexit_table     10016469 f   libucrt:onexit.obj
 0001:00015498       __initialize_onexit_table  10016498 f   libucrt:onexit.obj
 0001:000154c1       __register_onexit_function 100164c1 f   libucrt:onexit.obj
 0001:0001551d       ___acrt_uninitialize_command_line 1001651d f   libucrt:argv_data.obj
 0001:000155f6       ___acrt_initialize         100165f6 f   libucrt:initialization.obj
 0001:00015608       ___acrt_thread_attach      10016608 f   libucrt:initialization.obj
 0001:00015613       ___acrt_thread_detach      10016613 f   libucrt:initialization.obj
 0001:0001561b       ___acrt_uninitialize       1001661b f   libucrt:initialization.obj
 0001:0001564b       ___acrt_uninitialize_critical 1001664b f   libucrt:initialization.obj
 0001:0001565d       __initterm                 1001665d f   libucrt:initterm.obj
 0001:000156a4       __initterm_e               100166a4 f   libucrt:initterm.obj
 0001:000156d2       _terminate                 100166d2 f   libucrt:terminate.obj
 0001:0001570e       __wcsdup                   1001670e f   libucrt:wcsdup.obj
 0001:0001570e       _wcsdup                    1001670e f   libucrt:wcsdup.obj
 0001:0001576d       _strcpy_s                  1001676d f   libucrt:strcpy_s.obj
 0001:000157c7       _abort                     100167c7 f   libucrt:abort.obj
 0001:0001580b       _calloc                    1001680b f   libucrt:calloc.obj
 0001:00015816       _wcsncmp                   10016816 f   libucrt:wcsncmp.obj
 0001:00015850       _strncmp                   10016850 f   libucrt:strncmp.obj
 0001:000158c8       ___acrt_call_reportfault   100168c8 f   libucrt:invalid_parameter.obj
 0001:00015a03       ___acrt_initialize_invalid_parameter_handler 10016a03 f   libucrt:invalid_parameter.obj
 0001:00015a12       __invalid_parameter        10016a12 f   libucrt:invalid_parameter.obj
 0001:00015a76       __invalid_parameter_noinfo 10016a76 f   libucrt:invalid_parameter.obj
 0001:00015a86       __invoke_watson            10016a86 f   libucrt:invalid_parameter.obj
 0001:00015c1d       __tolower_l                10016c1d f   libucrt:tolower_toupper.obj
 0001:00015c37       ___acrt_errno_from_os_error 10016c37 f   libucrt:errno.obj
 0001:00015c7a       ___acrt_errno_map_os_error 10016c7a f   libucrt:errno.obj
 0001:00015c9d       ___doserrno                10016c9d f   libucrt:errno.obj
 0001:00015cb0       __errno                    10016cb0 f   libucrt:errno.obj
 0001:00015cd0       ___ascii_memicmp           10016cd0 f   libucrt:_memicmp.obj
 0001:00016043       ___acrt_freeptd            10017043 f   libucrt:per_thread_data.obj
 0001:0001606f       ___acrt_getptd             1001706f f   libucrt:per_thread_data.obj
 0001:0001612c       ___acrt_getptd_head        1001712c f   libucrt:per_thread_data.obj
 0001:000161c6       ___acrt_getptd_noexit      100171c6 f   libucrt:per_thread_data.obj
 0001:0001627b       ___acrt_initialize_ptd     1001727b f   libucrt:per_thread_data.obj
 0001:000162a7       ___acrt_uninitialize_ptd   100172a7 f   libucrt:per_thread_data.obj
 0001:000162c1       ___acrt_update_locale_info 100172c1 f   libucrt:locale_update.obj
 0001:000162ee       ___acrt_update_multibyte_info 100172ee f   libucrt:locale_update.obj
 0001:0001637f       ___acrt_set_locale_changed 1001737f f   libucrt:wsetlocale.obj
 0001:0001638a       ___acrt_uninitialize_locale 1001738a f   libucrt:wsetlocale.obj
 0001:000163b3       __free_base                100173b3 f   libucrt:free_base.obj
 0001:000163ed       __malloc_base              100173ed f   libucrt:malloc_base.obj
 0001:0001643b       ___pctype_func             1001743b f   libucrt:ctype.obj
 0001:00016461       _iswctype                  10017461 f   libucrt:iswctype.obj
 0001:000164cc       __isctype_l                100174cc f   libucrt:isctype.obj
 0001:000165a1       ___acrt_wcstok_s_novalidation 100175a1 f   libucrt:wcstok_s.obj
 0001:0001667c       ___acrt_initialize_locks   1001767c f   libucrt:locks.obj
 0001:000166bd       ___acrt_lock               100176bd f   libucrt:locks.obj
 0001:000166d4       ___acrt_uninitialize_locks 100176d4 f   libucrt:locks.obj
 0001:00016705       ___acrt_unlock             10017705 f   libucrt:locks.obj
 0001:0001671c       ___acrt_get_process_end_policy 1001771c f   libucrt:win_policies.obj
 0001:0001674f       __calloc_base              1001774f f   libucrt:calloc_base.obj
 0001:00016945       ??$__acrt_mbs_to_wcs_cp@U__crt_win32_buffer_internal_dynamic_resizing@@@@YAHQBDAAV?$__crt_win32_buffer@_WU__crt_win32_buffer_internal_dynamic_resizing@@@@I@Z 10017945 f i libucrt:argv_wildcards.obj
 0001:00016e61       ?__acrt_get_utf8_acp_compatibility_codepage@@YAIXZ 10017e61 f i libucrt:argv_wildcards.obj
 0001:00016ea2       ?_deallocate@?$__crt_win32_buffer@DU__crt_win32_buffer_internal_dynamic_resizing@@@@AAEXXZ 10017ea2 f i libucrt:argv_wildcards.obj
 0001:00016ea2       ?_deallocate@?$__crt_win32_buffer@_WU__crt_win32_buffer_internal_dynamic_resizing@@@@AAEXXZ 10017ea2 f i libucrt:argv_wildcards.obj
 0001:00016ebc       ?allocate@?$__crt_win32_buffer@DU__crt_win32_buffer_internal_dynamic_resizing@@@@QAEHI@Z 10017ebc f i libucrt:argv_wildcards.obj
 0001:00016ef8       ?allocate@?$__crt_win32_buffer@_WU__crt_win32_buffer_internal_dynamic_resizing@@@@QAEHI@Z 10017ef8 f i libucrt:argv_wildcards.obj
 0001:00016f37       ?allocate@__crt_win32_buffer_internal_dynamic_resizing@@SAHQAPAXIABV__crt_win32_buffer_empty_debug_info@@@Z 10017f37 f i libucrt:argv_wildcards.obj
 0001:00016fdd       ___acrt_expand_narrow_argv_wildcards 10017fdd f   libucrt:argv_wildcards.obj
 0001:000170af       ?allocate@?$__crt_win32_buffer@DU__crt_win32_buffer_no_resizing@@@@QAEHI@Z 100180af f i libucrt:getmodulefilenamea.obj
 0001:000170d6       ?set_to_nullptr@?$__crt_win32_buffer@DU__crt_win32_buffer_no_resizing@@@@QAEXXZ 100180d6 f i libucrt:getmodulefilenamea.obj
 0001:000170ea       ___acrt_GetModuleFileNameA 100180ea f   libucrt:getmodulefilenamea.obj
 0001:0001769d       ___acrt_initialize_multibyte 1001869d f   libucrt:mbctype.obj
 0001:000176e5       ___acrt_update_thread_multibyte_data 100186e5 f   libucrt:mbctype.obj
 0001:000176f8       __setmbcp_nolock           100186f8 f   libucrt:mbctype.obj
 0001:000179c7       __ismbblead                100189c7 f   libucrt:ismbbyte.obj
 0001:000179df       ___acrt_initialize_command_line 100189df f   libucrt:argv_data.obj
 0001:000179f8       _wcscpy_s                  100189f8 f   libucrt:wcscpy_s.obj
 0001:00017a5c       ___acrt_MultiByteToWideChar 10018a5c f   libucrt:multibytetowidechar.obj
 0001:00017ad8       ___acrt_WideCharToMultiByte 10018ad8 f   libucrt:widechartomultibyte.obj
 0001:00017bbc       ___dcrt_get_narrow_environment_from_os 10018bbc f   libucrt:get_environment_from_os.obj
 0001:00017c42       __recalloc_base            10018c42 f   libucrt:recalloc.obj
 0001:00017e1b       ___acrt_initialize_lowio   10018e1b f   libucrt:ioinit.obj
 0001:00017e71       ___acrt_uninitialize_lowio 10018e71 f   libucrt:ioinit.obj
 0001:00018037       ___acrt_AppPolicyGetProcessTerminationMethodInternal@4 10019037 f   libucrt:winapi_thunks.obj
 0001:00018077       ___acrt_AreFileApisANSI@0  10019077 f   libucrt:winapi_thunks.obj
 0001:00018096       ___acrt_FlsAlloc@4         10019096 f   libucrt:winapi_thunks.obj
 0001:000180d5       ___acrt_FlsFree@4          100190d5 f   libucrt:winapi_thunks.obj
 0001:00018114       ___acrt_FlsGetValue@4      10019114 f   libucrt:winapi_thunks.obj
 0001:00018153       ___acrt_FlsSetValue@8      10019153 f   libucrt:winapi_thunks.obj
 0001:00018195       ___acrt_InitializeCriticalSectionEx@12 10019195 f   libucrt:winapi_thunks.obj
 0001:000181e0       ___acrt_LCMapStringEx@36   100191e0 f   libucrt:winapi_thunks.obj
 0001:0001823d       ___acrt_LocaleNameToLCID@8 1001923d f   libucrt:winapi_thunks.obj
 0001:0001826e       ___acrt_initialize_winapi_thunks 1001926e f   libucrt:winapi_thunks.obj
 0001:00018299       ___acrt_uninitialize_winapi_thunks 10019299 f   libucrt:winapi_thunks.obj
 0001:000182cf       ___acrt_initialize_heap    100192cf f   libucrt:heap_handle.obj
 0001:000182e0       ___acrt_uninitialize_heap  100192e0 f   libucrt:heap_handle.obj
 0001:000182ea       ___acrt_execute_initializers 100192ea f   libucrt:shared_initialization.obj
 0001:00018352       ___acrt_execute_uninitializers 10019352 f   libucrt:shared_initialization.obj
 0001:00018447       ___acrt_get_sigabrt_handler 10019447 f   libucrt:signal.obj
 0001:00018470       ___acrt_initialize_signal_handlers 10019470 f   libucrt:signal.obj
 0001:0001848e       ___fpecode                 1001948e f   libucrt:signal.obj
 0001:00018497       _raise                     10019497 f   libucrt:signal.obj
 0001:0001867e       ___acrt_has_user_matherr   1001967e f   libucrt:matherr.obj
 0001:00018696       ___acrt_initialize_user_matherr 10019696 f   libucrt:matherr.obj
 0001:000186a5       ___acrt_invoke_user_matherr 100196a5 f   libucrt:matherr.obj
 0001:000188a2       ___acrt_stdio_flush_nolock 100198a2 f   libucrt:fflush.obj
 0001:00018907       __fflush_nolock            10019907 f   libucrt:fflush.obj
 0001:0001894f       __flushall                 1001994f f   libucrt:fflush.obj
 0001:00018958       ___acrt_initialize_stdio   10019958 f   libucrt:_file.obj
 0001:00018a20       ___acrt_uninitialize_stdio 10019a20 f   libucrt:_file.obj
 0001:00018a6c       __lock_file                10019a6c f   libucrt:_file.obj
 0001:00018a80       __unlock_file              10019a80 f   libucrt:_file.obj
 0001:00018a94       __mbtowc_l                 10019a94 f   libucrt:mbtowc.obj
 0001:00018bd8       _mbtowc                    10019bd8 f   libucrt:mbtowc.obj
 0001:00018bf2       __fileno                   10019bf2 f   libucrt:fileno.obj
 0001:00018e05       ___acrt_LCMapStringA       10019e05 f   libucrt:lcmapstringa.obj
 0001:00018e50       __freea_crt                10019e50 f i libucrt:lcmapstringa.obj
 0001:00018e70       ___acrt_add_locale_ref     10019e70 f   libucrt:locale_refcounting.obj
 0001:00018eed       ___acrt_free_locale        10019eed f   libucrt:locale_refcounting.obj
 0001:00019037       ___acrt_locale_add_lc_time_reference 1001a037 f   libucrt:locale_refcounting.obj
 0001:00019060       ___acrt_locale_free_lc_time_if_unreferenced 1001a060 f   libucrt:locale_refcounting.obj
 0001:00019091       ___acrt_locale_release_lc_time_reference 1001a091 f   libucrt:locale_refcounting.obj
 0001:000190ba       ___acrt_release_locale_ref 1001a0ba f   libucrt:locale_refcounting.obj
 0001:0001913b       ___acrt_update_thread_locale_data 1001a13b f   libucrt:locale_refcounting.obj
 0001:000191b2       __updatetlocinfoEx_nolock  1001a1b2 f   libucrt:locale_refcounting.obj
 0001:00019202       ___acrt_locale_free_monetary 1001a202 f   libucrt:initmon.obj
 0001:00019300       ___acrt_locale_free_numeric 1001a300 f   libucrt:initnum.obj
 0001:000193a1       ___acrt_locale_free_time   1001a3a1 f   libucrt:inittime.obj
 0001:00019485       ___acrt_GetStringTypeA     1001a485 f   libucrt:getstringtypea.obj
 0001:0001958a       __query_new_mode           1001a58a f   libucrt:new_mode.obj
 0001:00019591       ___acrt_GetStringTypeW     1001a591 f   libucrt:getstringtypew.obj
 0001:000195f0       _qsort                     1001a5f0 f   libucrt:qsort.obj
 0001:00019ae7       _strncpy_s                 1001aae7 f   libucrt:strncpy_s.obj
 0001:00019b00       _strpbrk                   1001ab00 f   libucrt:strpbrk.obj
 0001:00019b40       __mbsdec                   1001ab40 f   libucrt:mbsdec.obj
 0001:00019b57       __mbsdec_l                 1001ab57 f   libucrt:mbsdec.obj
 0001:00019bf5       __msize_base               1001abf5 f   libucrt:msize.obj
 0001:00019c28       __realloc_base             1001ac28 f   libucrt:realloc_base.obj
 0001:00019c91       ___acrt_lowio_create_handle_array 1001ac91 f   libucrt:osfinfo.obj
 0001:00019d0e       ___acrt_lowio_destroy_handle_array 1001ad0e f   libucrt:osfinfo.obj
 0001:00019d43       ___acrt_lowio_ensure_fh_exists 1001ad43 f   libucrt:osfinfo.obj
 0001:00019dd7       ___acrt_lowio_lock_fh      1001add7 f   libucrt:osfinfo.obj
 0001:00019dfa       ___acrt_lowio_unlock_fh    1001adfa f   libucrt:osfinfo.obj
 0001:00019e1d       __free_osfhnd              1001ae1d f   libucrt:osfinfo.obj
 0001:00019eae       __get_osfhandle            1001aeae f   libucrt:osfinfo.obj
 0001:00019fcc       ___acrt_DownlevelLocaleNameToLCID 1001afcc f   libucrt:lcidtoname_downlevel.obj
 0001:0001a090       __commit                   1001b090 f   libucrt:commit.obj
 0001:0001a894       __write                    1001b894 f   libucrt:write.obj
 0001:0001a97c       __write_nolock             1001b97c f   libucrt:write.obj
 0001:0001ab60       __fcloseall                1001bb60 f   libucrt:closeall.obj
 0001:0001ac01       ___acrt_stdio_free_buffer_nolock 1001bc01 f   libucrt:_freebuf.obj
 0001:0001ac41       __isatty                   1001bc41 f   libucrt:isatty.obj
 0001:0001acc3       ?__mbrtowc_utf8@__crt_mbstring@@YAIPA_WPBDIPAU_Mbstatet@@@Z 1001bcc3 f   libucrt:mbrtowc.obj
 0001:0001ad05       ?__mbsrtowcs_utf8@__crt_mbstring@@YAIPA_WPAPBDIPAU_Mbstatet@@@Z 1001bd05 f   libucrt:mbrtowc.obj
 0001:0001ae02       ?return_illegal_sequence@__crt_mbstring@@YAIPAU_Mbstatet@@@Z 1001be02 f i libucrt:c32rtomb.obj
 0001:0001ae21       ___strncnt                 1001be21 f   libucrt:strncnt.obj
 0001:0001ae3d       __query_app_type           1001be3d f   libucrt:report_runtime_error.obj
 0001:0001aec1       __lseeki64_nolock          1001bec1 f   libucrt:lseek.obj
 0001:0001aedc       __putwch_nolock            1001bedc f   libucrt:putwch.obj
 0001:0001af10       __fclose_nolock            1001bf10 f   libucrt:fclose.obj
 0001:0001af87       _fclose                    1001bf87 f   libucrt:fclose.obj
 0001:0001b001       ?__mbrtoc32_utf8@__crt_mbstring@@YAIPA_UPBDIPAU_Mbstatet@@@Z 1001c001 f   libucrt:mbrtoc32.obj
 0001:0001b1c0       __CIlog10                  1001c1c0 f   libucrt:log10_impl.obj
 0001:0001b1fb       __CIlog10_default          1001c1fb f   libucrt:log10_impl.obj
 0001:0001b20f       __log10_default            1001c20f     libucrt:log10_impl.obj
 0001:0001b2d0       _ceil                      1001c2d0 f   libucrt:ceil_pentium4.obj
 0001:0001b310       __ceil_pentium4            1001c310 f   libucrt:ceil_pentium4.obj
 0001:0001b3f0       ___ascii_strnicmp          1001c3f0 f   libucrt:_strnicm.obj
 0001:0001b470       ___dcrt_lowio_ensure_console_output_initialized 1001c470 f   libucrt:initcon.obj
 0001:0001b48f       ___dcrt_terminate_console_output 1001c48f f   libucrt:initcon.obj
 0001:0001b4a6       ___dcrt_write_console      1001c4a6 f   libucrt:initcon.obj
 0001:0001b57d       __close                    1001c57d f   libucrt:close.obj
 0001:0001b60c       __close_nolock             1001c60c f   libucrt:close.obj
 0001:0001b6a8       ?__acrt_stdio_free_stream@@YAXV__crt_stdio_stream@@@Z 1001c6a8 f   libucrt:stream.obj
 0001:0001b6e3       ___acrt_initialize_sse2    1001c6e3 f   libucrt:mathfcns.obj
 0001:0001b700       __CIlog10_pentium4         1001c700 f   libucrt:log10_pentium4.obj
 0001:0001b718       __log10_pentium4           1001c718     libucrt:log10_pentium4.obj
 0001:0001b9b0       __fFEXP                    1001c9b0 f   libucrt:87tran.obj
 0001:0001ba07       __rtinfpopse               1001ca07     libucrt:87tran.obj
 0001:0001ba09       __rtinfnpopse              1001ca09     libucrt:87tran.obj
 0001:0001ba19       __fFLN                     1001ca19     libucrt:87tran.obj
 0001:0001bace       __rtinfpop                 1001cace     libucrt:87tran.obj
 0001:0001bad0       __rtinfnpop                1001cad0     libucrt:87tran.obj
 0001:0001bae0       __rtforexpinf              1001cae0 f   libucrt:87tran.obj
 0001:0001baed       __ffexpm1                  1001caed     libucrt:87tran.obj
 0001:0001bba0       __trandisp1                1001cba0 f   libucrt:87disp.obj
 0001:0001bc15       __trandisp2                1001cc15 f   libucrt:87disp.obj
 0001:0001bcaf       __rttospopde               1001ccaf     libucrt:87disp.obj
 0001:0001bcb4       __rttospop                 1001ccb4     libucrt:87disp.obj
 0001:0001bcc0       __rtnospop                 1001ccc0 f   libucrt:87disp.obj
 0001:0001bcd0       __rttosnpop                1001ccd0 f   libucrt:87disp.obj
 0001:0001bcd1       __rtnospopde               1001ccd1     libucrt:87disp.obj
 0001:0001bcd8       __rtzeropop                1001ccd8     libucrt:87disp.obj
 0001:0001bcda       __rtzeronpop               1001ccda     libucrt:87disp.obj
 0001:0001bce0       __rtzerospop               1001cce0 f   libucrt:87disp.obj
 0001:0001bced       __rtonepop                 1001cced     libucrt:87disp.obj
 0001:0001bcf0       __rtonenpop                1001ccf0 f   libucrt:87disp.obj
 0001:0001bd00       __tosnan1                  1001cd00 f   libucrt:87disp.obj
 0001:0001bd30       __nosnan2                  1001cd30 f   libucrt:87disp.obj
 0001:0001bd40       __tosnan2                  1001cd40 f   libucrt:87disp.obj
 0001:0001bd70       __nan2                     1001cd70 f   libucrt:87disp.obj
 0001:0001bdb0       __rtindfpop                1001cdb0 f   libucrt:87disp.obj
 0001:0001bdb2       __rtindfnpop               1001cdb2     libucrt:87disp.obj
 0001:0001bdc3       __rttosnpopde              1001cdc3     libucrt:87disp.obj
 0001:0001bdd0       __rtatan2inf               1001cdd0 f   libucrt:87disp.obj
 0001:0001bded       __rtchsifneg               1001cded     libucrt:87disp.obj
 0001:0001be00       __twoToTOS                 1001ce00 f   libucrt:common.obj
 0001:0001be15       __load_CW                  1001ce15 f   libucrt:common.obj
 0001:0001be2c       __convertTOStoQNaN         1001ce2c f   libucrt:common.obj
 0001:0001be45       __fload_withFB             1001ce45 f   libucrt:common.obj
 0001:0001be88       __checkTOS_withFB          1001ce88 f   libucrt:common.obj
 0001:0001be9e       __fast_exit                1001ce9e f   libucrt:common.obj
 0001:0001beab       __math_exit                1001ceab f   libucrt:common.obj
 0001:0001bed5       __check_overflow_exit      1001ced5 f   libucrt:common.obj
 0001:0001bee9       __check_range_exit         1001cee9 f   libucrt:common.obj
 0001:0001bf90       __startTwoArgErrorHandling 1001cf90 f   libucrt:genexcep.obj
 0001:0001bfa7       __startOneArgErrorHandling 1001cfa7 f   libucrt:genexcep.obj
 0001:0001bfe5       ___libm_error_support      1001cfe5 f   libucrt:libm_error.obj
 0001:0001c1db       __ceil_default             1001d1db f   libucrt:ceil.obj
 0001:0001c292       __clrfp                    1001d292 f   libucrt:fpctrl.obj
 0001:0001c2a5       __ctrlfp                   1001d2a5 f   libucrt:fpctrl.obj
 0001:0001c2d1       __set_statfp               1001d2d1 f   libucrt:fpctrl.obj
 0001:0001c32c       __statfp                   1001d32c f   libucrt:fpctrl.obj
 0001:0001c33e       __d_inttype                1001d33e f   libucrt:powhlp.obj
 0001:0001c3a8       __powhlp                   1001d3a8 f   libucrt:powhlp.obj
 0001:0001c4d3       __87except                 1001d4d3 f   libucrt:87except.obj
 0001:0001c5dd       __frnd                     1001d5dd f   libucrt:frnd.obj
 0001:0001c5f3       __errcode                  1001d5f3 f   libucrt:fpexcept.obj
 0001:0001c627       __except1                  1001d627 f   libucrt:fpexcept.obj
 0001:0001c6f5       __handle_exc               1001d6f5 f   libucrt:fpexcept.obj
 0001:0001c8e2       __raise_exc                1001d8e2 f   libucrt:fpexcept.obj
 0001:0001c905       __raise_exc_ex             1001d905 f   libucrt:fpexcept.obj
 0001:0001cbfb       __set_errno_from_matherr   1001dbfb f   libucrt:fpexcept.obj
 0001:0001cc2a       __umatherr                 1001dc2a f   libucrt:fpexcept.obj
 0001:0001cccc       __decomp                   1001dccc f   libucrt:util.obj
 0001:0001cdaa       __set_exp                  1001ddaa f   libucrt:util.obj
 0001:0001cdd9       __sptype                   1001ddd9 f   libucrt:util.obj
 0001:0001ce37       __fpclass                  1001de37 f   libucrt:ieeemisc.obj
 0001:0001cedb       _IsProcessorFeaturePresent@4 1001dedb f   kernel32:KERNEL32.dll
 0001:0001cef0       __FindPESection            1001def0 f   LIBCMT:pesect.obj
 0001:0001cf40       __IsNonwritableInCurrentImage 1001df40 f   LIBCMT:pesect.obj
 0001:0001d000       __ValidateImageBase        1001e000 f   LIBCMT:pesect.obj
 0001:0001d040       __aulldvrm                 1001e040 f   LIBCMT:ulldvrm.obj
 0001:0001d0e0       __alldvrm                  1001e0e0 f   LIBCMT:lldvrm.obj
 0001:0001d1c0       __aullshr                  1001e1c0 f   LIBCMT:ullshr.obj
 0001:0001d1e0       __alloca_probe_16          1001e1e0 f   LIBCMT:alloca16.obj
 0001:0001d1f6       __alloca_probe_8           1001e1f6     LIBCMT:alloca16.obj
 0001:0001d210       __allshl                   1001e210 f   LIBCMT:llshl.obj
 0001:0001d230       __ftol2_sse                1001e230 f   LIBCMT:ftol2.obj
 0001:0001d239       __ftol2_pentium4           1001e239 f   LIBCMT:ftol2.obj
 0001:0001d24c       __ftol2_sse_excpt          1001e24c f   LIBCMT:ftol2.obj
 0001:0001d270       __ftol2                    1001e270 f   LIBCMT:ftol2.obj
 0001:0001d2f0       _strchr                    1001e2f0 f   libvcruntime:strchr.obj
 0001:0001d35e       ___from_strstr_to_strchr   1001e35e     libvcruntime:strchr.obj
 0001:0001d420       _strrchr                   1001e420 f   libvcruntime:strrchr.obj
 0001:0001d61c       __TI2?AVbad_alloc@std@@    1001e61c     LIBCMT:throw_bad_alloc.obj
 0001:0001d62c       __CTA2?AVbad_alloc@std@@   1001e62c     LIBCMT:throw_bad_alloc.obj
 0001:0001d638       __CT??_R0?AVbad_alloc@std@@@8??0bad_alloc@std@@QAE@ABV01@@Z12 1001e638     LIBCMT:throw_bad_alloc.obj
 0001:0001d654       __CT??_R0?AVexception@std@@@8??0exception@std@@QAE@ABV01@@Z12 1001e654     LIBCMT:throw_bad_alloc.obj
 0001:0001d670       __TI3?AVbad_array_new_length@std@@ 1001e670     LIBCMT:throw_bad_alloc.obj
 0001:0001d680       __CTA3?AVbad_array_new_length@std@@ 1001e680     LIBCMT:throw_bad_alloc.obj
 0001:0001d690       __CT??_R0?AVbad_array_new_length@std@@@8??0bad_array_new_length@std@@QAE@ABV01@@Z12 1001e690     LIBCMT:throw_bad_alloc.obj
 0002:00000000       ?DescIDs@@3PAHA            1001f000     Pclass.obj
 0002:00000080       ?Counters@@3PAU_Counters@@A 1001f080     perfthread.obj
 0002:00000188       ?pNtQueryInformationProcess@@3P6GJPAXW4_PROCESSINFOCLASS@@0KPAK@ZA 1001f188     Proclist.obj
 0002:0000018c       ?pNtQueryInformationThread@@3P6GJPAXK0KPAK@ZA 1001f18c     Proclist.obj
 0002:00000190       ?pNtQueryObject@@3P6GJPAXK0K0@ZA 1001f190     Proclist.obj
 0002:00000194       ?pNtQuerySystemInformation@@3P6GJKPAXKPAK@ZA 1001f194     Proclist.obj
 0002:00000198       ?pNtQueryInformationFile@@3P6GJPAX00KK@ZA 1001f198     Proclist.obj
 0002:0000019c       ?pIsValidSid@@3P6GHPAX@ZA  1001f19c     Proclist.obj
 0002:000001a0       ?pGetSidIdentifierAuthority@@3P6GPAU_SID_IDENTIFIER_AUTHORITY@@PAX@ZA 1001f1a0     Proclist.obj
 0002:000001a4       ?pGetSidSubAuthorityCount@@3P6GPAEPAX@ZA 1001f1a4     Proclist.obj
 0002:000001a8       ?pGetSidSubAuthority@@3P6GPAKPAXK@ZA 1001f1a8     Proclist.obj
 0002:000001ac       ?pLookupAccountName@@3P6GHPB_W0PAXPAKPA_W2PAW4_SID_NAME_USE@@@ZA 1001f1ac     Proclist.obj
 0002:000001b0       ?pIsWow64Process@@3P6GHPAXPAH@ZA 1001f1b0     Proclist.obj
 0002:000001b4       ?pGetGuiResources@@3P6GKPAXK@ZA 1001f1b4     Proclist.obj
 0002:000001b8       ?pCoSetProxyBlanket@@3P6GJPAUIUnknown@@KKPA_WKKPAXK@ZA 1001f1b8     Proclist.obj
 0002:000001c0       ___scrt_native_dllmain_reason 1001f1c0     LIBCMT:utility.obj
 0002:000001c4       ___isa_enabled             1001f1c4     LIBCMT:cpu_disp.obj
 0002:000001d0       ___security_cookie_complement 1001f1d0     LIBCMT:gs_cookie.obj
 0002:000001d4       ___security_cookie         1001f1d4     LIBCMT:gs_cookie.obj
 0002:000001f0       __NLG_Destination          1001f1f0     libvcruntime:exsup.obj
 0002:00000200       ___abort_behavior          1001f200     libucrt:abort.obj
 0002:00000228       ___acrt_initial_locale_data 1001f228     libucrt:nlsdata.obj
 0002:000002e0       ___acrt_initial_locale_pointers 1001f2e0     libucrt:nlsdata.obj
 0002:000002e8       ___acrt_wide_c_locale_string 1001f2e8     libucrt:nlsdata.obj
 0002:000002ec       __pwctype                  1001f2ec     libucrt:ctype.obj
 0002:000002f0       ___acrt_initial_multibyte_data 1001f2f0     libucrt:mbctype.obj
 0002:00000810       __iob                      1001f810     libucrt:_file.obj
 0002:000008b8       ___globallocalestatus      1001f8b8     libucrt:glstatus.obj
 0002:000008c0       ___acrt_lconv_c            1001f8c0     libucrt:localeconv.obj
 0002:00000910       ___acrt_lconv_static_decimal 1001f910     libucrt:localeconv.obj
 0002:00000914       ___acrt_lconv_static_W_decimal 1001f914     libucrt:localeconv.obj
 0002:00000920       __lookuptrailbytes         1001f920     libucrt:read.obj
 0002:00000a30       __fltused                  1001fa30     LIBCMT:fltused.obj
 0002:00000a40       ??_R0?AVbad_alloc@std@@@8  1001fa40     LIBCMT:throw_bad_alloc.obj
 0002:00000a5c       ??_R0?AVexception@std@@@8  1001fa5c     LIBCMT:throw_bad_alloc.obj
 0002:00000a78       ??_R0?AVbad_array_new_length@std@@@8 1001fa78     LIBCMT:throw_bad_alloc.obj
 0002:00000aa0       ??_R0?AVtype_info@@@8      1001faa0     LIBCMT:std_type_info_static.obj
 0002:00000ab8       ?FPRINTFbuffer@@3PA_WA     1001fab8     fileio.obj
 0002:00020cc0       ?bInit@Plist@@2_NA         1003fcc0     Pclass.obj
 0002:00020cc8       ?PanelModesLocal@Plist@@2PAUPanelMode@@A 1003fcc8     Pclass.obj
 0002:00020e08       ?PanelModesRemote@Plist@@2PAUPanelMode@@A 1003fe08     Pclass.obj
 0002:00020f48       ?ProcPanelModesLocal@Plist@@2PAY0FA@_WA 1003ff48     Pclass.obj
 0002:00021588       ?ProcPanelModesRemote@Plist@@2PAY0FA@_WA 10040588     Pclass.obj
 0002:00021bc8       ?PanelModeBuffer@Plist@@2PA_WA 10040bc8     Pclass.obj
 0002:000258c8       ?hDebugToken@DebugToken@@0RAXA 100448c8     Plist.obj
 0002:00025920       ?Info@@3UPluginStartupInfo@@A 10044920     Proclist.obj
 0002:000259a8       ?FSF@@3UFarStandardFunctions@@A 100449a8     Proclist.obj
 0002:00025a6c       ?Opt@@3U_Opt@@A            10044a6c     Proclist.obj
 0002:00025a90       ?_ui64Table@@3PAVui64Table@@A 10044a90     Proclist.obj
 0002:00025a94       ?PluginRootKey@@3PA_WA     10044a94     Proclist.obj
 0002:00025aa8       ?Ptr@?1???R<lambda_1af49d8e19f959e583a46d83b89ae789>@@QBE@XZ@4PAXA 10044aa8     vc_crt_fix_impl.obj
 0002:00025b40       ___scrt_current_native_startup_state 10044b40     LIBCMT:utility.obj
 0002:00025b44       ___scrt_native_startup_lock 10044b44     LIBCMT:utility.obj
 0002:00025b68       ___isa_available           10044b68     LIBCMT:cpu_disp.obj
 0002:00025b6c       ___favor                   10044b6c     LIBCMT:cpu_disp.obj
 0002:00025b70       ___scrt_debugger_hook_flag 10044b70     LIBCMT:utility_desktop.obj
 0002:00025b78       ?__type_info_root_node@@3U__type_info_node@@A 10044b78     LIBCMT:tncleanup.obj
 0002:00025b80       ?_OptionsStorage@?1??__local_stdio_printf_options@@9@4_KA 10044b80     LIBCMT:default_local_stdio_options.obj
 0002:00025b88       ?_OptionsStorage@?1??__local_stdio_scanf_options@@9@4_KA 10044b88     LIBCMT:default_local_stdio_options.obj
 0002:00025f10       ___pPurecall               10044f10     libvcruntime:purevirt_data.obj
 0002:00025f14       ?pArgList@UnDecorator@@0PAVReplicator@@A 10044f14     libvcruntime:undname.obj
 0002:00025f18       ?pZNameList@UnDecorator@@0PAVReplicator@@A 10044f18     libvcruntime:undname.obj
 0002:00025f1c       ?pTemplateArgList@UnDecorator@@0PAVReplicator@@A 10044f1c     libvcruntime:undname.obj
 0002:00025f20       ?gName@UnDecorator@@0PBDB  10044f20     libvcruntime:undname.obj
 0002:00025f24       ?name@UnDecorator@@0PBDB   10044f24     libvcruntime:undname.obj
 0002:00025f28       ?disableFlags@UnDecorator@@0KA 10044f28     libvcruntime:undname.obj
 0002:00025f2c       ?fExplicitTemplateParams@UnDecorator@@0_NA 10044f2c     libvcruntime:undname.obj
 0002:00025f2d       ?fGetTemplateArgumentList@UnDecorator@@0_NA 10044f2d     libvcruntime:undname.obj
 0002:00025f30       ?m_pGetParameter@UnDecorator@@0P6APADJ@ZA 10044f30     libvcruntime:undname.obj
 0002:00025f34       ?m_CHPENameOffset@UnDecorator@@0KA 10044f34     libvcruntime:undname.obj
 0002:00025f38       ?m_recursionLevel@UnDecorator@@0KA 10044f38     libvcruntime:undname.obj
 0002:00025f50       ?__WinRTOutOfMemoryExceptionCallback@@3P6GPAXXZA 10044f50     libvcruntime:ehhelpers.obj
 0002:00025f60       ?c_exit_complete@?1???R<lambda_6e4b09c48022b2350581041d5f6b0c4c>@@QBE@XZ@4_NA 10044f60     libucrt:exit.obj
 0002:00026070       __environ_table            10045070     libucrt:environment_initialization.obj
 0002:00026074       __wenviron_table           10045074     libucrt:environment_initialization.obj
 0002:00026078       ___dcrt_initial_wide_environment 10045078     libucrt:environment_initialization.obj
 0002:0002607c       ___dcrt_initial_narrow_environment 1004507c     libucrt:environment_initialization.obj
 0002:00026080       ___acrt_atexit_table       10045080     libucrt:onexit.obj
 0002:0002608c       ___acrt_at_quick_exit_table 1004508c     libucrt:onexit.obj
 0002:0002609c       ___acrt_locale_changed_data 1004509c     libucrt:wsetlocale.obj
 0002:000260a0       ___acrt_current_locale_data 100450a0     libucrt:nlsdata.obj
 0002:000261fc       ___acrt_current_multibyte_data 100451fc     libucrt:mbctype.obj
 0002:00026200       __mbctype                  10045200     libucrt:mbctype.obj
 0002:00026204       __mbcasemap                10045204     libucrt:mbctype.obj
 0002:00026210       __pgmptr                   10045210     libucrt:argv_data.obj
 0002:00026214       ___argc                    10045214     libucrt:argv_data.obj
 0002:00026218       ___argv                    10045218     libucrt:argv_data.obj
 0002:0002621c       ___wargv                   1004521c     libucrt:argv_data.obj
 0002:00026220       __acmdln                   10045220     libucrt:argv_data.obj
 0002:00026224       __wcmdln                   10045224     libucrt:argv_data.obj
 0002:00026228       ___pioinfo                 10045228     libucrt:ioinit.obj
 0002:00026428       __nhandle                  10045428     libucrt:ioinit.obj
 0002:00026508       ___acrt_heap               10045508     libucrt:heap_handle.obj
 0002:00026520       __nstream                  10045520     libucrt:_file.obj
 0002:00026524       ___piob                    10045524     libucrt:_file.obj
 0002:00026528       ___acrt_stdout_buffer      10045528     libucrt:_sftbuf.obj
 0002:0002652c       ___acrt_stderr_buffer      1004552c     libucrt:_sftbuf.obj
 0002:00026538       ___acrt_lconv_static_null  10045538     libucrt:localeconv.obj
 0002:0002653c       ___acrt_lconv_static_W_null 1004553c     libucrt:localeconv.obj
 0002:00026550       ___fastflag                10045550     libucrt:fp_flags.obj
 0002:00026558       ___dyn_tls_init_callback   10045558     <common>
 0002:0002655c       ___scrt_ucrt_dll_is_in_use 1004555c     <common>
 0002:00026560       __pmatherr                 10045560     <common>
 0002:00026564       ___use_sse2_mathfcns       10045564     <common>
 0003:00000000       __imp__OpenThreadToken@16  10046000     advapi32:ADVAPI32.dll
 0003:00000004       __imp__LookupPrivilegeValueW@12 10046004     advapi32:ADVAPI32.dll
 0003:00000008       __imp__DuplicateTokenEx@24 10046008     advapi32:ADVAPI32.dll
 0003:0000000c       __imp__AdjustTokenPrivileges@24 1004600c     advapi32:ADVAPI32.dll
 0003:00000010       __imp__OpenProcessToken@12 10046010     advapi32:ADVAPI32.dll
 0003:00000014       __imp__SetThreadToken@8    10046014     advapi32:ADVAPI32.dll
 0003:00000018       __imp__RegQueryValueExW@24 10046018     advapi32:ADVAPI32.dll
 0003:0000001c       __imp__RegOpenKeyExW@20    1004601c     advapi32:ADVAPI32.dll
 0003:00000020       __imp__RegConnectRegistryW@12 10046020     advapi32:ADVAPI32.dll
 0003:00000024       __imp__RegCloseKey@4       10046024     advapi32:ADVAPI32.dll
 0003:00000028       __imp__GetUserNameW@8      10046028     advapi32:ADVAPI32.dll
 0003:0000002c       \177ADVAPI32_NULL_THUNK_DATA 1004602c     advapi32:ADVAPI32.dll
 0003:00000030       __imp__VirtualFree@12      10046030     kernel32:KERNEL32.dll
 0003:00000034       __imp__lstrcpynW@12        10046034     kernel32:KERNEL32.dll
 0003:00000038       __imp__lstrlenW@4          10046038     kernel32:KERNEL32.dll
 0003:0000003c       __imp__CreateFileW@28      1004603c     kernel32:KERNEL32.dll
 0003:00000040       __imp__SetEvent@4          10046040     kernel32:KERNEL32.dll
 0003:00000044       __imp__GetCurrentThreadId@0 10046044     kernel32:KERNEL32.dll
 0003:00000048       __imp__SetPriorityClass@8  10046048     kernel32:KERNEL32.dll
 0003:0000004c       __imp__GetPriorityClass@4  1004604c     kernel32:KERNEL32.dll
 0003:00000050       __imp__GetSystemTimeAsFileTime@4 10046050     kernel32:KERNEL32.dll
 0003:00000054       __imp__GetLocalTime@4      10046054     kernel32:KERNEL32.dll
 0003:00000058       __imp__GetTickCount@0      10046058     kernel32:KERNEL32.dll
 0003:0000005c       __imp__lstrcmpW@8          1004605c     kernel32:KERNEL32.dll
 0003:00000060       __imp__lstrcmpiW@8         10046060     kernel32:KERNEL32.dll
 0003:00000064       __imp__lstrcpyW@8          10046064     kernel32:KERNEL32.dll
 0003:00000068       __imp__lstrcatW@8          10046068     kernel32:KERNEL32.dll
 0003:0000006c       __imp__SystemTimeToTzSpecificLocalTime@12 1004606c     kernel32:KERNEL32.dll
 0003:00000070       __imp__FileTimeToSystemTime@8 10046070     kernel32:KERNEL32.dll
 0003:00000074       __imp__ResetEvent@4        10046074     kernel32:KERNEL32.dll
 0003:00000078       __imp__CreateMutexW@12     10046078     kernel32:KERNEL32.dll
 0003:0000007c       __imp__CreateEventW@16     1004607c     kernel32:KERNEL32.dll
 0003:00000080       __imp__WaitForMultipleObjects@16 10046080     kernel32:KERNEL32.dll
 0003:00000084       __imp__GetProcessTimes@20  10046084     kernel32:KERNEL32.dll
 0003:00000088       __imp__GetLastError@0      10046088     kernel32:KERNEL32.dll
 0003:0000008c       __imp__TerminateProcess@8  1004608c     kernel32:KERNEL32.dll
 0003:00000090       __imp__GetCurrentThread@0  10046090     kernel32:KERNEL32.dll
 0003:00000094       __imp__OpenProcess@12      10046094     kernel32:KERNEL32.dll
 0003:00000098       __imp__ReadProcessMemory@20 10046098     kernel32:KERNEL32.dll
 0003:0000009c       __imp__FileTimeToLocalFileTime@8 1004609c     kernel32:KERNEL32.dll
 0003:000000a0       __imp__VirtualAlloc@16     100460a0     kernel32:KERNEL32.dll
 0003:000000a4       __imp__LocalFree@4         100460a4     kernel32:KERNEL32.dll
 0003:000000a8       __imp__FormatMessageW@28   100460a8     kernel32:KERNEL32.dll
 0003:000000ac       __imp__GetDateFormatW@24   100460ac     kernel32:KERNEL32.dll
 0003:000000b0       __imp__GetTimeFormatW@24   100460b0     kernel32:KERNEL32.dll
 0003:000000b4       __imp__GetProcAddress@8    100460b4     kernel32:KERNEL32.dll
 0003:000000b8       __imp__InitializeCriticalSection@4 100460b8     kernel32:KERNEL32.dll
 0003:000000bc       __imp__EnterCriticalSection@4 100460bc     kernel32:KERNEL32.dll
 0003:000000c0       __imp__LeaveCriticalSection@4 100460c0     kernel32:KERNEL32.dll
 0003:000000c4       __imp__DeleteCriticalSection@4 100460c4     kernel32:KERNEL32.dll
 0003:000000c8       __imp__GetThreadTimes@20   100460c8     kernel32:KERNEL32.dll
 0003:000000cc       __imp__VirtualQuery@12     100460cc     kernel32:KERNEL32.dll
 0003:000000d0       __imp__GetModuleFileNameW@12 100460d0     kernel32:KERNEL32.dll
 0003:000000d4       __imp__LoadLibraryW@4      100460d4     kernel32:KERNEL32.dll
 0003:000000d8       __imp__SetFilePointerEx@20 100460d8     kernel32:KERNEL32.dll
 0003:000000dc       __imp__GetConsoleMode@8    100460dc     kernel32:KERNEL32.dll
 0003:000000e0       __imp__GetConsoleCP@0      100460e0     kernel32:KERNEL32.dll
 0003:000000e4       __imp__FlushFileBuffers@4  100460e4     kernel32:KERNEL32.dll
 0003:000000e8       __imp__SetStdHandle@8      100460e8     kernel32:KERNEL32.dll
 0003:000000ec       __imp__HeapReAlloc@16      100460ec     kernel32:KERNEL32.dll
 0003:000000f0       __imp__HeapSize@12         100460f0     kernel32:KERNEL32.dll
 0003:000000f4       __imp__GetStringTypeW@16   100460f4     kernel32:KERNEL32.dll
 0003:000000f8       __imp__GetProcessHeap@0    100460f8     kernel32:KERNEL32.dll
 0003:000000fc       __imp__TerminateThread@8   100460fc     kernel32:KERNEL32.dll
 0003:00000100       __imp__CreateThread@24     10046100     kernel32:KERNEL32.dll
 0003:00000104       __imp__GetCurrentProcessId@0 10046104     kernel32:KERNEL32.dll
 0003:00000108       __imp__GetCurrentProcess@0 10046108     kernel32:KERNEL32.dll
 0003:0000010c       __imp__Sleep@4             1004610c     kernel32:KERNEL32.dll
 0003:00000110       __imp__WaitForSingleObject@8 10046110     kernel32:KERNEL32.dll
 0003:00000114       __imp__ReleaseMutex@4      10046114     kernel32:KERNEL32.dll
 0003:00000118       __imp__WriteFile@20        10046118     kernel32:KERNEL32.dll
 0003:0000011c       __imp__SetLastError@4      1004611c     kernel32:KERNEL32.dll
 0003:00000120       __imp__DuplicateHandle@28  10046120     kernel32:KERNEL32.dll
 0003:00000124       __imp__CloseHandle@4       10046124     kernel32:KERNEL32.dll
 0003:00000128       __imp__GetModuleHandleW@4  10046128     kernel32:KERNEL32.dll
 0003:0000012c       __imp__LCMapStringW@24     1004612c     kernel32:KERNEL32.dll
 0003:00000130       __imp__GetFileType@4       10046130     kernel32:KERNEL32.dll
 0003:00000134       __imp__GetStdHandle@4      10046134     kernel32:KERNEL32.dll
 0003:00000138       __imp__FreeEnvironmentStringsW@4 10046138     kernel32:KERNEL32.dll
 0003:0000013c       __imp__GetEnvironmentStringsW@0 1004613c     kernel32:KERNEL32.dll
 0003:00000140       __imp__WideCharToMultiByte@32 10046140     kernel32:KERNEL32.dll
 0003:00000144       __imp__MultiByteToWideChar@24 10046144     kernel32:KERNEL32.dll
 0003:00000148       __imp__GetCommandLineW@0   10046148     kernel32:KERNEL32.dll
 0003:0000014c       __imp__GetCommandLineA@0   1004614c     kernel32:KERNEL32.dll
 0003:00000150       __imp__IsProcessorFeaturePresent@4 10046150     kernel32:KERNEL32.dll
 0003:00000154       __imp__IsDebuggerPresent@0 10046154     kernel32:KERNEL32.dll
 0003:00000158       __imp__UnhandledExceptionFilter@4 10046158     kernel32:KERNEL32.dll
 0003:0000015c       __imp__SetUnhandledExceptionFilter@4 1004615c     kernel32:KERNEL32.dll
 0003:00000160       __imp__GetStartupInfoW@4   10046160     kernel32:KERNEL32.dll
 0003:00000164       __imp__QueryPerformanceCounter@4 10046164     kernel32:KERNEL32.dll
 0003:00000168       __imp__RaiseException@16   10046168     kernel32:KERNEL32.dll
 0003:0000016c       __imp__InitializeCriticalSectionAndSpinCount@8 1004616c     kernel32:KERNEL32.dll
 0003:00000170       __imp__TlsAlloc@0          10046170     kernel32:KERNEL32.dll
 0003:00000174       __imp__TlsGetValue@4       10046174     kernel32:KERNEL32.dll
 0003:00000178       __imp__TlsSetValue@8       10046178     kernel32:KERNEL32.dll
 0003:0000017c       __imp__TlsFree@4           1004617c     kernel32:KERNEL32.dll
 0003:00000180       __imp__FreeLibrary@4       10046180     kernel32:KERNEL32.dll
 0003:00000184       __imp__LoadLibraryExW@12   10046184     kernel32:KERNEL32.dll
 0003:00000188       __imp__RtlUnwind@16        10046188     kernel32:KERNEL32.dll
 0003:0000018c       __imp__ExitProcess@4       1004618c     kernel32:KERNEL32.dll
 0003:00000190       __imp__HeapFree@12         10046190     kernel32:KERNEL32.dll
 0003:00000194       __imp__HeapAlloc@12        10046194     kernel32:KERNEL32.dll
 0003:00000198       __imp__FindClose@4         10046198     kernel32:KERNEL32.dll
 0003:0000019c       __imp__FindFirstFileExW@24 1004619c     kernel32:KERNEL32.dll
 0003:000001a0       __imp__FindNextFileW@8     100461a0     kernel32:KERNEL32.dll
 0003:000001a4       __imp__IsValidCodePage@4   100461a4     kernel32:KERNEL32.dll
 0003:000001a8       __imp__GetACP@0            100461a8     kernel32:KERNEL32.dll
 0003:000001ac       __imp__GetOEMCP@0          100461ac     kernel32:KERNEL32.dll
 0003:000001b0       __imp__GetCPInfo@8         100461b0     kernel32:KERNEL32.dll
 0003:000001b4       __imp__WriteConsoleW@20    100461b4     kernel32:KERNEL32.dll
 0003:000001b8       \177KERNEL32_NULL_THUNK_DATA 100461b8     kernel32:KERNEL32.dll
 0003:000001bc       __imp__WNetAddConnection2W@16 100461bc     mpr:MPR.dll
 0003:000001c0       __imp__WNetCancelConnection2W@12 100461c0     mpr:MPR.dll
 0003:000001c4       \177MPR_NULL_THUNK_DATA    100461c4     mpr:MPR.dll
 0003:000001c8       __imp__VariantClear@4      100461c8     oleaut32:OLEAUT32.dll
 0003:000001cc       __imp__SysAllocString@4    100461cc     oleaut32:OLEAUT32.dll
 0003:000001d0       __imp__SysFreeString@4     100461d0     oleaut32:OLEAUT32.dll
 0003:000001d4       \177OLEAUT32_NULL_THUNK_DATA 100461d4     oleaut32:OLEAUT32.dll
 0003:000001d8       __imp__GetParent@4         100461d8     user32:USER32.dll
 0003:000001dc       __imp__wsprintfW           100461dc     user32:USER32.dll
 0003:000001e0       __imp__ShowWindowAsync@8   100461e0     user32:USER32.dll
 0003:000001e4       __imp__GetWindowPlacement@8 100461e4     user32:USER32.dll
 0003:000001e8       __imp__IsWindowVisible@4   100461e8     user32:USER32.dll
 0003:000001ec       __imp__IsIconic@4          100461ec     user32:USER32.dll
 0003:000001f0       __imp__SetForegroundWindow@4 100461f0     user32:USER32.dll
 0003:000001f4       __imp__SystemParametersInfoW@16 100461f4     user32:USER32.dll
 0003:000001f8       __imp__GetWindowThreadProcessId@8 100461f8     user32:USER32.dll
 0003:000001fc       __imp__EnumWindows@8       100461fc     user32:USER32.dll
 0003:00000200       __imp__GetWindowLongW@8    10046200     user32:USER32.dll
 0003:00000204       __imp__GetWindowTextW@12   10046204     user32:USER32.dll
 0003:00000208       \177USER32_NULL_THUNK_DATA 10046208     user32:USER32.dll
 0003:0000020c       __imp__GetFileVersionInfoSizeW@8 1004620c     version:VERSION.dll
 0003:00000210       __imp__GetFileVersionInfoW@16 10046210     version:VERSION.dll
 0003:00000214       __imp__VerQueryValueW@16   10046214     version:VERSION.dll
 0003:00000218       \177VERSION_NULL_THUNK_DATA 10046218     version:VERSION.dll
 0003:0000021c       __imp__CoCreateInstance@20 1004621c     ole32:ole32.dll
 0003:00000220       __imp__CoInitialize@4      10046220     ole32:ole32.dll
 0003:00000224       __imp__CoUninitialize@0    10046224     ole32:ole32.dll
 0003:00000228       \177ole32_NULL_THUNK_DATA  10046228     ole32:ole32.dll
 0003:0000022c       ___guard_check_icall_fptr  1004622c     LIBCMT:guard_support.obj
 0003:00000230       __IMPORT_DESCRIPTOR_KERNEL32 10046230     kernel32:KERNEL32.dll
 0003:00000244       __IMPORT_DESCRIPTOR_USER32 10046244     user32:USER32.dll
 0003:00000258       __IMPORT_DESCRIPTOR_ADVAPI32 10046258     advapi32:ADVAPI32.dll
 0003:0000026c       __IMPORT_DESCRIPTOR_ole32  1004626c     ole32:ole32.dll
 0003:00000280       __IMPORT_DESCRIPTOR_MPR    10046280     mpr:MPR.dll
 0003:00000294       __IMPORT_DESCRIPTOR_VERSION 10046294     version:VERSION.dll
 0003:000002a8       __IMPORT_DESCRIPTOR_OLEAUT32 100462a8     oleaut32:OLEAUT32.dll
 0003:000002bc       __NULL_IMPORT_DESCRIPTOR   100462bc     kernel32:KERNEL32.dll

 entry point at        0001:00011bf8

 Static symbols

 0001:00000040       ?constStrTypes@@3QBQB_WB   10001040     handles.obj
 0001:000005b0       ?StatusWidth@?1??InitializePanelModes@Plist@@SAXXZ@4QB_WB 100015b0     Pclass.obj
 0001:000005c0       ?StatusCols@?1??InitializePanelModes@Plist@@SAXXZ@4QB_WB 100015c0     Pclass.obj
 0001:000005d0       ?DefaultModes@?1??InitializePanelModes@Plist@@SAXXZ@4QBU<unnamed-type-DefaultModes>@?1??12@SAXXZ@B 100015d0     Pclass.obj
 0001:00000848       ?DefaultModesRemote@?1??InitializePanelModes@Plist@@SAXXZ@4QBU<unnamed-type-DefaultModesRemote>@?1??12@SAXXZ@B 10001848     Pclass.obj
 0001:000009b8       ?invalid_chars@?1??GetFiles@Plist@@QAEHPAUPluginPanelItem@@HHPAPB_W_KAAU_Opt@@@Z@4QB_WB 100019b8     Pclass.obj
 0001:000009d0       ?Styles@?IN@??GetFiles@Plist@@QAEHPAUPluginPanelItem@@HHPAPB_W_KAAU_Opt@@@Z@4QBIB 100019d0     Pclass.obj
 0001:00000a10       ?StrStyles@?IN@??GetFiles@Plist@@QAEHPAUPluginPanelItem@@HHPAPB_W_KAAU_Opt@@@Z@4QBQB_WB 10001a10     Pclass.obj
 0001:00000be8       ?ExtStyles@?IN@??GetFiles@Plist@@QAEHPAUPluginPanelItem@@HHPAPB_W_KAAU_Opt@@@Z@4QBHB 10001be8     Pclass.obj
 0001:00000c38       ?StrExtStyles@?IN@??GetFiles@Plist@@QAEHPAUPluginPanelItem@@HHPAPB_W_KAAU_Opt@@@Z@4QBQB_WB 10001c38     Pclass.obj
 0001:0000107c       ?PrClasses@?EO@??ProcessKey@Plist@@QAEHPBU_INPUT_RECORD@@@Z@4QBGB 1000207c     Pclass.obj
 0001:00001088       ?Pr@?HO@??ProcessKey@Plist@@QAEHPBU_INPUT_RECORD@@@Z@4QBEB 10002088     Pclass.obj
 0001:00001140       ?MonthDays@?O@??FileTimeToText@Plist@@AAEXPAU_FILETIME@@0PA_W@Z@4QBHB 10002140     Pclass.obj
 0001:000011bc       ?WSFI@?1??GetVersionInfo@Plist@@SA_NPA_WAAPAEAAPA_W2@Z@4QB_WB 100021bc     Pclass.obj
 0001:00001b84       ?kernel32@modules@@3QB_WB  10002b84     vc_crt_fix_impl.obj
 0001:00001b98       ?ntdll@modules@@3QB_WB     10002b98     vc_crt_fix_impl.obj
 0001:00001d3c       _GS_ExceptionPointers      10002d3c     LIBCMT:gs_report.obj
 0001:00001d44       ?ExceptionTemplate@?1??_CxxThrowException@@9@8@4UEHExceptionRecord@@B 10002d44     libvcruntime:throw.obj
 0001:00001d64       ?module_names@?A0x5c520fe1@@3QBQB_WB 10002d64     libvcruntime:winapi_downlevel.obj
 0001:00001e08       ?candidate_modules@?1??try_get_FlsAlloc@@YAP6GKP6GXPAX@Z@ZXZ@4QBW4module_id@?A0x5c520fe1@@B 10002e08     libvcruntime:winapi_downlevel.obj
 0001:00001e1c       ?candidate_modules@?1??try_get_FlsFree@@YAP6GHK@ZXZ@4QBW4module_id@?A0x5c520fe1@@B 10002e1c     libvcruntime:winapi_downlevel.obj
 0001:00001e2c       ?candidate_modules@?1??try_get_FlsGetValue@@YAP6GPAXK@ZXZ@4QBW4module_id@?A0x5c520fe1@@B 10002e2c     libvcruntime:winapi_downlevel.obj
 0001:00001e40       ?candidate_modules@?1??try_get_FlsSetValue@@YAP6GHKPAX@ZXZ@4QBW4module_id@?A0x5c520fe1@@B 10002e40     libvcruntime:winapi_downlevel.obj
 0001:00001e54       ?candidate_modules@?1??try_get_InitializeCriticalSectionEx@@YAP6GHPAU_RTL_CRITICAL_SECTION@@KK@ZXZ@4QBW4module_id@?A0x5c520fe1@@B 10002e54     libvcruntime:winapi_downlevel.obj
 0001:00001e78       ?tokenTable@@3QBQBDB       10002e78     libvcruntime:undname.obj
 0001:00001eb8       ?nameTable@@3QBQBDB        10002eb8     libvcruntime:undname.obj
 0001:00002000       ?rttiTable@@3QBQBDB        10003000     libvcruntime:undname.obj
 0001:000026e0       ___acrt_initializers       100036e0     libucrt:initialization.obj
 0001:00002760       ?errtable@@3QBUerrentry@?A0x31fdb9ec@@B 10003760     libucrt:errno.obj
 0001:0000358c       ?_mb_locale_names@@3QBQB_WB 1000458c     libucrt:mbctype.obj
 0001:000035d0       ?module_names@?A0x391cf84c@@3QBQB_WB 100045d0     libucrt:winapi_thunks.obj
 0001:00003af0       ?candidate_modules@?1??try_get_AreFileApisANSI@@YAP6GHXZXZ@4QBW4module_id@?A0x391cf84c@@B 10004af0     libucrt:winapi_thunks.obj
 0001:00003b04       ?candidate_modules@?1??try_get_FlsAlloc@@YAP6GKP6GXPAX@Z@ZXZ@4QBW4module_id@?A0x391cf84c@@B 10004b04     libucrt:winapi_thunks.obj
 0001:00003b18       ?candidate_modules@?1??try_get_FlsFree@@YAP6GHK@ZXZ@4QBW4module_id@?A0x391cf84c@@B 10004b18     libucrt:winapi_thunks.obj
 0001:00003b28       ?candidate_modules@?1??try_get_FlsGetValue@@YAP6GPAXK@ZXZ@4QBW4module_id@?A0x391cf84c@@B 10004b28     libucrt:winapi_thunks.obj
 0001:00003b3c       ?candidate_modules@?1??try_get_FlsSetValue@@YAP6GHKPAX@ZXZ@4QBW4module_id@?A0x391cf84c@@B 10004b3c     libucrt:winapi_thunks.obj
 0001:00003b50       ?candidate_modules@?1??try_get_InitializeCriticalSectionEx@@YAP6GHPAU_RTL_CRITICAL_SECTION@@KK@ZXZ@4QBW4module_id@?A0x391cf84c@@B 10004b50     libucrt:winapi_thunks.obj
 0001:00003b74       ?candidate_modules@?1??try_get_LCMapStringEx@@YAP6GHPB_WK0HPA_WHPAU_nlsversioninfo@@PAXJ@ZXZ@4QBW4module_id@?A0x391cf84c@@B 10004b74     libucrt:winapi_thunks.obj
 0001:00003b8c       ?candidate_modules@?1??try_get_LocaleNameToLCID@@YAP6GKPB_WK@ZXZ@4QBW4module_id@?A0x391cf84c@@B 10004b8c     libucrt:winapi_thunks.obj
 0001:00003ba8       ?candidate_modules@?1??try_get_AppPolicyGetProcessTerminationMethod@@YAP6GJPAXPAW4AppPolicyProcessTerminationMethod@@@ZXZ@4QBW4module_id@?A0x391cf84c@@B 10004ba8     libucrt:winapi_thunks.obj
 0001:00003be0       ?LcidToLocaleNameTable@?A0x881e4c05@@3QBULcidToLocaleName@1@B 10004be0     libucrt:lcidtoname_downlevel.obj
 0001:00004d00       ?LocaleNameToIndexTable@?A0x881e4c05@@3QBULocaleNameIndex@1@B 10005d00     libucrt:lcidtoname_downlevel.obj
 0001:00005c60       LOG_name                   10006c60     libucrt:log10_impl.obj
 0001:00005c70       _One                       10006c70     libucrt:ceil_pentium4.obj
 0001:00005c80       _Bns                       10006c80     libucrt:ceil_pentium4.obj
 0001:00005c90       _Zero                      10006c90     libucrt:ceil_pentium4.obj
 0001:00005ca0       _S                         10006ca0     libucrt:ceil_pentium4.obj
 0001:00005cb0       _NegZero                   10006cb0     libucrt:ceil_pentium4.obj
 0001:00005cd0       emask                      10006cd0     libucrt:log10_pentium4.obj
 0001:00005ce0       CC                         10006ce0     libucrt:log10_pentium4.obj
 0001:00005cf0       Magic                      10006cf0     libucrt:log10_pentium4.obj
 0001:00005d00       hi_mask                    10006d00     libucrt:log10_pentium4.obj
 0001:00005d10       LOG10_2                    10006d10     libucrt:log10_pentium4.obj
 0001:00005d20       place_L                    10006d20     libucrt:log10_pentium4.obj
 0001:00005d40       One                        10006d40     libucrt:log10_pentium4.obj
 0001:00005d50       Zero                       10006d50     libucrt:log10_pentium4.obj
 0001:00005d60       Two52                      10006d60     libucrt:log10_pentium4.obj
 0001:00005d70       Infs                       10006d70     libucrt:log10_pentium4.obj
 0001:00005d80       NaN                        10006d80     libucrt:log10_pentium4.obj
 0001:00005d90       coeff                      10006d90     libucrt:log10_pentium4.obj
 0001:00005dee       _log2max                   10006dee     libucrt:87tran.obj
 0001:00005df8       _smallarg                  10006df8     libucrt:87tran.obj
 0001:00005e02       _half                      10006e02     libucrt:87tran.obj
 0001:00005e4e       One                        10006e4e     libucrt:87disp.obj
 0001:00005e56       Three                      10006e56     libucrt:87disp.obj
 0001:00005e5e       XAMtoTagTab                10006e5e     libucrt:87disp.obj
 0001:00005e70       One                        10006e70     libucrt:common.obj
 0001:00005e84       DblMax                     10006e84     libucrt:common.obj
 0001:00005e8c       DblMin                     10006e8c     libucrt:common.obj
 0001:00005e94       IeeeAdjO                   10006e94     libucrt:common.obj
 0001:00005e9c       IeeeAdjU                   10006e9c     libucrt:common.obj
 0001:00005ea4       _infinity                  10006ea4     libucrt:common.obj
 0001:00005eac       _zero                      10006eac     libucrt:common.obj
 0001:00005ee8       _over                      10006ee8     libucrt:fpctrl.obj
 0001:00005ef4       _under                     10006ef4     libucrt:fpctrl.obj
 0001:00006728       ?_names@?1??_get_fname@@9@9 10007728     libucrt:fpexcept.obj
 0001:00006d80       $$000000                   10007d80     chkstk.obj
 0001:00006de0       ?GetFileNameThread@@YGKPAX@Z 10007de0 f   handles.obj
 0001:00006e30       ?GetUserAccountID@@YAPB_WXZ 10007e30 f   handles.obj
 0001:00007200       ?PrintNameAndType@@YA_NPAXK0PAVPerfThread@@@Z 10008200 f   handles.obj
 0001:000073e0       ?PrintNameByType@@YA_NPAXG0PAVPerfThread@@@Z 100083e0 f   handles.obj
 0001:00007c58       $LN42                      10008c58     PCFG.OBJ
 0001:00007c68       $LN39                      10008c68     PCFG.OBJ
 0001:00007da0       ?fIsWow64Process@@YGHPAXPAH@Z 10008da0 f i Proclist.obj
 0001:00007da0       ?fGetSidSubAuthority@@YGPAKPAXK@Z 10008da0 f i Proclist.obj
 0001:00007da0       ?fGetGuiResources@@YGKPAXK@Z 10008da0 f i Proclist.obj
 0001:00008670       ?fGetSidIdentifierAuthority@@YGPAU_SID_IDENTIFIER_AUTHORITY@@PAX@Z 10009670 f i Proclist.obj
 0001:00008670       ?fGetSidSubAuthorityCount@@YGPAEPAX@Z 10009670 f i Proclist.obj
 0001:00008670       ?fIsValidSid@@YGHPAX@Z     10009670 f i Proclist.obj
 0001:000087d4       $LN12                      100097d4     PCFG.OBJ
 0001:000087e4       $LN10                      100097e4     PCFG.OBJ
 0001:00008e54       $LN39                      10009e54     PCFG.OBJ
 0001:00008e64       $LN36                      10009e64     PCFG.OBJ
 0001:00009a6c       $LN48                      1000aa6c     Pclass.obj
 0001:00009d70       $LN60                      1000ad70     Pclass.obj
 0001:00009d7c       $LN54                      1000ad7c     Pclass.obj
 0001:00009da0       $LN61                      1000ada0     Pclass.obj
 0001:00009da8       $LN55                      1000ada8     Pclass.obj
 0001:00009de0       $LN62                      1000ade0     Pclass.obj
 0001:00009de8       $LN56                      1000ade8     Pclass.obj
 0001:00009e20       ?GenerateTitles@@YAXQAY0FA@_WPAUPanelMode@@QAY0BI@PA_W@Z 1000ae20 f   Pclass.obj
 0001:0000a098       $LN74                      1000b098     Pclass.obj
 0001:0000a0a8       $LN70                      1000b0a8     Pclass.obj
 0001:0000a0d8       $LN75                      1000b0d8     Pclass.obj
 0001:0000a0ec       $LN71                      1000b0ec     Pclass.obj
 0001:0000a124       $LN76                      1000b124     Pclass.obj
 0001:0000a144       $LN72                      1000b144     Pclass.obj
 0001:0000b65c       $LN191                     1000c65c     Pclass.obj
 0001:0000b670       $LN176                     1000c670     Pclass.obj
 0001:0000b6a8       $LN192                     1000c6a8     Pclass.obj
 0001:0000b6c8       $LN177                     1000c6c8     Pclass.obj
 0001:0000d558       $LN415                     1000e558     Pclass.obj
 0001:0000d568       $LN406                     1000e568     Pclass.obj
 0001:0000da0c       $LN55                      1000ea0c     Pclass.obj
 0001:0000da18       $LN46                      1000ea18     Pclass.obj
 0001:0000da3c       $LN56                      1000ea3c     Pclass.obj
 0001:0000da44       $LN47                      1000ea44     Pclass.obj
 0001:0000da7c       $LN57                      1000ea7c     Pclass.obj
 0001:0000da84       $LN48                      1000ea84     Pclass.obj
 0001:0000e960       ?getcounter@@YAHPA_W@Z     1000f960 f   perfthread.obj
 0001:0000ed90       ?FreeUserData@@YGXPAXPBUFarPanelItemFreeInfo@@@Z 1000fd90 f   Plist.obj
 0001:000105f0       ?fNtQueryObject@@YGJPAXK0K0@Z 100115f0 f   Proclist.obj
 0001:000105f0       ?fNtQueryInformationThread@@YGJPAXK0KPAK@Z 100115f0 f   Proclist.obj
 0001:000105f0       ?fNtQueryInformationFile@@YGJPAX00KK@Z 100115f0 f   Proclist.obj
 0001:000105f0       ?fNtQueryInformationProcess@@YGJPAXW4_PROCESSINFOCLASS@@0KPAK@Z 100115f0 f   Proclist.obj
 0001:00010600       ?fNtQuerySystemInformation@@YGJKPAXKPAK@Z 10011600 f   Proclist.obj
 0001:00010610       ?fLookupAccountName@@YGHPB_W0PAXPAKPA_W2PAW4_SID_NAME_USE@@@Z 10011610 f   Proclist.obj
 0001:00010620       ?fCoSetProxyBlanket@@YGJPAUIUnknown@@KKPA_WKKPAXK@Z 10011620 f   Proclist.obj
 0001:00010660       ?dynamic_bind@@YAXXZ       10011660 f   Proclist.obj
 0001:00010b60       ?DecodePointer@implementation@?1??DecodePointerWrapper@@YGPAXPAX@Z@SGPAX0@Z 10011b60 f   vc_crt_fix_impl.obj
 0001:00010b60       ?EncodePointer@implementation@?1??EncodePointerWrapper@@YGPAXPAX@Z@SGPAX0@Z 10011b60 f   vc_crt_fix_impl.obj
 0001:00010b70       ?GetLogicalProcessorInformation@implementation@?1??GetLogicalProcessorInformationWrapper@@YGHPAU_SYSTEM_LOGICAL_PROCESSOR_INFORMATION@@PAK@Z@SGH01@Z 10011b70 f   vc_crt_fix_impl.obj
 0001:00010b80       ?GetModuleHandleExW@implementation@?1??GetModuleHandleExWWrapper@@YGHKPB_WPAPAUHINSTANCE__@@@Z@SGHK01@Z 10011b80 f   vc_crt_fix_impl.obj
 0001:00010c50       ?GetNumaHighestNodeNumber@implementation@?1??GetNumaHighestNodeNumberWrapper@@YGHPAK@Z@SGH0@Z 10011c50 f   vc_crt_fix_impl.obj
 0001:00010c70       ?InitializeSListHead@implementation@slist@@YGXPAT_SLIST_HEADER@@@Z 10011c70 f   vc_crt_fix_impl.obj
 0001:00010d50       ?InterlockedFlushSList@implementation@slist@@YGPAU_SINGLE_LIST_ENTRY@@PAT_SLIST_HEADER@@@Z 10011d50 f   vc_crt_fix_impl.obj
 0001:00010d80       ?InterlockedPopEntrySList@implementation@slist@@YGPAU_SINGLE_LIST_ENTRY@@PAT_SLIST_HEADER@@@Z 10011d80 f   vc_crt_fix_impl.obj
 0001:00010dd0       ?InterlockedPushEntrySList@implementation@slist@@YGPAU_SINGLE_LIST_ENTRY@@PAT_SLIST_HEADER@@PAU3@@Z 10011dd0 f   vc_crt_fix_impl.obj
 0001:00010e10       ?InterlockedPushListSListEx@implementation@slist@@YGPAU_SINGLE_LIST_ENTRY@@PAT_SLIST_HEADER@@PAU3@1K@Z 10011e10 f   vc_crt_fix_impl.obj
 0001:00010e50       ?QueryDepthSList@implementation@slist@@YGGPAT_SLIST_HEADER@@@Z 10011e50 f   vc_crt_fix_impl.obj
 0001:00010e80       ?RtlFirstEntrySList@implementation@slist@@YGPAU_SINGLE_LIST_ENTRY@@PAT_SLIST_HEADER@@@Z 10011e80 f   vc_crt_fix_impl.obj
 0001:00010eb0       ?SetThreadStackGuarantee@implementation@?1??SetThreadStackGuaranteeWrapper@@YGHPAK@Z@SGH0@Z 10011eb0 f   vc_crt_fix_impl.obj
 0001:00010ec0       ?XorPointer@@YAPAXPAX@Z    10011ec0 f   vc_crt_fix_impl.obj
 0001:000113a0       $$000000                   100123a0     LIBCMT:ulldiv.obj
 0001:00011410       $$000000                   10012410     LIBCMT:lldiv.obj
 0001:000114c0       $$000000                   100124c0     LIBCMT:llmul.obj
 0001:00011500       $$000000                   10012500     LIBCMT:ullrem.obj
 0001:00011592       ?find_pe_section@@YAPAU_IMAGE_SECTION_HEADER@@QAEI@Z 10012592 f   LIBCMT:utility.obj
 0001:000118d8       ?dllmain_crt_dispatch@@YGHQAUHINSTANCE__@@KQAX@Z 100128d8 f   LIBCMT:dll_dllmain.obj
 0001:0001192b       ?dllmain_crt_process_attach@@YAHQAUHINSTANCE__@@QAX@Z 1001292b f   LIBCMT:dll_dllmain.obj
 0001:00011a35       ?dllmain_crt_process_detach@@YAH_N@Z 10012a35 f   LIBCMT:dll_dllmain.obj
 0001:00011ac7       ?dllmain_dispatch@@YAHQAUHINSTANCE__@@KQAX@Z 10012ac7 f   LIBCMT:dll_dllmain.obj
 0001:00011bcd       ?dllmain_raw@@YGHQAUHINSTANCE__@@KQAX@Z 10012bcd f   LIBCMT:dll_dllmain.obj
 0001:00012000       $$000000                   10013000     LIBCMT:sehprolg4.obj
 0001:0001205c       ___get_entropy             1001305c f   LIBCMT:gs_support.obj
 0001:000122f0       $$000000                   100132f0     libvcruntime:memset.obj
 0001:000125c0       $$000000                   100135c0     libvcruntime:memcpy.obj
 0001:00012824       TrailingUpVec              10013824     libvcruntime:memcpy.obj
 0001:000128d0       TrailingDownVec            100138d0     libvcruntime:memcpy.obj
 0001:00012b40       $$000000                   10013b40     libvcruntime:memmove.obj
 0001:00012da4       TrailingUpVec              10013da4     libvcruntime:memmove.obj
 0001:00012e50       TrailingDownVec            10013e50     libvcruntime:memmove.obj
 0001:00013120       _ValidateLocalCookies      10014120 f   libvcruntime:chandler4.obj
 0001:00013566       ?try_get_first_available_module@@YAPAUHINSTANCE__@@QBW4module_id@?A0x5c520fe1@@0@Z 10014566 f   libvcruntime:winapi_downlevel.obj
 0001:0001362a       ?try_get_function@@YAPAXW4function_id@?A0x5c520fe1@@QBDQBW4module_id@2@2@Z 1001462a f   libvcruntime:winapi_downlevel.obj
 0001:00013840       $$000000                   10014840     libvcruntime:exsup4.obj
 0001:000138d0       __unwind_handler4          100148d0 f   libvcruntime:exsup4.obj
 0001:00013a10       $$000000                   10014a10     libvcruntime:exsup.obj
 0001:00013a31       __unwind_handler           10014a31 f   libvcruntime:exsup.obj
 0001:00013b50       $$000000                   10014b50     libvcruntime:lowhelpr.obj
 0001:00014586       ??$common_xtox@_K_W@@YAH_KQA_WII_N@Z 10015586 f   libucrt:xtoa.obj
 0001:000149f0       ??$?RV<lambda_03b1d95aef87969028cfba75ccab2455>@@AAV<lambda_6e4b09c48022b2350581041d5f6b0c4c>@@V<lambda_22bdf7517842c4b3e53723af5aa32b9e>@@@?$__crt_seh_guarded_call@X@@QAEX$$QAV<lambda_03b1d95aef87969028cfba75ccab2455>@@AAV<lambda_6e4b09c48022b2350581041d5f6b0c4c>@@$$QAV<lambda_22bdf7517842c4b3e53723af5aa32b9e>@@@Z 100159f0 f   libucrt:exit.obj
 0001:00014a33       ??R<lambda_6e4b09c48022b2350581041d5f6b0c4c>@@QBE@XZ 10015a33 f   libucrt:exit.obj
 0001:00014b03       ?atexit_exception_filter@@YAHK@Z 10015b03 f   libucrt:exit.obj
 0001:00014b16       ?common_exit@@YAXHW4_crt_exit_cleanup_mode@@W4_crt_exit_return_mode@@@Z 10015b16 f   libucrt:exit.obj
 0001:00014b7c       ?exit_or_terminate_process@@YAXI@Z 10015b7c f   libucrt:exit.obj
 0001:00014bbe       ?is_managed_app@@YA_NXZ    10015bbe f   libucrt:exit.obj
 0001:00014c01       ?try_cor_exit_process@@YAXI@Z 10015c01 f   libucrt:exit.obj
 0001:00014c91       ??$common_configure_argv@D@@YAHW4_crt_argv_mode@@@Z 10015c91 f   libucrt:argv_parsing.obj
 0001:00014dc9       ??$parse_command_line@D@@YAXPADPAPAD0PAI2@Z 10015dc9 f   libucrt:argv_parsing.obj
 0001:00014f9c       ??$common_initialize_environment_nolock@D@@YAHXZ 10015f9c f   libucrt:environment_initialization.obj
 0001:00014fef       ??$create_environment@D@@YAQAPADQAD@Z 10015fef f   libucrt:environment_initialization.obj
 0001:000150c1       ??$free_environment@_W@@YAXQAPA_W@Z 100160c1 f   libucrt:environment_initialization.obj
 0001:000150c1       ??$free_environment@D@@YAXQAPAD@Z 100160c1 f   libucrt:environment_initialization.obj
 0001:00015119       ??$uninitialize_environment_internal@D@@YAXAAPAPAD@Z 10016119 f   libucrt:environment_initialization.obj
 0001:00015134       ??$uninitialize_environment_internal@_W@@YAXAAPAPA_W@Z 10016134 f   libucrt:environment_initialization.obj
 0001:0001518b       ??$?RV<lambda_69a2805e680e0e292e8ba93315fe43a8>@@AAV<lambda_f03950bc5685219e0bcd2087efbe011e>@@V<lambda_03fcd07e894ec930e3f35da366ca99d6>@@@?$__crt_seh_guarded_call@H@@QAEH$$QAV<lambda_69a2805e680e0e292e8ba93315fe43a8>@@AAV<lambda_f03950bc5685219e0bcd2087efbe011e>@@$$QAV<lambda_03fcd07e894ec930e3f35da366ca99d6>@@@Z 1001618b f   libucrt:onexit.obj
 0001:000151dc       ??$?RV<lambda_8e746cf0007f6ed984d6f78af1fec997>@@AAV<lambda_22ebabd17bc4fa466a2aca6d8deb888d>@@V<lambda_18ed0c0b38a6dc0daf1e7ac6d6adf05e>@@@?$__crt_seh_guarded_call@H@@QAEH$$QAV<lambda_8e746cf0007f6ed984d6f78af1fec997>@@AAV<lambda_22ebabd17bc4fa466a2aca6d8deb888d>@@$$QAV<lambda_18ed0c0b38a6dc0daf1e7ac6d6adf05e>@@@Z 100161dc f   libucrt:onexit.obj
 0001:0001524c       ??R<lambda_22ebabd17bc4fa466a2aca6d8deb888d>@@QBEHXZ 1001624c f   libucrt:onexit.obj
 0001:00015377       ??R<lambda_f03950bc5685219e0bcd2087efbe011e>@@QBEHXZ 10016377 f   libucrt:onexit.obj
 0001:000154f6       _initialize_global_variables 100164f6 f   libucrt:initialization.obj
 0001:00015503       _initialize_c              10016503 f   libucrt:initialization.obj
 0001:0001551d       _initialize_global_state_isolation 1001651d f   libucrt:initialization.obj
 0001:0001551d       _uninitialize_c            1001651d f   libucrt:initialization.obj
 0001:0001551d       _initialize_environment    1001651d f   libucrt:initialization.obj
 0001:0001551d       _uninitialize_global_state_isolation 1001651d f   libucrt:initialization.obj
 0001:0001551d       _report_memory_leaks       1001651d f   libucrt:initialization.obj
 0001:00015520       _uninitialize_environment  10016520 f   libucrt:initialization.obj
 0001:00015528       _initialize_pointers       10016528 f   libucrt:initialization.obj
 0001:00015556       _uninitialize_vcruntime    10016556 f   libucrt:initialization.obj
 0001:0001555f       _uninitialize_allocated_memory 1001655f f   libucrt:initialization.obj
 0001:00015578       _uninitialize_allocated_io_buffers 10016578 f   libucrt:initialization.obj
 0001:000155c8       ??R<lambda_af42a3ee9806e9a7305d451646e05244>@@QBEXAAPAU__crt_multibyte_data@@@Z 100165c8 f   libucrt:initialization.obj
 0001:00015850       $$000000                   10016850     libucrt:strncmp.obj
 0001:00015aba       ??$common_tox_l@$1?internal_isupper_l@@YA_NHQAU__crt_locale_pointers@@@Z$1?internal_map_lower@@YAHH0@Z@@YAHHKQAU__crt_locale_pointers@@@Z 10016aba f   libucrt:tolower_toupper.obj
 0001:00015c01       ?internal_isupper_l@@YA_NHQAU__crt_locale_pointers@@@Z 10016c01 f   libucrt:tolower_toupper.obj
 0001:00015cd0       $$000000                   10016cd0     libucrt:_memicmp.obj
 0001:00015d29       ??$?RV<lambda_15ade71b0218206bbe3333a0c9b79046>@@AAV<lambda_da44e0f8b0f19ba52fefafb335991732>@@V<lambda_207f2d024fc103971653565357d6cd41>@@@?$__crt_seh_guarded_call@X@@QAEX$$QAV<lambda_15ade71b0218206bbe3333a0c9b79046>@@AAV<lambda_da44e0f8b0f19ba52fefafb335991732>@@$$QAV<lambda_207f2d024fc103971653565357d6cd41>@@@Z 10016d29 f   libucrt:per_thread_data.obj
 0001:00015d71       ??$?RV<lambda_38edbb1296d33220d7e4dd0ed76b244a>@@AAV<lambda_5ce1d447e08cb34b2473517608e21441>@@V<lambda_fb385d3da700c9147fc39e65dd577a8c>@@@?$__crt_seh_guarded_call@X@@QAEX$$QAV<lambda_38edbb1296d33220d7e4dd0ed76b244a>@@AAV<lambda_5ce1d447e08cb34b2473517608e21441>@@$$QAV<lambda_fb385d3da700c9147fc39e65dd577a8c>@@@Z 10016d71 f   libucrt:per_thread_data.obj
 0001:00015dd2       ??$?RV<lambda_6affb1475c98b40b75cdec977db92e3c>@@AAV<lambda_b8d4b9c228a6ecc3f80208dbb4b4a104>@@V<lambda_608742c3c92a14382c1684fc64f96c88>@@@?$__crt_seh_guarded_call@X@@QAEX$$QAV<lambda_6affb1475c98b40b75cdec977db92e3c>@@AAV<lambda_b8d4b9c228a6ecc3f80208dbb4b4a104>@@$$QAV<lambda_608742c3c92a14382c1684fc64f96c88>@@@Z 10016dd2 f   libucrt:per_thread_data.obj
 0001:00015e1d       ??$?RV<lambda_a7e850c220f1c8d1e6efeecdedd162c6>@@AAV<lambda_46720907175c18b6c9d2717bc0d2d362>@@V<lambda_9048902d66e8d99359bc9897bbb930a8>@@@?$__crt_seh_guarded_call@X@@QAEX$$QAV<lambda_a7e850c220f1c8d1e6efeecdedd162c6>@@AAV<lambda_46720907175c18b6c9d2717bc0d2d362>@@$$QAV<lambda_9048902d66e8d99359bc9897bbb930a8>@@@Z 10016e1d f   libucrt:per_thread_data.obj
 0001:00015e6d       ?construct_ptd@@YAXQAU__acrt_ptd@@QAPAU__crt_locale_data@@@Z 10016e6d f   libucrt:per_thread_data.obj
 0001:00015f08       ?destroy_fls@@YGXPAX@Z     10016f08 f   libucrt:per_thread_data.obj
 0001:00015f29       ?destroy_ptd@@YAXQAU__acrt_ptd@@@Z 10016f29 f   libucrt:per_thread_data.obj
 0001:00015ff8       ?replace_current_thread_locale_nolock@@YAXQAU__acrt_ptd@@QAU__crt_locale_data@@@Z 10016ff8 f   libucrt:per_thread_data.obj
 0001:0001631b       ??$?RV<lambda_e5124f882df8998aaf41531e079ba474>@@AAV<lambda_3e16ef9562a7dcce91392c22ab16ea36>@@V<lambda_e25ca0880e6ef98be67edffd8c599615>@@@?$__crt_seh_guarded_call@X@@QAEX$$QAV<lambda_e5124f882df8998aaf41531e079ba474>@@AAV<lambda_3e16ef9562a7dcce91392c22ab16ea36>@@$$QAV<lambda_e25ca0880e6ef98be67edffd8c599615>@@@Z 1001731b f   libucrt:wsetlocale.obj
 0001:000167ac       ?<lambda_invoker_cdecl>@<lambda_86056e3c024bff449830248dc1621ed2>@@CAHPBX0@Z 100177ac f   libucrt:argv_wildcards.obj
 0001:000167c4       ??$__acrt_convert_wcs_mbs_cp@D_WV<lambda_62f6974d9771e494a5ea317cc32e971c>@@U__crt_win32_buffer_internal_dynamic_resizing@@@@YAHQBDAAV?$__crt_win32_buffer@_WU__crt_win32_buffer_internal_dynamic_resizing@@@@ABV<lambda_62f6974d9771e494a5ea317cc32e971c>@@I@Z 100177c4 f   libucrt:argv_wildcards.obj
 0001:00016876       ??$__acrt_convert_wcs_mbs_cp@_WDV<lambda_28bda7af82a03b66c1cb3803a755f95d>@@U__crt_win32_buffer_internal_dynamic_resizing@@@@YAHQB_WAAV?$__crt_win32_buffer@DU__crt_win32_buffer_internal_dynamic_resizing@@@@ABV<lambda_28bda7af82a03b66c1cb3803a755f95d>@@I@Z 10017876 f   libucrt:argv_wildcards.obj
 0001:00016964       ??$common_expand_argv_wildcards@D@@YAHQAPADQAPAPAD@Z 10017964 f   libucrt:argv_wildcards.obj
 0001:00016b55       ??$copy_and_add_argument_to_buffer@D@@YAHQBD0IAAV?$argument_list@D@?A0x5f5c8891@@@Z 10017b55 f   libucrt:argv_wildcards.obj
 0001:00016c08       ??$expand_argument_wildcards@D@@YAHQAD0AAV?$argument_list@D@?A0x5f5c8891@@@Z 10017c08 f   libucrt:argv_wildcards.obj
 0001:00016f56       ?expand_if_necessary@?$argument_list@D@?A0x5f5c8891@@AAEHXZ 10017f56 f   libucrt:argv_wildcards.obj
 0001:00016fe8       ??$__acrt_convert_wcs_mbs_cp@_WDV<lambda_0fec1a7b3f42a53036604e18c2d5e07e>@@U__crt_win32_buffer_no_resizing@@@@YAHQB_WAAV?$__crt_win32_buffer@DU__crt_win32_buffer_no_resizing@@@@ABV<lambda_0fec1a7b3f42a53036604e18c2d5e07e>@@I@Z 10017fe8 f   libucrt:getmodulefilenamea.obj
 0001:0001718d       ??$?RV<lambda_ceb1ee4838e85a9d631eb091e2fbe199>@@AAV<lambda_ae742caa10f662c28703da3d2ea5e57e>@@V<lambda_cd08b5d6af4937fe54fc07d0c9bf6b37>@@@?$__crt_seh_guarded_call@X@@QAEX$$QAV<lambda_ceb1ee4838e85a9d631eb091e2fbe199>@@AAV<lambda_ae742caa10f662c28703da3d2ea5e57e>@@$$QAV<lambda_cd08b5d6af4937fe54fc07d0c9bf6b37>@@@Z 1001818d f   libucrt:mbctype.obj
 0001:000171d0       ??R<lambda_ae742caa10f662c28703da3d2ea5e57e>@@QBEXXZ 100181d0 f   libucrt:mbctype.obj
 0001:00017253       ?CPtoLocaleName@@YAPB_WH@Z 10018253 f   libucrt:mbctype.obj
 0001:00017291       ?getSystemCP@@YAHH@Z       10018291 f   libucrt:mbctype.obj
 0001:00017304       ?setSBCS@@YAXPAU__crt_multibyte_data@@@Z 10018304 f   libucrt:mbctype.obj
 0001:00017369       ?setSBUpLow@@YAXPAU__crt_multibyte_data@@@Z 10018369 f   libucrt:mbctype.obj
 0001:000174ec       ?setmbcp_internal@@YAHH_NQAU__acrt_ptd@@QAPAU__crt_multibyte_data@@@Z 100184ec f   libucrt:mbctype.obj
 0001:00017607       ?update_thread_multibyte_data_internal@@YAPAU__crt_multibyte_data@@QAU__acrt_ptd@@QAPAU1@@Z 10018607 f   libucrt:mbctype.obj
 0001:000178ed       _memcpy_s                  100188ed f   libucrt:mbctype.obj
 0001:0001796e       ?x_ismbbtype_l@@YAHPAU__crt_locale_pointers@@IHH@Z 1001896e f   libucrt:ismbbyte.obj
 0001:00017b85       ?find_end_of_double_null_terminated_sequence@@YAPB_WQB_W@Z 10018b85 f   libucrt:get_environment_from_os.obj
 0001:00017caf       ?initialize_inherited_file_handles_nolock@@YAXXZ 10018caf f   libucrt:ioinit.obj
 0001:00017d67       ?initialize_stdio_handles_nolock@@YAXXZ 10018d67 f   libucrt:ioinit.obj
 0001:00017e9d       ?try_get_AreFileApisANSI@@YAP6GHXZXZ 10018e9d f   libucrt:winapi_thunks.obj
 0001:00017eb7       ?try_get_LCMapStringEx@@YAP6GHPB_WK0HPA_WHPAU_nlsversioninfo@@PAXJ@ZXZ 10018eb7 f   libucrt:winapi_thunks.obj
 0001:00017ed1       ?try_get_LocaleNameToLCID@@YAP6GKPB_WK@ZXZ 10018ed1 f   libucrt:winapi_thunks.obj
 0001:00017eeb       ?try_get_first_available_module@@YAPAUHINSTANCE__@@QBW4module_id@?A0x391cf84c@@0@Z 10018eeb f   libucrt:winapi_thunks.obj
 0001:00017fb4       ?try_get_function@@YAPAXW4function_id@?A0x391cf84c@@QBDQBW4module_id@2@2@Z 10018fb4 f   libucrt:winapi_thunks.obj
 0001:00018383       ??$?RV<lambda_cbab9ec6f41b0180b23cc171c22676b0>@@AAV<lambda_44731a7d0e6d81c3e6aa82d741081786>@@V<lambda_4b292cb8dd18144e164572427af410ab>@@@?$__crt_seh_guarded_call@P6AXH@Z@@QAEP6AXH@Z$$QAV<lambda_cbab9ec6f41b0180b23cc171c22676b0>@@AAV<lambda_44731a7d0e6d81c3e6aa82d741081786>@@$$QAV<lambda_4b292cb8dd18144e164572427af410ab>@@@Z 10019383 f   libucrt:signal.obj
 0001:000183dd       ?get_global_action_nolock@@YAPAP6AXH@ZH@Z 100193dd f   libucrt:signal.obj
 0001:0001841f       ?siglookup@@YAPAU__crt_signal_action_t@@HQAU1@@Z 1001941f f   libucrt:signal.obj
 0001:000186d7       ??$?RV<lambda_2866be3712abc81a800a822484c830d8>@@AAV<lambda_39ca0ed439415581b5b15c265174cece>@@V<lambda_2b24c74d71094a6cd0cb82e44167d71b>@@@?$__crt_seh_guarded_call@X@@QAEX$$QAV<lambda_2866be3712abc81a800a822484c830d8>@@AAV<lambda_39ca0ed439415581b5b15c265174cece>@@$$QAV<lambda_2b24c74d71094a6cd0cb82e44167d71b>@@@Z 100196d7 f   libucrt:fflush.obj
 0001:00018759       ??$?RV<lambda_2cc53f568c5a2bb6f192f930a45d44ea>@@AAV<lambda_ab61a845afdef5b7c387490eaf3616ee>@@V<lambda_c2ffc0b7726aa6be21d5f0026187e748>@@@?$__crt_seh_guarded_call@X@@QAEX$$QAV<lambda_2cc53f568c5a2bb6f192f930a45d44ea>@@AAV<lambda_ab61a845afdef5b7c387490eaf3616ee>@@$$QAV<lambda_c2ffc0b7726aa6be21d5f0026187e748>@@@Z 10019759 f   libucrt:fflush.obj
 0001:000187fb       ?common_flush_all@@YAH_N@Z 100197fb f   libucrt:fflush.obj
 0001:0001884a       ?common_flush_all_should_try_to_flush_stream@@YA_NV__crt_stdio_stream@@QAH@Z 1001984a f   libucrt:fflush.obj
 0001:0001887d       ?is_stream_flushable_or_commitable@@YA_NJ@Z 1001987d f   libucrt:fflush.obj
 0001:00018c19       ?__acrt_LCMapStringA_stat@@YAHPAU__crt_locale_pointers@@PB_WKPBDHPADHHH@Z 10019c19 f   libucrt:lcmapstringa.obj
 0001:00019369       ?free_crt_array_internal@@YAXQAPBXI@Z 1001a369 f   libucrt:inittime.obj
 0001:000195b0       ?swap@@YAXPAD0I@Z          1001a5b0 f   libucrt:qsort.obj
 0001:00019a34       ??$common_tcsncpy_s@D@@YAHQADIQBDI@Z 1001aa34 f   libucrt:strncpy_s.obj
 0001:00019b00       $$000000                   1001ab00     libucrt:strpbrk.obj
 0001:00019be6       ?initialize_multibyte@@YAHXZ 1001abe6 f   libucrt:multibyte_initializer.obj
 0001:00019f18       ?GetTableIndexFromLocaleName@@YAHPB_W@Z 1001af18 f   libucrt:lcidtoname_downlevel.obj
 0001:00019ff8       ??$?RV<lambda_9e9de3de5fa147e2223d7db92bc10aa6>@@AAV<lambda_38ce7e780aa69e748d6df282ebc68efe>@@V<lambda_8ca6da459f0f6780f1cff60fdc3d00e5>@@@?$__crt_seh_guarded_call@H@@QAEH$$QAV<lambda_9e9de3de5fa147e2223d7db92bc10aa6>@@AAV<lambda_38ce7e780aa69e748d6df282ebc68efe>@@$$QAV<lambda_8ca6da459f0f6780f1cff60fdc3d00e5>@@@Z 1001aff8 f   libucrt:commit.obj
 0001:0001a10f       ?write_double_translated_ansi_nolock@@YA?AUwrite_result@?A0x17268360@@HQBDI@Z 1001b10f f   libucrt:write.obj
 0001:0001a4bb       ?write_double_translated_unicode_nolock@@YA?AUwrite_result@?A0x17268360@@QBDI@Z 1001b4bb f   libucrt:write.obj
 0001:0001a525       ?write_requires_double_translation_nolock@@YA_NH@Z 1001b525 f   libucrt:write.obj
 0001:0001a598       ?write_text_ansi_nolock@@YA?AUwrite_result@?A0x17268360@@HQBDI@Z 1001b598 f   libucrt:write.obj
 0001:0001a675       ?write_text_utf16le_nolock@@YA?AUwrite_result@?A0x17268360@@HQBDI@Z 1001b675 f   libucrt:write.obj
 0001:0001a760       ?write_text_utf8_nolock@@YA?AUwrite_result@?A0x17268360@@HQBDI@Z 1001b760 f   libucrt:write.obj
 0001:0001ac97       ??R<lambda_0f007d4f94c691a9a85cf1869a09f0c3>@@QBEIPBD@Z 1001bc97 f   libucrt:mbrtowc.obj
 0001:0001ae43       ??$common_lseek_nolock@_J@@YA_JH_JH@Z 1001be43 f   libucrt:lseek.obj
 0001:0001b1c0       $$000000                   1001c1c0     libucrt:log10_impl.obj
 0001:0001b2d0       $$000000                   1001c2d0     libucrt:ceil_pentium4.obj
 0001:0001b3f0       $$000000                   1001c3f0     libucrt:_strnicm.obj
 0001:0001b451       ?__dcrt_lowio_initialize_console_output@@YAXXZ 1001c451 f   libucrt:initcon.obj
 0001:0001b4fb       ??$?RV<lambda_218ce3db14220d0be481dae8ef3383b6>@@AAV<lambda_628dfdc04ba53c8bfc02c9951375f3f5>@@V<lambda_57dc472bd5c9d5f3b2cbca59b8a843ae>@@@?$__crt_seh_guarded_call@H@@QAEH$$QAV<lambda_218ce3db14220d0be481dae8ef3383b6>@@AAV<lambda_628dfdc04ba53c8bfc02c9951375f3f5>@@$$QAV<lambda_57dc472bd5c9d5f3b2cbca59b8a843ae>@@@Z 1001c4fb f   libucrt:close.obj
 0001:0001b700       $$000000                   1001c700     libucrt:log10_pentium4.obj
 0001:0001b990       $$000000                   1001c990     libucrt:87tran.obj
 0001:0001bba0       $$000000                   1001cba0     libucrt:87disp.obj
 0001:0001be00       $$000000                   1001ce00     libucrt:common.obj
 0001:0001bf90       $$000000                   1001cf90     libucrt:genexcep.obj
 0001:0001d040       $$000000                   1001e040     LIBCMT:ulldvrm.obj
 0001:0001d0e0       $$000000                   1001e0e0     LIBCMT:lldvrm.obj
 0001:0001d1c0       $$000000                   1001e1c0     LIBCMT:ullshr.obj
 0001:0001d1e0       $$000000                   1001e1e0     LIBCMT:alloca16.obj
 0001:0001d210       $$000000                   1001e210     LIBCMT:llshl.obj
 0001:0001d230       $$000000                   1001e230     LIBCMT:ftol2.obj
 0001:0001d2f0       $$000000                   1001e2f0     libvcruntime:strchr.obj
 0001:0001d420       $$000000                   1001e420     libvcruntime:strrchr.obj
 0001:0001d560       ??__FDeleter@?1??InitializeSListHead@implementation@slist@@YGXPAT_SLIST_HEADER@@@Z@YAXXZ 1001e560 f   vc_crt_fix_impl.obj
 0001:0001d5a0       __sehtable$___scrt_is_nonwritable_in_current_image 1001e5a0     LIBCMT:utility.obj
 0001:0001d5c0       __sehtable$?dllmain_crt_process_attach@@YAHQAUHINSTANCE__@@QAX@Z 1001e5c0     LIBCMT:dll_dllmain.obj
 0001:0001d5e0       __sehtable$?dllmain_crt_process_detach@@YAH_N@Z 1001e5e0     LIBCMT:dll_dllmain.obj
 0001:0001d600       __sehtable$?dllmain_dispatch@@YAHQAUHINSTANCE__@@KQAX@Z 1001e600     LIBCMT:dll_dllmain.obj
 0001:0001d6b0       __sehtable$___DestructExceptionObject 1001e6b0     libvcruntime:ehhelpers.obj
 0001:0001d6d0       __sehtable$__query_new_handler 1001e6d0     libucrt:new_handler.obj
 0001:0001d6f0       __sehtable$??R<lambda_6e4b09c48022b2350581041d5f6b0c4c>@@QBE@XZ 1001e6f0     libucrt:exit.obj
 0001:0001d710       __sehtable$??$?RV<lambda_03b1d95aef87969028cfba75ccab2455>@@AAV<lambda_6e4b09c48022b2350581041d5f6b0c4c>@@V<lambda_22bdf7517842c4b3e53723af5aa32b9e>@@@?$__crt_seh_guarded_call@X@@QAEX$$QAV<lambda_03b1d95aef87969028cfba75ccab2455>@@AAV<lambda_6e4b09c48022b2350581041d5f6b0c4c>@@$$QAV<lambda_22bdf7517842c4b3e53723af5aa32b9e>@@@Z 1001e710     libucrt:exit.obj
 0001:0001d730       __sehtable$??$?RV<lambda_8e746cf0007f6ed984d6f78af1fec997>@@AAV<lambda_22ebabd17bc4fa466a2aca6d8deb888d>@@V<lambda_18ed0c0b38a6dc0daf1e7ac6d6adf05e>@@@?$__crt_seh_guarded_call@H@@QAEH$$QAV<lambda_8e746cf0007f6ed984d6f78af1fec997>@@AAV<lambda_22ebabd17bc4fa466a2aca6d8deb888d>@@$$QAV<lambda_18ed0c0b38a6dc0daf1e7ac6d6adf05e>@@@Z 1001e730     libucrt:onexit.obj
 0001:0001d750       __sehtable$??$?RV<lambda_69a2805e680e0e292e8ba93315fe43a8>@@AAV<lambda_f03950bc5685219e0bcd2087efbe011e>@@V<lambda_03fcd07e894ec930e3f35da366ca99d6>@@@?$__crt_seh_guarded_call@H@@QAEH$$QAV<lambda_69a2805e680e0e292e8ba93315fe43a8>@@AAV<lambda_f03950bc5685219e0bcd2087efbe011e>@@$$QAV<lambda_03fcd07e894ec930e3f35da366ca99d6>@@@Z 1001e750     libucrt:onexit.obj
 0001:0001d770       __sehtable$_terminate      1001e770     libucrt:terminate.obj
 0001:0001d790       __sehtable$??$?RV<lambda_15ade71b0218206bbe3333a0c9b79046>@@AAV<lambda_da44e0f8b0f19ba52fefafb335991732>@@V<lambda_207f2d024fc103971653565357d6cd41>@@@?$__crt_seh_guarded_call@X@@QAEX$$QAV<lambda_15ade71b0218206bbe3333a0c9b79046>@@AAV<lambda_da44e0f8b0f19ba52fefafb335991732>@@$$QAV<lambda_207f2d024fc103971653565357d6cd41>@@@Z 1001e790     libucrt:per_thread_data.obj
 0001:0001d7b0       __sehtable$??$?RV<lambda_a7e850c220f1c8d1e6efeecdedd162c6>@@AAV<lambda_46720907175c18b6c9d2717bc0d2d362>@@V<lambda_9048902d66e8d99359bc9897bbb930a8>@@@?$__crt_seh_guarded_call@X@@QAEX$$QAV<lambda_a7e850c220f1c8d1e6efeecdedd162c6>@@AAV<lambda_46720907175c18b6c9d2717bc0d2d362>@@$$QAV<lambda_9048902d66e8d99359bc9897bbb930a8>@@@Z 1001e7b0     libucrt:per_thread_data.obj
 0001:0001d7d0       __sehtable$??$?RV<lambda_38edbb1296d33220d7e4dd0ed76b244a>@@AAV<lambda_5ce1d447e08cb34b2473517608e21441>@@V<lambda_fb385d3da700c9147fc39e65dd577a8c>@@@?$__crt_seh_guarded_call@X@@QAEX$$QAV<lambda_38edbb1296d33220d7e4dd0ed76b244a>@@AAV<lambda_5ce1d447e08cb34b2473517608e21441>@@$$QAV<lambda_fb385d3da700c9147fc39e65dd577a8c>@@@Z 1001e7d0     libucrt:per_thread_data.obj
 0001:0001d7f0       __sehtable$??$?RV<lambda_6affb1475c98b40b75cdec977db92e3c>@@AAV<lambda_b8d4b9c228a6ecc3f80208dbb4b4a104>@@V<lambda_608742c3c92a14382c1684fc64f96c88>@@@?$__crt_seh_guarded_call@X@@QAEX$$QAV<lambda_6affb1475c98b40b75cdec977db92e3c>@@AAV<lambda_b8d4b9c228a6ecc3f80208dbb4b4a104>@@$$QAV<lambda_608742c3c92a14382c1684fc64f96c88>@@@Z 1001e7f0     libucrt:per_thread_data.obj
 0001:0001d810       __sehtable$??$?RV<lambda_e5124f882df8998aaf41531e079ba474>@@AAV<lambda_3e16ef9562a7dcce91392c22ab16ea36>@@V<lambda_e25ca0880e6ef98be67edffd8c599615>@@@?$__crt_seh_guarded_call@X@@QAEX$$QAV<lambda_e5124f882df8998aaf41531e079ba474>@@AAV<lambda_3e16ef9562a7dcce91392c22ab16ea36>@@$$QAV<lambda_e25ca0880e6ef98be67edffd8c599615>@@@Z 1001e810     libucrt:wsetlocale.obj
 0001:0001d830       __sehtable$?update_thread_multibyte_data_internal@@YAPAU__crt_multibyte_data@@QAU__acrt_ptd@@QAPAU1@@Z 1001e830     libucrt:mbctype.obj
 0001:0001d850       __sehtable$??$?RV<lambda_ceb1ee4838e85a9d631eb091e2fbe199>@@AAV<lambda_ae742caa10f662c28703da3d2ea5e57e>@@V<lambda_cd08b5d6af4937fe54fc07d0c9bf6b37>@@@?$__crt_seh_guarded_call@X@@QAEX$$QAV<lambda_ceb1ee4838e85a9d631eb091e2fbe199>@@AAV<lambda_ae742caa10f662c28703da3d2ea5e57e>@@$$QAV<lambda_cd08b5d6af4937fe54fc07d0c9bf6b37>@@@Z 1001e850     libucrt:mbctype.obj
 0001:0001d870       __sehtable$___acrt_initialize_lowio 1001e870     libucrt:ioinit.obj
 0001:0001d890       __sehtable$_raise          1001e890     libucrt:signal.obj
 0001:0001d8b0       __sehtable$??$?RV<lambda_cbab9ec6f41b0180b23cc171c22676b0>@@AAV<lambda_44731a7d0e6d81c3e6aa82d741081786>@@V<lambda_4b292cb8dd18144e164572427af410ab>@@@?$__crt_seh_guarded_call@P6AXH@Z@@QAEP6AXH@Z$$QAV<lambda_cbab9ec6f41b0180b23cc171c22676b0>@@AAV<lambda_44731a7d0e6d81c3e6aa82d741081786>@@$$QAV<lambda_4b292cb8dd18144e164572427af410ab>@@@Z 1001e8b0     libucrt:signal.obj
 0001:0001d8d0       __sehtable$??$?RV<lambda_2866be3712abc81a800a822484c830d8>@@AAV<lambda_39ca0ed439415581b5b15c265174cece>@@V<lambda_2b24c74d71094a6cd0cb82e44167d71b>@@@?$__crt_seh_guarded_call@X@@QAEX$$QAV<lambda_2866be3712abc81a800a822484c830d8>@@AAV<lambda_39ca0ed439415581b5b15c265174cece>@@$$QAV<lambda_2b24c74d71094a6cd0cb82e44167d71b>@@@Z 1001e8d0     libucrt:fflush.obj
 0001:0001d8f0       __sehtable$??$?RV<lambda_2cc53f568c5a2bb6f192f930a45d44ea>@@AAV<lambda_ab61a845afdef5b7c387490eaf3616ee>@@V<lambda_c2ffc0b7726aa6be21d5f0026187e748>@@@?$__crt_seh_guarded_call@X@@QAEX$$QAV<lambda_2cc53f568c5a2bb6f192f930a45d44ea>@@AAV<lambda_ab61a845afdef5b7c387490eaf3616ee>@@$$QAV<lambda_c2ffc0b7726aa6be21d5f0026187e748>@@@Z 1001e8f0     libucrt:fflush.obj
 0001:0001d910       __sehtable$___acrt_update_thread_locale_data 1001e910     libucrt:locale_refcounting.obj
 0001:0001d930       __sehtable$___acrt_lowio_ensure_fh_exists 1001e930     libucrt:osfinfo.obj
 0001:0001d950       __sehtable$??$?RV<lambda_9e9de3de5fa147e2223d7db92bc10aa6>@@AAV<lambda_38ce7e780aa69e748d6df282ebc68efe>@@V<lambda_8ca6da459f0f6780f1cff60fdc3d00e5>@@@?$__crt_seh_guarded_call@H@@QAEH$$QAV<lambda_9e9de3de5fa147e2223d7db92bc10aa6>@@AAV<lambda_38ce7e780aa69e748d6df282ebc68efe>@@$$QAV<lambda_8ca6da459f0f6780f1cff60fdc3d00e5>@@@Z 1001e950     libucrt:commit.obj
 0001:0001d970       __sehtable$__write         1001e970     libucrt:write.obj
 0001:0001d990       __sehtable$__fcloseall     1001e990     libucrt:closeall.obj
 0001:0001d9b0       __sehtable$_fclose         1001e9b0     libucrt:fclose.obj
 0001:0001d9d0       __sehtable$??$?RV<lambda_218ce3db14220d0be481dae8ef3383b6>@@AAV<lambda_628dfdc04ba53c8bfc02c9951375f3f5>@@V<lambda_57dc472bd5c9d5f3b2cbca59b8a843ae>@@@?$__crt_seh_guarded_call@H@@QAEH$$QAV<lambda_218ce3db14220d0be481dae8ef3383b6>@@AAV<lambda_628dfdc04ba53c8bfc02c9951375f3f5>@@$$QAV<lambda_57dc472bd5c9d5f3b2cbca59b8a843ae>@@@Z 1001e9d0     libucrt:close.obj
 0001:0001d9f0       __sehtable$__IsNonwritableInCurrentImage 1001e9f0     LIBCMT:pesect.obj
 0001:0001da10       .edata                     1001ea10     ProcList.exp
 0001:0001da38       rgpv                       1001ea38     ProcList.exp
 0001:0001da74       rgszName                   1001ea74     ProcList.exp
 0001:0001dab0       rgwOrd                     1001eab0     ProcList.exp
 0001:0001dace       szName                     1001eace     ProcList.exp
 0001:0001dadb       $N00001                    1001eadb     ProcList.exp
 0001:0001dae7       $N00002                    1001eae7     ProcList.exp
 0001:0001daf0       $N00003                    1001eaf0     ProcList.exp
 0001:0001dafb       $N00004                    1001eafb     ProcList.exp
 0001:0001db08       $N00005                    1001eb08     ProcList.exp
 0001:0001db11       $N00006                    1001eb11     ProcList.exp
 0001:0001db1f       $N00007                    1001eb1f     ProcList.exp
 0001:0001db29       $N00008                    1001eb29     ProcList.exp
 0001:0001db36       $N00009                    1001eb36     ProcList.exp
 0001:0001db45       $N00010                    1001eb45     ProcList.exp
 0001:0001db57       $N00011                    1001eb57     ProcList.exp
 0001:0001db66       $N00012                    1001eb66     ProcList.exp
 0001:0001db6c       $N00013                    1001eb6c     ProcList.exp
 0001:0001db7f       $N00014                    1001eb7f     ProcList.exp
 0001:0001db92       $N00015                    1001eb92     ProcList.exp
 0002:00000010       ?FKeys@?1??GetOpenPanelInfo@Plist@@QAEXPAUOpenPanelInfo@@@Z@4PAGA 1001f010     Pclass.obj
 0002:00000054       ?kbt@?1??GetOpenPanelInfo@Plist@@QAEXPAUOpenPanelInfo@@@Z@4UKeyBarTitles@@A 1001f054     Pclass.obj
 0002:0000005c       ?nr@?7??Connect@Plist@@QAE_NPB_W00@Z@4U_NETRESOURCEW@@A 1001f05c     Pclass.obj
 0002:000001e0       ?__vcrt_flsindex@@3KA      1001f1e0     libvcruntime:per_thread_data.obj
 0002:00000210       ?errno_no_memory@@3HA      1001f210     libucrt:errno.obj
 0002:00000214       ?doserrno_no_memory@@3KA   1001f214     libucrt:errno.obj
 0002:00000220       ?__acrt_flsindex@@3KA      1001f220     libucrt:per_thread_data.obj
 0002:00000510       __mbctypes                 1001f510     libucrt:mbctype.obj
 0002:00000618       __mbcasemaps               1001f618     libucrt:mbctype.obj
 0002:00000718       ?__rgctypeflag@@3PADA      1001f718     libucrt:mbctype.obj
 0002:00000720       ?__rgcode_page_info@@3PAUcode_page_info@@A 1001f720     libucrt:mbctype.obj
 0002:00000a20       ?__dcrt_lowio_console_output_handle@@3PAXA 1001fa20     libucrt:initcon.obj
 0002:00020ab8       ?pUserAccountID@@3PB_WB    1003fab8     handles.obj
 0002:00020ac0       ?UserAccountID@?1??GetUserAccountID@@YAPB_WXZ@4PA_WA 1003fac0     handles.obj
 0002:00024dc8       ?TitlesLocal@?1??PanelModes@Plist@@QAEPAUPanelMode@@AAI@Z@4PAY0BI@PA_WA 10043dc8     Pclass.obj
 0002:00025188       ?TitlesRemote@?1??PanelModes@Plist@@QAEPAUPanelMode@@AAI@Z@4PAY0BI@PA_WA 10044188     Pclass.obj
 0002:00025548       ?OldMsg0@?1??PanelModes@Plist@@QAEPAUPanelMode@@AAI@Z@4PB_WB 10044548     Pclass.obj
 0002:00025550       ?Title@?1??GetOpenPanelInfo@Plist@@QAEXPAUOpenPanelInfo@@@Z@4PA_WA 10044550     Pclass.obj
 0002:00025618       ?kbl@?1??GetOpenPanelInfo@Plist@@QAEXPAUOpenPanelInfo@@@Z@4PAUKeyBarLabel@@A 10044618     Pclass.obj
 0002:000256c8       ?FullStr@?1??PrintTitle@Plist@@SAPA_WH@Z@4PA_WA 100446c8     Pclass.obj
 0002:000258d0       ?buf@?1??PrintTime@@YAPA_WK_N@Z@4PA_WA 100448d0     Plist.obj
 0002:00025910       ?items@?1??WinError@@YAHPA_W@Z@4PAPB_WA 10044910     Pmix.obj
 0002:00025a98       ?Inited@?1??dynamic_bind@@YAXXZ@4HA 10044a98     Proclist.obj
 0002:00025a9c       ?PluginMenuStrings@?4??GetPluginInfoW@@9@4@4PAPB_WA 10044a9c     Proclist.obj
 0002:00025aa0       ?DiskMenuStrings@?7??GetPluginInfoW@@9@4@4PAPB_WA 10044aa0     Proclist.obj
 0002:00025aa4       ?PluginCfgStrings@?1??GetPluginInfoW@@9@4@4PAPB_WA 10044aa4     Proclist.obj
 0002:00025aac       ?Cookie@?1??XorPointer@@YAPAXPAX@Z@4IB 10044aac     vc_crt_fix_impl.obj
 0002:00025ab0       ?$S1@?1??XorPointer@@YAPAXPAX@Z@4IA 10044ab0     vc_crt_fix_impl.obj
 0002:00025ab4       ?Function@?1??EncodePointerWrapper@@9@4@4Q6GPAXPAX@ZA 10044ab4     vc_crt_fix_impl.obj
 0002:00025ab8       ?$S2@?1??EncodePointerWrapper@@9@4@4IA 10044ab8     vc_crt_fix_impl.obj
 0002:00025abc       ?Function@?1??DecodePointerWrapper@@9@4@4Q6GPAXPAX@ZA 10044abc     vc_crt_fix_impl.obj
 0002:00025ac0       ?$S3@?1??DecodePointerWrapper@@9@4@4IA 10044ac0     vc_crt_fix_impl.obj
 0002:00025ac4       ?Function@?1??GetModuleHandleExWWrapper@@9@12@4Q6GHKPB_WPAPAUHINSTANCE__@@@ZA 10044ac4     vc_crt_fix_impl.obj
 0002:00025ac8       ?$S4@?1??GetModuleHandleExWWrapper@@9@12@4IA 10044ac8     vc_crt_fix_impl.obj
 0002:00025acc       ?Deleter@?1??InitializeSListHead@implementation@slist@@YGXPAT_SLIST_HEADER@@@Z@4Vservice_deleter@23@A 10044acc     vc_crt_fix_impl.obj
 0002:00025aec       ?$S5@?1??InitializeSListHead@implementation@slist@@YGXPAT_SLIST_HEADER@@@Z@4IA 10044aec     vc_crt_fix_impl.obj
 0002:00025af0       ?Function@?1??InitializeSListHeadWrapper@@9@4@4Q6GXPAT_SLIST_HEADER@@@ZA 10044af0     vc_crt_fix_impl.obj
 0002:00025af4       ?$S6@?1??InitializeSListHeadWrapper@@9@4@4IA 10044af4     vc_crt_fix_impl.obj
 0002:00025af8       ?Function@?1??InterlockedFlushSListWrapper@@9@4@4Q6GPAU_SINGLE_LIST_ENTRY@@PAT_SLIST_HEADER@@@ZA 10044af8     vc_crt_fix_impl.obj
 0002:00025afc       ?$S7@?1??InterlockedFlushSListWrapper@@9@4@4IA 10044afc     vc_crt_fix_impl.obj
 0002:00025b00       ?Function@?1??InterlockedPopEntrySListWrapper@@9@4@4Q6GPAU_SINGLE_LIST_ENTRY@@PAT_SLIST_HEADER@@@ZA 10044b00     vc_crt_fix_impl.obj
 0002:00025b04       ?$S8@?1??InterlockedPopEntrySListWrapper@@9@4@4IA 10044b04     vc_crt_fix_impl.obj
 0002:00025b08       ?Function@?1??InterlockedPushEntrySListWrapper@@9@8@4Q6GPAU_SINGLE_LIST_ENTRY@@PAT_SLIST_HEADER@@PAU2@@ZA 10044b08     vc_crt_fix_impl.obj
 0002:00025b0c       ?$S9@?1??InterlockedPushEntrySListWrapper@@9@8@4IA 10044b0c     vc_crt_fix_impl.obj
 0002:00025b10       ?Function@?1??InterlockedPushListSListExWrapper@@9@16@4Q6GPAU_SINGLE_LIST_ENTRY@@PAT_SLIST_HEADER@@PAU2@1K@ZA 10044b10     vc_crt_fix_impl.obj
 0002:00025b14       ?$S10@?1??InterlockedPushListSListExWrapper@@9@16@4IA 10044b14     vc_crt_fix_impl.obj
 0002:00025b18       ?Function@?1??RtlFirstEntrySListWrapper@@9@4@4Q6GPAU_SINGLE_LIST_ENTRY@@PAT_SLIST_HEADER@@@ZA 10044b18     vc_crt_fix_impl.obj
 0002:00025b1c       ?$S11@?1??RtlFirstEntrySListWrapper@@9@4@4IA 10044b1c     vc_crt_fix_impl.obj
 0002:00025b20       ?Function@?1??QueryDepthSListWrapper@@9@4@4Q6GGPAT_SLIST_HEADER@@@ZA 10044b20     vc_crt_fix_impl.obj
 0002:00025b24       ?$S12@?1??QueryDepthSListWrapper@@9@4@4IA 10044b24     vc_crt_fix_impl.obj
 0002:00025b28       ?Function@?1??GetNumaHighestNodeNumberWrapper@@9@4@4Q6GHPAK@ZA 10044b28     vc_crt_fix_impl.obj
 0002:00025b2c       ?$S13@?1??GetNumaHighestNodeNumberWrapper@@9@4@4IA 10044b2c     vc_crt_fix_impl.obj
 0002:00025b30       ?Function@?1??GetLogicalProcessorInformationWrapper@@9@8@4Q6GHPAU_SYSTEM_LOGICAL_PROCESSOR_INFORMATION@@PAK@ZA 10044b30     vc_crt_fix_impl.obj
 0002:00025b34       ?$S14@?1??GetLogicalProcessorInformationWrapper@@9@8@4IA 10044b34     vc_crt_fix_impl.obj
 0002:00025b38       ?Function@?1??SetThreadStackGuaranteeWrapper@@9@4@4Q6GHPAK@ZA 10044b38     vc_crt_fix_impl.obj
 0002:00025b3c       ?$S15@?1??SetThreadStackGuaranteeWrapper@@9@4@4IA 10044b3c     vc_crt_fix_impl.obj
 0002:00025b48       ?is_initialized_as_dll@@3_NA 10044b48     LIBCMT:utility.obj
 0002:00025b49       ?module_local_atexit_table_initialized@@3_NA 10044b49     LIBCMT:utility.obj
 0002:00025b4c       ?module_local_atexit_table@@3U_onexit_table_t@@A 10044b4c     LIBCMT:utility.obj
 0002:00025b58       ?module_local_at_quick_exit_table@@3U_onexit_table_t@@A 10044b58     LIBCMT:utility.obj
 0002:00025b64       ?__proc_attached@@3HA      10044b64     LIBCMT:dll_dllmain.obj
 0002:00025b90       _GS_ExceptionRecord        10044b90     LIBCMT:gs_report.obj
 0002:00025be0       _GS_ContextRecord          10044be0     LIBCMT:gs_report.obj
 0002:00025eac       ?__vcrt_startup_thread_ptd@@3U__vcrt_ptd@@A 10044eac     libvcruntime:per_thread_data.obj
 0002:00025ed4       ___vcrt_lock_table         10044ed4     libvcruntime:locks.obj
 0002:00025eec       ___vcrt_locks_initialized  10044eec     libvcruntime:locks.obj
 0002:00025ef0       ?module_handles@@3PAPAUHINSTANCE__@@A 10044ef0     libvcruntime:winapi_downlevel.obj
 0002:00025efc       ?encoded_function_pointers@@3PAPAXA 10044efc     libvcruntime:winapi_downlevel.obj
 0002:00025f3c       ?heap@@3V_HeapManager@@A   10044f3c     libvcruntime:undname.obj
 0002:00025f54       ?__acrt_new_handler@@3V?$dual_state_global@P6AHI@Z@__crt_state_management@@A 10044f54     libucrt:new_handler.obj
 0002:00025f58       ?c_termination_complete@@3JA 10044f58     libucrt:exit.obj
 0002:00025f5c       ?thread_local_exit_callback_func@@3P6GXPAXK0@ZA 10044f5c     libucrt:exit.obj
 0002:00025f68       ?program_name@?1???$common_configure_argv@D@@YAHW4_crt_argv_mode@@@Z@4PADA 10044f68     libucrt:argv_parsing.obj
 0002:00026098       ?__acrt_invalid_parameter_handler@@3V?$dual_state_global@P6AXPB_W00II@Z@__crt_state_management@@A 10045098     libucrt:invalid_parameter.obj
 0002:000260a8       ?__acrt_lock_table@@3PAU_RTL_CRITICAL_SECTION@@A 100450a8     libucrt:locks.obj
 0002:000261f8       ?__acrt_locks_initialized@@3IA 100451f8     libucrt:locks.obj
 0002:00026208       ?fSystemSet@@3HA           10045208     libucrt:mbctype.obj
 0002:0002620c       ?initialized@?1??__acrt_initialize_multibyte@@9@4_NA 1004520c     libucrt:mbctype.obj
 0002:00026430       ?module_handles@@3PAPAUHINSTANCE__@@A 10045430     libucrt:winapi_thunks.obj
 0002:00026480       ?encoded_function_pointers@@3PAPAXA 10045480     libucrt:winapi_thunks.obj
 0002:0002650c       ?ctrlc_action@@3V?$dual_state_global@P6AXH@Z@__crt_state_management@@A 1004550c     libucrt:signal.obj
 0002:00026510       ?ctrlbreak_action@@3V?$dual_state_global@P6AXH@Z@__crt_state_management@@A 10045510     libucrt:signal.obj
 0002:00026514       ?abort_action@@3V?$dual_state_global@P6AXH@Z@__crt_state_management@@A 10045514     libucrt:signal.obj
 0002:00026518       ?term_action@@3V?$dual_state_global@P6AXH@Z@__crt_state_management@@A 10045518     libucrt:signal.obj
 0002:0002651c       ?user_matherr@@3V?$dual_state_global@P6AHPAU_exception@@@Z@__crt_state_management@@A 1004551c     libucrt:matherr.obj
 0002:00026530       ?internal_state@?1??_mbtowc_l@@9@4U_Mbstatet@@A 10045530     libucrt:mbtowc.obj
 0002:00026540       ?__acrt_global_new_mode@@3V?$dual_state_global@J@__crt_state_management@@A 10045540     libucrt:new_mode.obj
 0002:00026544       ?__acrt_app_type@@3W4_crt_app_type@@A 10045544     libucrt:report_runtime_error.obj
 0002:00026548       ?internal_pst@?1??__mbrtoc32_utf8@__crt_mbstring@@YAIPA_UPBDIPAU_Mbstatet@@@Z@4U3@A 10045548     libucrt:mbrtoc32.obj
 0002:00026554       __pmatherr_set             10045554     libucrt:libm_error.obj
 0003:000008c6       .idata$6                   100468c6     kernel32:KERNEL32.dll
 0003:000009ae       .idata$6                   100469ae     user32:USER32.dll
 0003:00000a8e       .idata$6                   10046a8e     advapi32:ADVAPI32.dll
 0003:00000ad2       .idata$6                   10046ad2     ole32:ole32.dll
 0003:00000b0c       .idata$6                   10046b0c     mpr:MPR.dll
 0003:00000b56       .idata$6                   10046b56     version:VERSION.dll
 0003:00000b62       .idata$6                   10046b62     oleaut32:OLEAUT32.dll
 0004:00000060       $R000000                   10047060     ProcList.res
